:020000040000FA
:10000000480500203919000099190000C91700009F
:10001000C9170000C9170000C9170000C917000060
:10002000C9170000C9170000C9170000C11200005D
:10003000C9170000C91700006D12000085100000EC
:10004000F9180000F9180000F9180000F91800006C
:10005000F9180000F9180000F9180000F91800005C
:10006000F9180000F9180000F9180000F91800004C
:10007000F9180000F9180000F9180000F91800003C
:10008000F9180000F9180000F9180000F91800002C
:10009000F9180000F9180000F9180000F91800001C
:1000A000F9180000F9180000F9180000F91800000C
:1000B000F9180000F9180000F9180000F9180000FC
:1000C000F9180000F9180000F9180000F9180000EC
:1000D000F9180000F9180000F9180000F9180000DC
:1000E000F9180000F9180000F9180000F9180000CC
:1000F000F9180000F9180000F9180000F9180000BC
:10010000F9180000F9180000F9180000F9180000AB
:10011000F9180000F9180000F9180000F91800009B
:10012000F9180000F9180000F9180000F91800008B
:10013000F9180000F9180000F9180000F91800007B
:10014000F91800002DE9E04F2746A046A146A24637
:10015000A346A446A2B02DEC000A84F300882546ED
:100160002646A4473DEC000A22B0BDE8E08F00001F
:100170007BB972B90029BEBF00204FF0004106E0F4
:1001800008BF00281CBF6FF000414FF0FF3000F0A7
:10019000AFB9ADF1080C6DE904CE002909DB002BE5
:1001A0001ADB00F035F8DDF804E0DDE9022304B0E5
:1001B0007047404261EB4101002B1BDB00F028F847
:1001C000DDF804E0DDE9022304B0404261EB4101C7
:1001D000524263EB43037047524263EB430300F028
:1001E00017F8DDF804E0DDE9022304B0404261EBDA
:1001F00041017047524263EB430300F009F8DDF818
:1002000004E0DDE9022304B0524263EB430370478C
:100210002DE9F0478C46089D04468A46002B4AD1BA
:100220008A42174662D9B2FA82F64EB1C6F1200E62
:1002300001FA06F3B740B44020FA0EFE4EEA030A74
:100240004FEA1748230C1FFA87F9BAFBF8FE08FBA0
:100250001EAA0EFB09F243EA0A439A420BD9FB1885
:100260000EF1FF312CBF012000209A4202D9002854
:1002700000F02A818E469A1AA3B2B2FBF8F008FB6E
:10028000102200FB09F943EA0244A14507D93C19B1
:1002900000F1FF3302D2A14500F210811846A4EB11
:1002A000090440EA0E4000211DB1F4400023C5E9D5
:1002B0000043BDE8F0878B4208D9002D00F0F280A2
:1002C0000021C5E9000C0846BDE8F087B3FA83F1C8
:1002D00000294ED16345C0F0E880824240F2E580BB
:1002E0000846002DE5D0C5E9004AE2E702B9FFDE85
:1002F000B2FA82F6002E40F099808B1A4FEA124E25
:100300001FFA82F801214FEA144CB3FBFEF20EFBF8
:10031000123008FB02F94CEA004CE14508D917EB12
:100320000C0C02F1FF3302D2E14500F2CA801A46FA
:10033000ACEB090CA3B2BCFBFEF00EFB10CC08FB2F
:1003400000F843EA0C44A0450ED93C1900F1FF33F4
:100350002CBF4FF0010C4FF0000CA04503D9BCF1AD
:10036000000F00F0A8801846A4EB080440EA024001
:100370009AE7C1F120048B4002FA01FE0CFA01F663
:10038000E24020FA04F72CFA04FC00FA01F81343C7
:100390003E431F0C320C1FFA83F9BCFBF7F007FB3E
:1003A00010CC00FB09FA42EA0C4CE24508D913EBE9
:1003B0000C0C00F1FF3202D2E24500F289801046B7
:1003C000ACEB0A0CB6B2BCFBF7FA07FB1ACC0AFB83
:1003D00009F946EA0C42914506D99A180AF1FF3606
:1003E00001D291457AD8B2464AEA0040A2EB09020E
:1003F000A0FB0E67BA42B446B94602D307D1B04556
:1004000005D2B6EB0E0C67EB030301389946002DBD
:100410006BD0B8EB0C0362EB090202FA04F4CB4098
:10042000CA4000211C43C5E9004242E7B740C6F17B
:10043000200201FA06F3B44021FA02FC4FEA174EFB
:1004400020FA02F21FFA87F8BCFBFEF11A430EFBFA
:1004500011CC01FB08F0130C43EA0C4C604507D9A2
:1004600017EB0C0C01F1FF3301D2604533D819466C
:10047000ACEB000C92B2BCFBFEF00EFB10CC00FB10
:1004800008F342EA0C4C634507D917EB0C0C00F15A
:10049000FF3201D2634525D81046ACEB030340EA96
:1004A000014130E72946284603E7841A6CEB030331
:1004B00001209A4615E702383C4455E702383C448F
:1004C000EDE6023ABC4433E7AEF1020E3B44D2E61D
:1004D00002389C4474E70239BC44C9E7AAF1020A15
:1004E0001A4481E70238BC44D7E72946E1E600BF59
:1004F000704700BF830003F1A04303F54053D3F8D6
:10050000002810B4002A1BDAD3F8002802F00302F6
:10051000022A05D0D3F8002802F00302032A0FD1E3
:10052000012100F01F04A1404209074C203244F889
:100530002210BFF34F8FBFF36F8F044AC3F8002818
:10054000002110BC01F0E2B800E100E000010080F1
:100550008FB55C4800F094FB002440F217175A4E08
:100560005A4D04F5C073214646F8237028460134DD
:1005700000F086FB082CF4D140F20717524E544D80
:1005800004F5C073214646F823702846013400F074
:1005900077FB202CF4D14F4800F072FB002440F28E
:1005A0001717494E4C4D04F5E073214646F8237069
:1005B0002846013400F064FB082CF4D140F2071700
:1005C000414D464E04F5E073214645F82370304610
:1005D000013400F055FB202CF4D10024404800F0F9
:1005E0004FFBC5F8C0444FF480250520FFF782FF7C
:1005F0001520FFF77FFF2A20FFF77CFF3920FFF748
:1006000079FF3A20FFF776FF4220FFF773FF312092
:10061000FFF770FF0920FFF76DFF0A20FFF76AFF61
:100620001C20FFF767FF1D20FFF764FF2C20FFF75A
:1006300061FF0A20FFF75EFF0B20FFF75BFF0F2033
:10064000FFF758FF1020FFF755FF1120FFF752FF6B
:100650002968244800F014FB10222146684601F066
:10066000A9FB2B6868460093029500F04BF8012027
:1006700000F078F8204600F061F8204600F086F897
:100680000121204600F096F8174A1848D2F88C301D
:1006900043F44063C2F88C304FF004131C6800F040
:1006A000EFFA0820FFF726FF24F00104BFF34F8F75
:1006B000BFF36F8F6408640020462146224623461C
:1006C000FFF740FDFC2C0000003000501A2D000008
:1006D000452D00007A2D0000972D0000C72D000049
:1006E000FB2D00001F2E000000ED00E0372E000063
:1006F00040E800F313F4803FD8B208BF6FF0150054
:100700007047000082680C4B9A60036883F3888806
:10071000436883F38988027B02F00101EFF394833D
:1007200023F00303920748BF43F0020309B143F0EB
:10073000010383F39488704700ED02E0084AD36810
:1007400048B123F400531B041B0C43F0BF6343F474
:100750000033D36070479BB243F40053F5E700BF0A
:1007600000ED00E0084AD36840B19BB243F48043F7
:1007700043F0BF6343F40033D360704723F48043F6
:100780001B041B0CF4E700BF00ED00E0084AD3682F
:1007900040B19BB243F0080343F0BF6343F400331E
:1007A000D360704723F008031B041B0CF4E700BF61
:1007B00000ED00E0084B1A6818B142F001021A601F
:1007C000704722F001021A601A6811B142F0020269
:1007D000F5E722F00202F2E7D0ED00E070B50C255B
:1007E0004D43C66890F90B0074198842A8BF214692
:1007F0004FF0200492FBF4F4B8BF715902F01F00CF
:1008000001EB8401196070BD07B501ABFFF7E6FF8E
:100810000123019A03FA00F013680343136003B045
:100820005DF804FB2DE9F8430446FF2200214FF058
:100830000C0E4368058900685D4394F80AC028449B
:10084000E2728C4505DC00252389AB4222DCBDE841
:10085000F883B5FBF3F20EFB01F7D4F80C801F2AE6
:1008600008EB0706C8BF1F324FEA930306F10409DD
:10087000C8BF520903F10303C6E9019923F003033A
:10088000D4BFE17248F8070001F10101C8BF00EBD5
:100890008200D6E76268E3686A4320681E1D8118FB
:1008A00086509A6820464A609A68116099602A4684
:1008B0000021FFF7A9FF0135C6E708B50446084641
:1008C00011461A46A04701F0DBFE00F0F1FF0020C0
:1008D000704770B50D4604464520A0472946522072
:1008E000A04729462346BDE8704052201847000023
:1008F0000B6801330B60014B1B681847880E002002
:100900002DE9F04F85B00E9C9B46012CB8BF012409
:10091000012B0CBF30232023154680468946012633
:100920000A270022DFF870A0019402930AF1010463
:100930000AB9AA451ED2B5FBF4F049463030C0478B
:1009400001220136B5FBF4F10A23013F012F04FB1C
:100950001155BAFBF3FAE9D1494605F13000C04719
:10096000BBF1030F03D1019B9C1B002C0FDC05B0D6
:10097000BDE8F08F019BBB42E4DBBBF1020FE1D885
:100980004946029803920136C047039ADAE749467E
:100990002020C047013CE8E7FFC99A3B014B1860A3
:1009A000704700BF880E00202DE9F04F4FF0000A7D
:1009B00006460F464FF0FF39D04689B01C46531EFD
:1009C0000393002505E06DB9252800F03D813946E7
:1009D000B047039B13F8010F03930028F3D109B02C
:1009E000BDE8F08F642862D019D839280AD8312898
:1009F00051D22D283DD030283ED0252808D1394667
:100A0000B047DEE7582800F0A880632800F0168180
:100A100039462520B047039B39461878F0E77028FF
:100A200000F0918006D8692841D06C283CD0682815
:100A3000CFD0EDE775286DD017D87328E8D1256899
:100A400004F1040B2B461C4614F8010B002840F05F
:100A5000EC80B8F1030F40F000815C1BA9EB0404AB
:100A6000002C00F3E6805C46ABE7782875D07A2846
:100A7000DEE74FF00308ACE7B9F1000F0EDAB8F18A
:100A8000000F00F0E780A0F13009B8F1000F08BFB7
:100A90004FF002089DE7B9F1000FF4DB0A2303FBD6
:100AA0000909A9F13009F0E70AF1010A91E7BAF161
:100AB000000F12D125680434002D05DA39462D20A7
:100AC000B0476D4209F1FF3943462A46CDF8009000
:100AD00039463046FFF714FF73E7BAF1010FE9D04A
:100AE0004FF0000C4FF0FF3B073424F0070303F1F5
:100AF0000804D3E9002312F1004043F100018C45C2
:100B000008BF834504D239463046FFF7E2FE58E776
:100B10001546D1E7BAF1000F05D122680434CDF8AB
:100B200000904346D4E7BAF1010FF6D0073424F021
:100B3000070303F10804D3E90023002B08BFB2F137
:100B4000004FECD3DFE739463020B04739467820F4
:100B5000B0474FF008094FF00108BAF1010F27DC48
:100B60002368043407930023049310220023934640
:100B700002930693079B0BF1FF3B4FEA8B00C0F1FA
:100B8000200CA0F1200123FA00F0049B03FA0CFCD6
:100B900040EA0C0023FA01F1084310F00F0013D1D2
:100BA000069B13B9BBF1000F2ED14FF0300C11E0B2
:100BB000073424F007031A6803F108045B680792FE
:100BC0000493D2E7059AD5E709288CBF4FF0570C5C
:100BD0004FF0300C394660440592B047029B0695B1
:100BE00001330293BBF1000FECD1B8F1030F7FF496
:100BF000E8AE029BC3EB4905002D7FF7E2AE394614
:100C00002020B047013DF7E7531E91450593E9DBEE
:100C1000B8F1010F03D139463020B047E2E7B8F10F
:100C2000020FDFD139462020F7E73946B047234687
:100C300009E739462020B047013C11E72068251D0F
:100C40003946B0472C46BCE6AA46A8464FF0FF39C5
:100C50000125BEE64FF00108BBE65C460546B8E656
:100C6000002313B502AC44F8043D02460B4603488A
:100C70002146FFF799FE02B010BD00BFF108000049
:100C80000FB407B504A951F8040B0191FFF7E8FF71
:100C900003B05DF804EB04B07047704710B54FF037
:100CA0002003EFF3118483F3118800F011F801227F
:100CB000054BC3F840254FF0FF32044B9A62DA62CD
:100CC00084F31188002010BD0090035000ED00E077
:100CD0004D4A136843F0020313600022D30003F56A
:100CE0007F03D3F80013013108D0D3F80013013289
:100CF000D3F80433B2F5807F0B60EFD1434AD36958
:100D000013F001033BD0424B1946D3F80024012ACB
:100D1000FBD1C3F80425D1F80034012BFBD13B4BA8
:100D2000DA69D20708D5DA69394922F00102DA61B5
:100D3000D1F80024012AFBD11A6A01320AD11A6AB9
:100D400022F0FF0242F020021A62314AD2F8003447
:100D5000012BFBD100222E4BC3F80425D3F800242D
:100D6000012AFBD1BFF34F8F2A492B4BCA6802F4EB
:100D7000E0621343CB60BFF34F8F00BFFDE7126A01
:100D80000132C0D0254A116809290AD124490968CD
:100D9000013901299EBF4FF05021C1F81431C1F82B
:100DA00018311368092B09D11D4B1B68012B01BF9A
:100DB0001C4A1360A2F63822C2F87835174B1A681D
:100DC000092A0BD1164A1268022A07D10021154AB6
:100DD00011600121A2F63822C2F878151B68092B90
:100DE00006D10F4B1B68022B02BF0C220E4B1A6060
:100DF000084AD2F88C3043F44063C2F88C300B4B75
:100E00000B4A1A60704700BFD0ED00E00080FF0081
:100E10000090035000ED00E00400FA053001FF00EF
:100E20003401FF00384A0050E4AE03508C0E00201D
:100E30000090D0030A2838B50446074D04D128682D
:100E40000D2143685B6898472868E1B243685B6896
:100E50009847204638BD00BF0000002010B5044C64
:100E6000204600F0CBFF2046BDE81040FFF796BDBE
:100E7000350E000008B5044801F0FEF8034B186079
:100E8000FFF7ECFF002008BDA32E000000000020AB
:100E900010B54FF02003EFF3118283F31188114C4A
:100EA000237823B982F311886FF0440010BD013B11
:100EB000DBB2237023B182F311886FF00F00F5E7E6
:100EC000094B0121187828B1217082F311886FF045
:100ED0000A00EBE7197082F31188044A1160187058
:100EE000E4E700BF06000020050000200450005089
:100EF00010B54FF02002EFF3118382F31188124CEA
:100F0000207888B183F311884FF05022D2F81C3436
:100F1000D2F8182403F0030343F48033934314BF3F
:100F20006FF04300002010BD0122227083F311886E
:100F30004FF05023C3F80401C3F818150221C3F879
:100F400004139A60E0E700BF040000204FF0502334
:100F500030B5D3F80851D3F80423D3F8004102F098
:100F60000102D3F80413D3F8040115B10025C3F826
:100F70000851B4B14FF050230024C3F8004122B10E
:100F80004FF050230122C3F8082348B100224FF04C
:100F90005023C3F804218A0702D50222C3F808238C
:100FA00030BD002AF1D04FF05023D3F80C3403F0B9
:100FB0000113B3F1011FE8D1E2E708B500220121D6
:100FC000052000F089FB052000F062FB002008BD31
:100FD000F8B54FF02002EFF3118382F31188264A0F
:100FE0001078441C147070B183F311884FF05023B3
:100FF000D3F80C3403F00113B3F1011F0CBF002030
:101000006FF0430007E01D4D2F782FB1107083F370
:1010100011886FF00A00F8BD01262E7083F3118845
:101020004FF0502421B3052000F042FBC4F80071BA
:10103000D4F80433C4F804632660D4F800219AB1CC
:101040000022DB0758BF0123C4F800214FF0200223
:1010500058BFC4F808330A4B0520C3F8802100F0BC
:1010600017FB00232B70C1E720BF40BF20BFE4E780
:10107000C4F800112660F4E70600002005000020F7
:1010800000E100E07047704700220E4B10B4C3F837
:1010900040214FF02002EFF3118482F31188D3F83E
:1010A000040540F24713084A1168401A20F07F40B7
:1010B000B0FBF3F003FB0013136084F3118810BC42
:1010C00001F080BC005001500800002038B51A48DB
:1010D00000F0D2FF60B3436801211B6898470024E9
:1010E00040F24713154D4FF40012C5F80845C5F8F6
:1010F00040354FF48033C5F84433C5F80433104B02
:1011000001211C600F4B1520C3F88021224600F0FE
:10111000E3FA152000F0BCFA012320460A4A1360C6
:101120002B60D5F8043503F24713C5F8403538BDB8
:101130004FF0FF30FBE700BFC42E0000005001500D
:101140004051015000E100E0085001504CF66A03A4
:10115000B0F1FF3F08BF184601389842A8BF1846B3
:1011600040F2471220EAE07000FB0220164B30B537
:10117000984228BF18464FF02003EFF3118483F301
:101180001188124B1249D3F8043509685B1A23F011
:101190007F43B3F5A27F10D3B3F5A37F07D9B3FB89
:1011A000F2F56A439B1AB3F5A27F104401D300F213
:1011B0004710054B984228BF1846044B0844C3F813
:1011C000400584F3118830BD66FFFF0000500150D8
:1011D000080000204FF02002EFF3118382F3118802
:1011E000074AD2F80405074A1268801A40F24712EB
:1011F00020F07F40B0FBF2F083F31188704700BF0E
:10120000005001500800002004488168406A88426C
:1012100003D003494FF080520A607047FC00002061
:1012200004ED00E0002320210348C2180133412BC4
:1012300082F80013F9D1704700E100E0084A09493B
:10124000936809685866996607494B6843F080536C
:101250004B60002383F311889368986E704700BF3A
:10126000FC000020AC34000000ED00E0202080F302
:10127000118811498A684FF028001044EFF3098C57
:1012800080E8F01F0D4F4FF000664A6A8A603E60AA
:10129000506E0023536680F3118804B506488068B9
:1012A00000F0AAFBBDE8044002F1280090E8F01F1E
:1012B0008CF3098870470000FC00002004ED00E07A
:1012C0001EF0040F0CBFEFF30880EFF30980816973
:1012D00031F8021C11F0FF010229FFD001B500F026
:1012E000B7FA01BD38B51B4C05461B48FFF7C8FCD3
:1012F000A36AD90602D51948FFF7C2FCA36A1A07E8
:1013000002D51748FFF7BCFCA36A9B070ED515480A
:10131000FFF7B6FC616BA36A180607D51248FFF702
:10132000AFFC1DB1A36A23F08003A362094CA36A3A
:10133000DA0702D50D48FFF7A3FCA36A9B0602D586
:101340000B48FFF79DFCA36AA36A002043F0FF034C
:10135000A36238BD00ED00E0883000009F3000003F
:10136000D3300000E73000000031000017310000EA
:101370003731000038B51E4C05461E48FFF780FC8B
:10138000A36AD90402D51C48FFF77AFCA36A1A05A0
:1013900002D51A48FFF774FCA36A9B050ED51848BE
:1013A000FFF76EFCA16BA36A180407D51548FFF779
:1013B00067FC1DB1A36A23F40043A3620C4CA36A2B
:1013C000590502D51048FFF75BFCA36ADA0509D579
:1013D0000E48FFF755FC064A0020936A43F47F430A
:1013E000936238BDA36A9B04F5D50948F1E700BFB5
:1013F00000ED00E0E22E0000F92E0000D3300000E6
:101400000B2F0000252F00003B2F0000572F00005E
:101410003731000010B51C4C1C48FFF731FCA36AA3
:101420009A0102D51A48FFF72BFCA36ADB0102D50B
:101430001848FFF725FCA36ADC0202D51648FFF71F
:101440001FFC114CA36A180302D51448FFF718FCBF
:10145000A36A590302D51248FFF712FCA36A9A0344
:1014600002D51048FFF70CFC074CA36ADB0302D53A
:101470000D48FFF705FCA36A00206FEA03436FEAFB
:101480001343A36210BD00BF00ED00E0473200002F
:1014900060320000743200008F320000BA32000067
:1014A000D9320000FF3200001A33000010B51A4C88
:1014B0001A48FFF7E5FBA1696369580602D5184889
:1014C000FFF7DEFB6369D90707D51648FFF7D8FB9E
:1014D000636943F0FF03636110BD63699A0701D537
:1014E0001148F3E763695B0701D51048EEE76369CC
:1014F000180701D50E48E9E76369D90601D50D48FB
:10150000E4E763699A0601D50B48DFE763691B06C8
:10151000DED50A48DAE700BFD0ED00E06731000011
:101520008131000092310000A9310000C831000073
:10153000E4310000023200001832000033320000B3
:10154000F8B5404B06465F6801F07F43B3F17F4F2B
:101550000D4663D111F0010417D011F0400423D1DE
:101560000168394B0B44012B98BF016C3748FFF7DA
:1015700087FB15F00805334B0DD0EFF389865B68C8
:10158000180511D43248FFF77BFB31462046BDE8F1
:10159000F84000F02BB9EFF388865B68190503D596
:1015A0002B48FFF76DFB39E0C7F30807FA1E092A3D
:1015B0003CD8DFE802F005353727313B3B3B3B3970
:1015C0002448FFF75DFB1F4BDA6A920701D52248DA
:1015D000E7E7DC6A14F08044D7D02048FFF750FBDF
:1015E0001F4B1B781BB10120FFF77CFE0CE01D4B4D
:1015F0001B781BB10120FFF7BDFE05E01A4B1C88CC
:10160000A5B22DB1FFF706FF06280446BDD1F8BDEF
:10161000164B5C69002CB8D0FFF748FF0024B4E7F4
:101620000020E1E70020E6E71148BAE71148124937
:10163000A7F110020F2FD8BF01461048FFF720FB7B
:10164000ECE700BF00ED00E0A6ED05019E2F0000D5
:10165000BE2F0000E32F0000FB2F00001D30000014
:1016600028ED00E029ED00E02AED00E0D0ED00E0FB
:101670003D300000702F0000852F00007430000006
:10168000024A536943F010035361704700ED00E0D4
:1016900043B2002B08DB012200F01F0002FA00F029
:1016A000024A5B0942F82300704700BF00E100E0F6
:1016B00043B2002B0DDB012200F01F0002FA00F004
:1016C0005B09044A203342F82300BFF34F8FBFF376
:1016D0006F8F704700E100E043B2002B01F1010180
:1016E000A8BF03F160434FEA4111B8BF054BC9B22F
:1016F000ABBF03F5614300F00F0083F800131954EA
:10170000704700BF14ED00E000F05EB843B2A9B12D
:10171000002B12DB01215B099B0003F1604303F501
:101720006143D3F8802200F01F0001FA00F022EAA2
:101730000000C3F88002D3F880327047002BFCDB36
:1017400001225B099B0003F1604303F56143D3F879
:10175000801200F01F0002FA00F00843E9E70000E1
:10176000F8B516460C461F4604220A9B0999054601
:1017700001F064F80023A6F120010C4A214421F075
:10178000070122F00102C5E91333C5E916468A6153
:10179000069A0F604A60079A8A60089ACA604FF0FA
:1017A0008072CA61A9646B66F8BD00BFBB08000007
:1017B000014910220A60704710ED00E0404080F3BC
:1017C000118830BF704700BF404080F311884FF050
:1017D00004007146014202D0EFF3098001D1EFF31A
:1017E0000880714601B5FFF7ABFE01BD38B5044670
:1017F0000D4605281AD8DFE800F00319191315174C
:101800000D48FFF73DFA00F03BFFAA6901460B487F
:10181000FFF736FA29462046BDE8384000F01CB8EC
:101820000748EEE70748ECE70748EAE701460748BC
:10183000FFF726FAE7E700BF46330000E433000075
:10184000663300008C330000A6330000C133000073
:1018500001460068FFF7CABF052810B50CD000F09C
:101860001FFF60B100F01CFF0C490D4B002808BFA2
:1018700019460C48FFF704FAFFF7A0FFFCE700F059
:101880001FFF0028EED1084C0848A168FFF7F8F9BF
:10189000A068BDE8104000F00BB800BF2034000085
:1018A0002434000035340000FC00002055340000D2
:1018B00038B505464FF02003EFF3118483F3118808
:1018C00000F040FF0A4B9B68AB420BD1094B5A68B2
:1018D000C2F3080212B92046FFF7B0FC5A6842F082
:1018E00080525A602046BDE8384000F054BD00BF29
:1018F000FC00002000ED00E001B572B60B4A106A52
:1019000000281EBF0021116200F0DCFB62B6EFF37D
:101910000580A0F110004FEAC0000549014409C943
:101920009847BDE80140034800470000FC00002044
:10193000942A00000912000000F006F800F008F8F0
:1019400030BFFFF7FDBF00BF202383F3118870472E
:1019500008B50E4B83F30988EFF3148343F00203B9
:1019600083F31488BFF36F8F094B0A4A23F07F0378
:101970009360BFF34F8FBFF36F8F00F0BDFB00F09C
:10198000C5FBFFF74FFC00F0F3FB00BF880E002003
:101990000000000000ED00E008B5FFF7D1FFBDE852
:1019A0000840FFF731BC000010B50D4B86B0009326
:1019B0000C4B0D4C01930D4B0D4A02936846234688
:1019C000012100F049F9002305930A4B0121E41A93
:1019D00003A80393049400F049F906B010BD00BFBA
:1019E00000000020000000000000012006000100AF
:1019F000000000200000002007B5002101A800F031
:101A00007BF903B05DF804FB10B50B680C7A23F08A
:101A10001F0304F01F021A43CB68640923F01F035D
:101A2000044943F0010343EA44038860CA600B6140
:101A300010BD00BF90ED00E030B585B09DF80820E6
:101A40000D890B684C68498965F3040261F34712FC
:101A500000938DF8082023F01F03621E134423F027
:101A60001F030393084B04461B68C3F30723013B82
:101A7000984205DC6946FFF7C7FF204605B030BD38
:101A80006FF01504F9E700BF90ED00E02DE9F04F8D
:101A90000E46144680460025504F85B0B54209DAFF
:101AA000D8F80490B9F1000F39D0B9F11F0F05D85B
:101AB0006FF01504204605B0BDE8F08F19F01F0F38
:101AC000F6D1D8F800A01AF01F0FF1D15046FEF75A
:101AD0000FFE834609EB0A000138FEF709FE834535
:101AE000E6D11BF1160FE3D0631E5B45E0DBC7F8C0
:101AF00008B0F968C7F808B03B6921F01F0143F04E
:101B00001F0AD8E900321A44994202F1FF391CD168
:101B1000CA4508D141465FFA8BF0FFF78DFF0135CA
:101B200008F10C08BAE74146C7F808B0FB6822F094
:101B30001F0203F01F031A43FA60E0B2FFF77CFFB5
:101B400010F1160FB4D0441CE9E7013BCA45E0B2DE
:101B500023F01F03C7F808B006D13A69414602F0E6
:101B60001F0213433B61E9E7396901F01F010B4391
:101B70003B614146FFF760FF10F1160F98D0C7F8A0
:101B800008B0FA689DF80830441C62F304038DF82D
:101B900008303B699DF808205B0863F347128DF815
:101BA0000820D8E900210A4400920AF1FF3322F00C
:101BB0001F021344A3EB090323F01F0303933B68A5
:101BC000E4B2C3F30723013BA342FFF671AF204603
:101BD0006946FFF719FF0134A1E700BF90ED00E06F
:101BE0000522034B5A60BFF34F8FBFF36F8F7047CF
:101BF00090ED00E0BFF35F8F0022014B5A60704709
:101C000090ED00E0104970B5104D0A682E68C2F3DF
:101C10000722964214D8FFF7EDFF00240C4B0B630C
:101C2000A64205D10B4B1E70FFF7DAFF002070BDF6
:101C30006968204601EB0411FFF7E6FE0134EFE787
:101C40004FF0FF30F3E700BF90ED00E06C2E000096
:101C5000AAFF44002000002010B5034C2278FFF7B3
:101C600015FF207010BD00BF200000202DE9F84FA7
:101C70008846064600251D4F1D4C454501DBBDE845
:101C8000F88FD6F804A0BAF1000F2CD0D6F800B027
:101C90005846FEF72DFD81460AEB0B000138FEF792
:101CA00027FD1423814518BF6FF01500114A6B43BF
:101CB0001278C0B28242D855E1D9A0603B44A060FE
:101CC000E068197B60F3040119732169187B4908E6
:101CD00061F347101873E26822F01F025A6022690C
:101CE00022F01F021A6101350C36C6E70C000020F5
:101CF00090ED00E02000002070B50E4B0E461C78E1
:101D00000022234605460C480168C1F307218B4297
:101D10000BDB0A4911F8040BFFF776FE2246314629
:101D20002846BDE87040FFF7B1BE83600261013311
:101D3000EAE700BF2000002090ED00E00C0000204A
:101D40000138013910F8013F11F8012F934202D1F7
:101D5000002BF7D11A46981A7047F0B581EA0004B3
:101D6000A50703460BD0013B0A4491421DD1F0BDAB
:101D7000002AFCD011F8014B013A03F8014B9C07F3
:101D8000F6D10C461D1F8F183E1B032E08D86FF08E
:101D90000305940805FB0422A40023442144E2E740
:101DA00054F8046B45F8046FEEE711F8014B03F8A3
:101DB000014FDAE70346F0B5C9B29C070FD11D46C3
:101DC00041EA012444EA04449F187E1B032E0CD8E8
:101DD000940803EB840413449C4209D1F0BD002A0B
:101DE000FCD003F8011B013AE7E745F8044BECE7A8
:101DF00004F8011BF0E74FF0FF307047014B18600B
:101E0000704700BF900E002070B54B79012B23D195
:101E10008B79032B20D1CC792CB1012C1CD10368F8
:101E20009B681B79C3B10A7912B1022A14D10E2220
:101E300047F6122603689B681D680B68B3426BD097
:101E400027D8B3F5965F61D012D8B3F5167F4DD081
:101E500005D8B3F5967F74D06FF0220052E0B3F549
:101E6000966F50D0B3F5166FF6D14FF41D233FE0B7
:101E7000B3F5615F4CD004D8B3F5165FECD1324BAB
:101E800036E0B3F5964F45D0B3F5E14FE4D12F4B93
:101E90002EE0B3F5E13F48D012D84DF6C026B3424C
:101EA0003DD005D8B3F5164FD6D14FF41D031FE032
:101EB000B3F5614F36D0B3F5963FCDD1244B17E043
:101EC000B3F5E12F37D008D8B3F5613F30D0214EBC
:101ED000B342C1D14FF080630AE0B3F5612F2DD03A
:101EE0001D4EB342B8D14FF0805301E04FF41C3384
:101EF000C5F824358368224303C9C5F86C2583E8F7
:101F00000300002070BD4FF49E23F1E7134BEFE771
:101F1000134BEDE7134BEBE74FF40003E8E74FF407
:101F20006503E5E74FF46B03E2E74FF0EB73DFE7A0
:101F30004FF06C73DCE74FF0E863D9E74FF0706364
:101F4000D6E74FF4A033D3E70050270000C0750058
:101F500000903A0190D0030040420F0000B01300FF
:101F600000F03A0000A04E000B46826892E80300A1
:101F700083E8030000207047036882689B681B6841
:101F8000D3F8100138B1127A00200A700122C3F888
:101F900010011A6070474FF0FF30704782B002AAFC
:101FA00002F8011D002103689B681B68C3F820111B
:101FB000C3F844250122C3F848259A60D3F82011BC
:101FC0000029FBD0DA6002B0704703689B681B6889
:101FD000D3F8240118B1D3F88004C3F88004704703
:101FE000026870B59268184B14684FF0005285680B
:101FF00003219A601D260022C3F87412C3F87022D0
:10200000C4F80C651C26C4F814654FF000669E6089
:10201000C3F86C12C3F868221B23C4F808351A23CE
:102020002946C4F81035FFF7EFFE58B90823C4F865
:1020300000351D440123C4F81001C4F83455C4F818
:102040003835236070BD00BF0025845070B5002670
:10205000084B53F82040013053F82050A54200D8D7
:1020600070BD236820465B68984700B166600C34F9
:10207000F4E700BF98340000104B70B505461E46CB
:102080000F4C9C4204D10E4CB44209D1002412E002
:1020900062681AB122681268AA420CD00C34F0E7C8
:1020A00063680BB90C34EFE7236828461968FFF71B
:1020B00047FE0028F6D1204670BD00BF080F002063
:1020C000A80E0020FEF7DFBF08B50A4D4FF0200232
:1020D000EFF3118382F3118800F052FC01210446D2
:1020E0000228D8BF084600F057FC2C62FFF766FBB9
:1020F000ECE700BFFC0000200248034A0021121A4E
:10210000FFF758BE000000204801002008B506482F
:10211000064A0749121AFFF720FEBDE80840054AA3
:1021200005490648FFF719BE880E00201C0F002045
:102130000035000000000000003500000000002015
:1021400008B50220FFF782FF0748FEF799FD03203C
:10215000FFF77CFF00F016FBFEF7FAF9034A137B4A
:1021600023F00103137308BDC03400009000002069
:1021700080B53F4BA2B083F308880024E0223D4B9A
:10218000012783F82220DC771C765C769C76DC764F
:102190005A6A394E42F4E0225A625A6A374D42F482
:1021A00000225A629C63DA6892B242F0BF6242F443
:1021B0000832DA60FFF764FAFFF7FAFA07AB6C222D
:1021C00021461846FFF7F6FDB06020468DF82970CD
:1021D000FFF73CFF3846FFF739FF00F045FA284B80
:1021E0004FF48062CDE90473CDE90244254BCDE97B
:1021F000004425492846756200F08AFA6B7B23F07B
:10220000040213F01B0F6A7304D1AB6913B928469B
:1022100000F038F91D4B0024059301220F231C4FB9
:10222000CDE903321B494FF4A0723846CDE9014491
:102230000094194B00F06CFA7B7BF76023F00403E9
:102240007B73164BC6E90633FFF7AEFBB560144B44
:1022500083F3098862B661B684F311880748FFF7F3
:10226000CBFB2346224621460648FEF726FB00BF4D
:10227000880E002000ED00E0FC000020900000200F
:10228000B03400004121000048010020B5340000B6
:102290002400002048050020C9200000140100206F
:1022A00048050020437BDB0603BF8069B0FA80F05D
:1022B0004009002070470000EFF305800D2809D881
:1022C00028B1054B586880F40060C0F3C02080F04E
:1022D000010070470120FAE700ED00E008B5FEF7C5
:1022E00079FF054B054A1B68002118441061184608
:1022F000BDE8084000F050BB34010020FC00002085
:10230000F8B50D464FF02003EFF3118483F31188E5
:102310004FF40041002700220A4E0B4BC1FB00671F
:102320001A6130464FF4A02200233946FDF720FF02
:10233000064B1860064B1D60FFF7D0FF84F3118831
:10234000F8BD00BFFFFF0400FC00002034010020A6
:102350003001002038B504464FF02003EFF311851B
:1023600083F311880146806800F03AF8637B23F01C
:102370000203637385F311880023A36038BD08B599
:10238000FFF79AFF20B1BDE808400846FEF756BFA8
:1023900081F3118808BD08B50246FFF78DFF20B113
:1023A000BDE808401046FEF749BF82F3118808BD1A
:1023B0004FF02003EFF3118083F31188FFF7EBBF99
:1023C0004FF02003EFF3118183F31188034B9A68D8
:1023D000D37B013BD37381F311887047FC0000204D
:1023E000094B03F12802824205D19B688B4202D13E
:1023F0004B7BDB0607D1D1E900231A600A685360E2
:102400000023C1E900337047FC00002003689842B4
:1024100014BF18460020704738B50D4C024604F131
:102420002800FFF7F3FF054600B9E568A3684AB93D
:102430005A7BD20606D1AA6922B9DA897F2A01D944
:10244000636238BD9D4201D0FFF748FF6562F8E73F
:10245000FC00002010B54FF02003EFF3118483F34C
:102460001188074B01209A68D37B0133D373FFF7A0
:10247000D3FF84F31188BDE81040FFF799BF00BF78
:10248000FC000020F8B54FF02003EFF3118483F334
:102490001188154A114651F8283F8B420CD05BB188
:1024A000D66A90F90E5093F90E70AF420BDCB3422E
:1024B00002D01B68002BF6D1D36A01604360D36A57
:1024C0001860D06205E05A68C0E900325A681060AE
:1024D0005860437B43F0400343730020FFF79CFFA9
:1024E00084F31188F8BD00BFFC00002050F8103CB8
:1024F00070B50446A0F11805ABB14FF02003EFF31F
:10250000118683F31188294650F8100CFFF768FFF5
:1025100014F80B3C23F0020304F80B3C86F31188FB
:10252000002344F8103C14F80B3C284623F0040325
:1025300004F80B3CFFF7B6FE20B12846BDE870401A
:10254000FFF7A0BF70BD0000F8B504464FF02003B0
:10255000EFF3118683F31188184F014607F1280520
:102560002846FFF73DFFBB6A3A46AB420CD05BB151
:10257000F86A94F90E1093F90E708F420BDC8342C7
:1025800002D01B68002BF6D1D36A25606360D36A42
:102590001C60D46205E05968C4E9003159680C60D8
:1025A0005C60637B906843F040036373031B584295
:1025B0005841FFF731FF86F31188F8BDFC00002079
:1025C00010B51449144C8B68226893424FF00002F6
:1025D000226003D1BDE81040FFF780BE0F4A1268A9
:1025E000BAB1DA897F2A14D80D4A93F90E401268DD
:1025F00094420EDB0B4A126893420AD09A6942B9A0
:102600000A69824203DC1846FFF79EFFE2E7121ACE
:102610000A6110BDFC0000202C01002034010020C4
:1026200030010020BC34000070B504464FF0200398
:10263000EFF3118683F31188437B5A060FD5094DBA
:10264000014605F12800FFF7CBFE637BA86823F065
:1026500040036373031B58425841FFF7DDFE86F3C6
:10266000118870BDFC0000200021044B084603F1D6
:102670002802C3E90A22FFF743BE00BFFC00002086
:10268000014B9868704700BFFC000020437BDB06CD
:1026900003BF8069B0FA80F0400900207047000055
:1026A000EFF305800D2807D838B1044B586880F443
:1026B0000060C0F3C02070470120704700ED00E0CB
:1026C000024B9B68187B00F001007047FC00002063
:1026D00010B502464FF02003EFF3118483F3118805
:1026E000437B590702D484F3118810BD23F00403FF
:1026F0004373FFF7CBFF10B11046FFF7C3FE21462F
:10270000BDE810400148FFF73ABE00BF3801002085
:1027100030B587B00E9D044604950D9D03950C9D24
:1027200002950B9D01950A9D0095FFF719F8044B42
:102730009B6813B9236607B030BD1B6EFAE700BF74
:10274000FC000020036D10B5044603B198472046F5
:10275000FFF79CFF38B12046FFF766FF637B43F02D
:102760000803637310BD637B9B0702D52046FFF708
:10277000F1FDA369002BF1D004F1180000F0EEF890
:10278000ECE700002DE9F04F284E294DB04687B008
:10279000B54205F130040FD3FFF712FE4FF40049A4
:1027A0000027234C234EDFF890A0444521D307B0E7
:1027B000BDE8F04FFFF74EBE54F8043C059354F8C3
:1027C000103C049354F8143C039354F8183C0293BF
:1027D00054F81C3C019354F8203C009354E90A231C
:1027E00054E90C01FFF794FF54F8303CDD642546B2
:1027F000CEE7616A4B1C04D0256821B92846FFF753
:1028000067FF3034D1E7B346BC46C9FB01BC4FF487
:10281000A022002358466146FDF7AAFC5146421CFF
:1028200005F1180000F05AF8EBE700BF080F002090
:10283000080F0020FFFF0400ED24000003730023B5
:1028400042738173C373C0E906337047034B1B683F
:102850000BB9FEF7BFBC0020704700BF3801002055
:10286000036840B1084A5268904204D01BB19A688C
:1028700081680A449A604268136003685A600023C2
:10288000C0E90033704700BFA00E002038B5104BE0
:102890001B78002B0F4B18BF4FF0FF301C6808BF90
:1028A0006FF000409C420AD04CB1A568FFF7CEFF04
:1028B000281A00280ADBA468FFF7C8FF201A064B75
:1028C0001B6913B19842A8BF184638BD0020F6E72F
:1028D0003C010020A00E0020FC00002070B5044642
:1028E0001646C1604FF02003EFF3118583F3118882
:1028F000FFF7ACFF012EACBF80190130164BA06072
:102900001A689A4201D05E6832B95A6823606260E0
:102910005A6814605C600BE09068A168884214DD1E
:10292000411A91605168C4E9002151680C605460FB
:102930001A689A4206D0944204D1FFF7A7FF0021FB
:10294000FEF704FC85F3118870BD091A9642A16058
:10295000DBD01268D8E700BFA00E002010B54FF002
:102960002002EFF3118482F3118803682BB1FFF783
:1029700077FF002084F3118810BD6FF01500F9E790
:1029800010B54FF02003EFF3118483F31188FFF7A4
:102990007DFF84F3118810BD70B504460E464FF0DC
:1029A0002003EFF3118583F31188FFF76FFFA04237
:1029B00005DD012803DD31462046FEF7C7FB85F320
:1029C000118870BD2DE9F04B0446FFF7F9FD4FF07B
:1029D0002003EFF3118583F311881E4F1E4EB84676
:1029E000DFF878903460D9F8004032684C45D7E978
:1029F00000BC05D024B1A368934212DD9B1AA360EA
:102A000000241BEB02004CEBE271C8E900013460CA
:102A1000FFF73CFF2146FEF799FB85F31188BDE8DF
:102A2000F08B1BEB03004CEBE371D31A33600023F4
:102A3000C7E90001A3602046FFF712FF85F3118864
:102A4000E36898474FF02003EFF3118583F3118873
:102A5000C9E700BF4001002038010020A00E00207F
:102A600038B5074C074DAC4201D3002038BD04F106
:102A700014032046C4E90533FDF7D4FE1C34F2E705
:102A8000080F0020080F00207047FFFF84D7FF7F4A
:102A90000100000000000000091700000000000015
:102AA00009170000000000000917000000000000E6
:102AB00009170000000000000917000000000000D6
:102AC0004D0F00000000000009170000000000008A
:102AD00009170000000000000917000000000000B6
:102AE00009170000000000000917000000000000A6
:102AF0000917000000000000091700000000000096
:102B00000917000000000000091700000000000085
:102B10000917000000000000091700000000000075
:102B20000917000000000000091700000000000065
:102B30000917000000000000091700000000000055
:102B400089100000000000000917000000000000CC
:102B50000917000000000000091700000000000035
:102B60000917000000000000091700000000000025
:102B70000917000000000000091700000000000015
:102B80000917000000000000091700000000000005
:102B900009170000000000000917000000000000F5
:102BA00009170000000000000917000000000000E5
:102BB00009170000000000000917000000000000D5
:102BC00009170000000000000917000000000000C5
:102BD00009170000000000000917000000000000B5
:102BE00009170000000000000917000000000000A5
:102BF0000917000000000000091700000000000095
:102C00000917000000000000091700000000000084
:102C10000917000000000000091700000000000074
:102C20000917000000000000091700000000000064
:102C30000917000000000000091700000000000054
:102C40000917000000000000091700000000000044
:102C50000917000000000000091700000000000034
:102C60000917000000000000091700000000000024
:102C70000917000000000000091700000000000014
:102C80000917000000000000091700000000000004
:102C9000091700000000000009170000B932000009
:102CA0009D0C000000000000B9320000750E00000D
:102CB00000000000C42E0000BB0F00000000000058
:102CC000CE2E0000BB0F000000000000D82E000038
:102CD000CD10000000000000B9320000051C00000B
:102CE00000000000A32E0000E11F0000903400004F
:102CF000B9320000612A00000000000053656375CE
:102D0000726520426F6F743A20636F6E66696775F3
:102D1000726520666C6173680A005365637572653D
:102D200020426F6F743A205350553A2073657420D7
:102D3000726567696F6E2025752061732053656326
:102D40007572650A0053656375726520426F6F7412
:102D50003A205350553A2073657420466C6173686D
:102D600020726567696F6E202575206173204E6F34
:102D70006E2D5365637572650A00536563757265E0
:102D800020426F6F743A20636F6E66696775726573
:102D9000205352414D0A0053656375726520426F9E
:102DA0006F743A205350553A207365742053524142
:102DB0004D20726567696F6E202575206173205301
:102DC00065637572650A0053656375726520426FAD
:102DD0006F743A205350553A207365742053524112
:102DE0004D20726567696F6E202575206173204ED6
:102DF0006F6E2D5365637572650A00536563757256
:102E00006520426F6F743A20636F6E6669677572F2
:102E100065207065726970686572616C730A005331
:102E2000656375726520426F6F743A204D53505F31
:102E30004E532025780A0053656375726520426FF2
:102E40006F743A207072657061726520746F206AC9
:102E5000756D7020746F204E6F6E2D5365637572A3
:102E60006520696D6167650A0000000002000000CE
:102E7000742E000000000000942E000006000000E8
:102E8000E0FF0F00000000209C2E00002100000049
:102E9000E0FF0020464C4153485F30005352414D03
:102EA0005F3000554152545F30000000F10E0000C9
:102EB0000000000000000000D10F0000910E000093
:102EC00000000000434C4F434B5F33324B00434CF8
:102ED0004F434B5F31364D007379735F636C6F63A3
:102EE0006B002A2A2A2A2A20425553204641554C53
:102EF00054202A2A2A2A2A0A002020537461636B4C
:102F0000696E67206572726F720A002020507265C8
:102F100063697365206461746120627573206572F2
:102F2000726F720A0020204246415220416464724E
:102F30006573733A20307825780A002020496D7037
:102F400072656369736520646174612062757320C2
:102F50006572726F720A002020496E737472756315
:102F600074696F6E20627573206572726F720A00E9
:102F7000526573657276656420457863657074691F
:102F80006F6E20280053707572696F757320696EBB
:102F90007465727275707420284952512000202087
:102FA0005320696E737472756374696F6E20616407
:102FB00064726573733A2020307825780A00524590
:102FC00054544F4241534520646F6573206E6F74B3
:102FD000206D61746368204558435F5245545552D3
:102FE0004E0A002A2A2A2A2A2048415244204641D1
:102FF000554C54202A2A2A2A2A0A00202042757376
:10300000206661756C74206F6E20766563746F72D4
:10301000207461626C6520726561640A002020463C
:1030200061756C7420657363616C6174696F6E2087
:10303000287365652062656C6F77290A002A2A2A41
:103040002A2A204465627567206D6F6E69746F72FD
:1030500020657863657074696F6E20286E6F7420C8
:10306000696D706C656D656E74656429202A2A2A05
:103070002A2A0A002A2A2A2A2A2025732025642996
:10308000202A2A2A2A2A0A002A2A2A2A2A204D50B5
:1030900055204641554C54202A2A2A2A2A0A002023
:1030A00020537461636B696E67206572726F722062
:1030B00028636F6E746578742061726561206D6934
:1030C000676874206265206E6F742076616C696435
:1030D000290A002020556E737461636B696E672046
:1030E0006572726F720A002020446174612041632E
:1030F000636573732056696F6C6174696F6E0A0043
:1031000020204D4D46415220416464726573733AEC
:1031100020307825780A002020496E737472756318
:1031200074696F6E204163636573732056696F6CB9
:103130006174696F6E0A002020466C6F6174696E5D
:10314000672D706F696E74206C617A792073746179
:10315000746520707265736572766174696F6E2034
:103160006572726F720A002A2A2A2A2A205345435E
:10317000555245204641554C54202A2A2A2A2A0ACB
:10318000002020416464726573733A20307825789A
:103190000A002020496E76616C696420656E747245
:1031A0007920706F696E740A002020496E76616C18
:1031B000696420696E7465677269747920736967E0
:1031C0006E61747572650A002020496E76616C69C3
:1031D0006420657863657074696F6E2072657475BC
:1031E000726E0A0020204174747269627574696F8E
:1031F0006E20756E69742076696F6C6174696F6E8C
:103200000A002020496E76616C6964207472616ED8
:10321000736974696F6E0A0020204C617A7920739B
:103220007461746520707265736572766174696F1C
:103230006E0A0020204C617A7920737461746520D5
:103240006572726F720A002A2A2A2A2A205553416F
:103250004745204641554C54202A2A2A2A2A0A004A
:1032600020204469766973696F6E206279207A65DF
:10327000726F0A002020556E616C69676E6564206C
:103280006D656D6F7279206163636573730A0020E9
:1032900020537461636B206F766572666C6F772064
:1032A00028636F6E746578742061726561206E6F3B
:1032B000742076616C6964290A0020204E6F2063B7
:1032C0006F70726F636573736F7220696E7374725F
:1032D000756374696F6E730A002020496C6C6567B2
:1032E000616C206C6F6164206F66204558435F52AB
:1032F000455455524E20696E746F2050430A002089
:1033000020496C6C6567616C20757365206F662061
:1033100074686520455053520A002020417474653A
:103320006D707420746F20657865637574652075A1
:103330006E646566696E656420696E737472756328
:1033400074696F6E0A002A2A2A2A2A204861726448
:103350007761726520657863657074696F6E202A85
:103360002A2A2A2A0A002A2A2A2A204B65726E65EE
:103370006C20416C6C6F636174696F6E204661698B
:103380006C75726521202A2A2A2A0A002A2A2A2AEA
:103390002A204B65726E656C204F4F505321202AB6
:1033A0002A2A2A2A0A002A2A2A2A2A204B65726EE9
:1033B000656C2050616E696321202A2A2A2A2A0A14
:1033C000002A2A2A2A20556E6B6E6F776E2046617E
:1033D00074616C204572726F7220256421202A2A44
:1033E0002A2A0A0043757272656E742074687265C9
:1033F0006164204944203D2025700A4661756C7443
:10340000696E6720696E737472756374696F6E207C
:1034100061646472657373203D20307825780A00FA
:1034200049535200657373656E7469616C207468EA
:103430007265616400466174616C206661756C74CC
:1034400020696E20257321205370696E6E696E6746
:103450002E2E2E0A00466174616C206661756C74B4
:1034600020696E2074687265616420257021204196
:10347000626F7274696E672E0A000000791F000087
:103480009D1F0000CB1F0000091E0000691F0000E7
:103490000080005001000000A80E0020FC0E00205B
:1034A000080F0020080F0020080F0020F5FFFFFF85
:1034B0006D61696E0069646C650000002400002085
:1034C0002A2A2A2A2A20426F6F74696E67205A6559
:1034D00070687972204F532076312E31332E39396E
:1034E0002D6E6373312D353032352D6737343533DA
:1034F0003236323636643963202A2A2A2A2A0A00CA
:10350000CF0800000090D003F71D000000C20100AA
:103510000001030000000000A00E0020A00E00200B
:103520009C2C00000000000000000000F02C0000B7
:103530000000000000000000D82C00000000000087
:1035400000000000B42C0000AC2E000000000000C1
:10355000C02C0000B82E000000000000E42C000089
:103560007C340000940E0020A82C00000000000015
:1035700000000000CC2C0000000000000000000053
:10358000080F0020080F00200000000000000000CD
:043590000F00000028
:020000040004F6
:10000000A0B10220093E0400AD3E0400693C04009A
:10001000693C0400693C0400693C0400693C04003C
:10002000693C0400693C0400693C0400C5370400D5
:10003000693C0400693C0400713704003135040058
:10004000C93D0400C93D0400C93D0400C93D040088
:10005000C93D0400C93D0400C93D0400C93D040078
:10006000C93D0400C93D0400C93D0400C93D040068
:10007000C93D0400C93D0400C93D0400C93D040058
:10008000C93D0400C93D0400C93D0400C93D040048
:10009000C93D0400C93D0400C93D0400C93D040038
:1000A000C93D0400C93D0400C93D0400C93D040028
:1000B0000D5604002F560400C93D0400C93D04003C
:1000C000C93D0400C93D0400C93D0400C93D040008
:1000D000C93D0400C93D0400C93D0400C93D0400F8
:1000E000C93D0400C93D040051560400C93D040047
:1000F000C93D0400C93D0400C93D0400C93D0400D8
:10010000C93D0400C93D0400C93D0400C93D0400C7
:10011000C93D0400C93D0400C93D0400C93D0400B7
:10012000C93D0400C93D0400C93D0400C93D0400A7
:10013000C93D0400C93D0400C93D0400C93D040097
:10014000C93D0400FFFFFFFF81F0004102E000BF56
:1001500083F0004330B54FEA41044FEA430594EA87
:10016000050F08BF90EA020F1FBF54EA000C55EAC2
:10017000020C7FEA645C7FEA655C00F0E2804FEA93
:100180005454D4EB5555B8BF6D420CDD2C4480EA75
:10019000020281EA030382EA000083EA010180EAA5
:1001A000020281EA0303362D88BF30BD11F0004FF3
:1001B0004FEA01314FF4801C4CEA113102D0404229
:1001C00061EB410113F0004F4FEA03334CEA133364
:1001D00002D0524263EB430394EA050F00F0A7807C
:1001E000A4F10104D5F1200E0DDB02FA0EFC22FA77
:1001F00005F2801841F1000103FA0EF2801843FA6B
:1002000005F359410EE0A5F120050EF1200E012A5B
:1002100003FA0EFC28BF4CF0020C43FA05F3C01899
:1002200051EBE37101F0004507D54FF0000EDCF112
:10023000000C7EEB00006EEB0101B1F5801F1BD3BB
:10024000B1F5001F0CD349085FEA30004FEA3C0CBF
:1002500004F101044FEA445212F5800F80F09A80B5
:10026000BCF1004F08BF5FEA500C50F1000041EBB9
:10027000045141EA050130BD5FEA4C0C404141EBBD
:10028000010111F4801FA4F10104E9D191F0000FE4
:1002900004BF01460020B1FA81F308BF2033A3F167
:1002A0000B03B3F120020CDA0C3208DD02F1140C5E
:1002B000C2F10C0201FA0CF021FA02F10CE002F199
:1002C0001402D8BFC2F1200C01FA02F120FA0CFC92
:1002D000DCBF41EA0C019040E41AA2BF01EB0451DB
:1002E000294330BD6FEA04041F3C1CDA0C340EDCD9
:1002F00004F11404C4F1200220FA04F001FA02F31C
:1003000040EA030021FA04F345EA030130BDC4F1D9
:100310000C04C4F1200220FA02F001FA04F340EACE
:100320000300294630BD21FA04F0294630BD94F07F
:10033000000F83F4801306BF81F480110134013D66
:100340004EE77FEA645C18BF7FEA655C29D094EAD7
:10035000050F08BF90EA020F05D054EA000C04BF55
:100360001946104630BD91EA030F1EBF0021002040
:1003700030BD5FEA545C05D14000494128BF41F0DF
:10038000004130BD14F580043CBF01F5801130BD43
:1003900001F0004545F0FE4141F470014FF00000CE
:1003A00030BD7FEA645C1ABF194610467FEA655C7F
:1003B0001CBF0B46024650EA013406BF52EA033521
:1003C00091EA030F41F4002130BD00BF90F0000F0F
:1003D00004BF0021704730B54FF4806404F132044B
:1003E0004FF000054FF0000150E700BF90F0000F04
:1003F00004BF0021704730B54FF4806404F132042B
:1004000010F0004548BF40424FF000013EE700BFFA
:1004100042004FEAE2014FEA31014FEA02701FBF8A
:1004200012F07F4393F07F4F81F06051704732F0BC
:100430007F4208BF704793F07F4F04BF41F4002113
:10044000704730B54FF4607401F0004521F0004171
:100450001CE700BF50EA010208BF704730B54FF0FB
:1004600000050AE050EA010208BF704730B511F0FC
:10047000004502D5404261EB41014FF4806404F134
:1004800032045FEA915C3FF4D8AE4FF003025FEABA
:10049000DC0C18BF03325FEADC0C18BF033202EB3E
:1004A000DC02C2F1200300FA03FC20FA02F001FA98
:1004B00003FE40EA0E0021FA02F11444BDE600BF3B
:1004C00070B54FF0FF0C4CF4E06C1CEA11541DBFEA
:1004D0001CEA135594EA0C0F95EA0C0F00F0DEF8B5
:1004E0002C4481EA030621EA4C5123EA4C5350EA9A
:1004F000013518BF52EA033541F4801143F48013EB
:1005000038D0A0FB02CE4FF00005E1FB02E506F07B
:100510000042E0FB03E54FF00006E1FB03569CF0D0
:10052000000F18BF4EF0010EA4F1FF04B6F5007FD6
:1005300064F5407404D25FEA4E0E6D4146EB060648
:1005400042EAC62141EA55514FEAC52040EA5E50D1
:100550004FEACE2EB4F1FD0C88BFBCF5E06F1ED87B
:10056000BEF1004F08BF5FEA500E50F1000041EBB2
:10057000045170BD06F0004646EA010140EA02005F
:1005800081EA0301B4EB5C04C2BFD4EB0C0541EA81
:10059000045170BD41F480114FF0000E013C00F396
:1005A000AB8014F1360FDEBF002001F0004170BDBA
:1005B000C4F10004203C35DA0C341BDC04F11404D3
:1005C000C4F1200500FA05F320FA04F001FA05F25F
:1005D00040EA020001F0004221F0004110EBD3702C
:1005E00021FA04F642EB06015EEA430E08BF20EA58
:1005F000D37070BDC4F10C04C4F1200500FA04F3FB
:1006000020FA05F001FA04F240EA020001F000418C
:1006100010EBD37041F100015EEA430E08BF20EAFF
:10062000D37070BDC4F1200500FA05F24EEA020E47
:1006300020FA04F301FA05F243EA020321FA04F076
:1006400001F0004121FA04F220EA020000EBD3702D
:100650005EEA430E08BF20EAD37070BD94F0000F2D
:100660000FD101F00046400041EB010111F4801F61
:1006700008BF013CF7D041EA060195F0000F18BF12
:10068000704703F00046520043EB030313F4801F4E
:1006900008BF013DF7D043EA0603704794EA0C0F08
:1006A0000CEA135518BF95EA0C0F0CD050EA41061E
:1006B00018BF52EA4306D1D181EA030101F000419B
:1006C0004FF0000070BD50EA410606BF10461946C3
:1006D00052EA430619D094EA0C0F02D150EA0136CF
:1006E00013D195EA0C0F05D152EA03361CBF104610
:1006F00019460AD181EA030101F0004141F0FE41AF
:1007000041F470014FF0000070BD41F0FE4141F432
:10071000780170BD70B54FF0FF0C4CF4E06C1CEA32
:1007200011541DBF1CEA135594EA0C0F95EA0C0FE7
:1007300000F0A7F8A4EB050481EA030E52EA0335A2
:100740004FEA013100F088804FEA03334FF08055C3
:1007500045EA131343EA12634FEA022245EA1115F0
:1007600045EA10654FEA00260EF000419D4208BFA1
:10077000964244F1FD0404F5407402D25B084FEA4E
:100780003202B61A65EB03055B084FEA32024FF4FA
:1007900080104FF4002CB6EB020E75EB030E22BF57
:1007A000B61A754640EA0C005B084FEA3202B6EB17
:1007B000020E75EB030E22BFB61A754640EA5C00C6
:1007C0005B084FEA3202B6EB020E75EB030E22BF56
:1007D000B61A754640EA9C005B084FEA3202B6EB57
:1007E000020E75EB030E22BFB61A754640EADC0016
:1007F00055EA060E18D04FEA051545EA16754FEA78
:1008000006164FEAC30343EA52734FEAC2025FEA95
:100810001C1CC0D111F4801F0BD141EA00014FF024
:1008200000004FF0004CB6E711F4801F04BF0143F5
:100830000020B4F1FD0C88BFBCF5E06F3FF6AFAE11
:10084000B5EB030C04BFB6EB020C5FEA500C50F1A1
:10085000000041EB045170BD0EF0004E4EEA113124
:1008600014EB5C04C2BFD4EB0C0541EA045170BD2B
:1008700041F480114FF0000E013C90E645EA060E6F
:100880008DE60CEA135594EA0C0F08BF95EA0C0F9D
:100890003FF43BAF94EA0C0F0AD150EA01347FF4E5
:1008A00034AF95EA0C0F7FF425AF104619462CE7BC
:1008B00095EA0C0F06D152EA03353FF4FDAE10461F
:1008C000194622E750EA410618BF52EA43067FF470
:1008D000C5AE50EA41047FF40DAF52EA43057FF400
:1008E000EBAE12E74FF0FF3C06E000BF4FF0010C0B
:1008F00002E000BF4FF0010C4DF804CD4FEA410C6F
:100900007FEA6C5C4FEA430C18BF7FEA6C5C1BD03B
:1009100001B050EA410C0CBF52EA430C91EA030FBC
:1009200002BF90EA020F0020704710F1000F91EA19
:10093000030F58BF994208BF90422CBFD8176FEAE7
:10094000E37040F0010070474FEA410C7FEA6C5CB5
:1009500002D150EA013C07D14FEA430C7FEA6C5CBC
:10096000D6D152EA033CD3D05DF8040B704700BFE8
:100970008446104662468C461946634600E000BF36
:1009800001B5FFF7B7FF002848BF10F1000F01BD08
:100990004DF808EDFFF7F4FF0CBF012000205DF8D3
:1009A00008FB00BF4DF808EDFFF7EAFF34BF012058
:1009B00000205DF808FB00BF4DF808EDFFF7E0FFF1
:1009C00094BF012000205DF808FB00BF4DF808ED42
:1009D000FFF7CEFF94BF012000205DF808FB00BFA9
:1009E0004DF808EDFFF7C4FF34BF012000205DF88B
:1009F00008FB00BF4FEA410212F5001215D211D5D3
:100A00006FF47873B3EB625212D94FEAC12343F00B
:100A1000004343EA505311F0004F23FA02F018BF8D
:100A2000404270474FF00000704750EA013005D156
:100A300011F0004008BF6FF0004070474FF0000019
:100A4000704700BF7BB972B90029BEBF00204FF0CC
:100A5000004106E008BF00281CBF6FF000414FF0C6
:100A6000FF3000F0C7B9ADF1080C6DE904CE0029E4
:100A700009DB002B1ADB00F04DF8DDF804E0DDE9BE
:100A8000022304B07047404261EB4101002B1BDBA5
:100A900000F040F8DDF804E0DDE9022304B0404254
:100AA00061EB4101524263EB43037047524263EBF7
:100AB000430300F02FF8DDF804E0DDE9022304B081
:100AC000404261EB41017047524263EB430300F047
:100AD00021F8DDF804E0DDE9022304B0524263EBC3
:100AE0004303704753B94AB9002908BF00281CBF07
:100AF0004FF0FF314FF0FF3000F07CB9ADF1080C42
:100B00006DE904CE00F006F8DDF804E0DDE902232B
:100B100004B070472DE9F0478C46089D04468A468C
:100B2000002B4AD18A42174662D9B2FA82F64EB1F8
:100B3000C6F1200E01FA06F3B740B44020FA0EFECB
:100B40004EEA030A4FEA1748230C1FFA87F9BAFB4B
:100B5000F8FE08FB1EAA0EFB09F243EA0A439A427A
:100B60000BD9FB180EF1FF312CBF012000209A4257
:100B700002D9002800F02A818E469A1AA3B2B2FB4D
:100B8000F8F008FB102200FB09F943EA0244A145F2
:100B900007D93C1900F1FF3302D2A14500F21081C0
:100BA0001846A4EB090440EA0E4000211DB1F440B0
:100BB0000023C5E90043BDE8F0878B4208D9002D2A
:100BC00000F0F2800021C5E9000C0846BDE8F0877E
:100BD000B3FA83F100294ED16345C0F0E880824228
:100BE00040F2E5800846002DE5D0C5E9004AE2E77D
:100BF00002B9FFDEB2FA82F6002E40F099808B1A1D
:100C00004FEA124E1FFA82F801214FEA144CB3FB4F
:100C1000FEF20EFB123008FB02F94CEA004CE145F3
:100C200008D917EB0C0C02F1FF3302D2E14500F2B8
:100C3000CA801A46ACEB090CA3B2BCFBFEF00EFB5B
:100C400010CC08FB00F843EA0C44A0450ED93C192F
:100C500000F1FF332CBF4FF0010C4FF0000CA0450A
:100C600003D9BCF1000F00F0A8801846A4EB0804DB
:100C700040EA02409AE7C1F120048B4002FA01FEEB
:100C80000CFA01F6E24020FA04F72CFA04FC00FA10
:100C900001F813433E431F0C320C1FFA83F9BCFBCF
:100CA000F7F007FB10CC00FB09FA42EA0C4CE245D6
:100CB00008D913EB0C0C00F1FF3202D2E24500F22E
:100CC00089801046ACEB0A0CB6B2BCFBF7FA07FB06
:100CD0001ACC0AFB09F946EA0C42914506D99A1842
:100CE0000AF1FF3601D291457AD8B2464AEA00406D
:100CF000A2EB0902A0FB0E67BA42B446B94602D382
:100D000007D1B04505D2B6EB0E0C67EB03030138F3
:100D10009946002D6BD0B8EB0C0362EB090202FA86
:100D200004F4CB40CA4000211C43C5E9004242E71D
:100D3000B740C6F1200201FA06F3B44021FA02FCE2
:100D40004FEA174E20FA02F21FFA87F8BCFBFEF1B9
:100D50001A430EFB11CC01FB08F0130C43EA0C4CB8
:100D6000604507D917EB0C0C01F1FF3301D2604548
:100D700033D81946ACEB000C92B2BCFBFEF00EFB74
:100D800010CC00FB08F342EA0C4C634507D917EB83
:100D90000C0C00F1FF3201D2634525D81046ACEBB4
:100DA000030340EA014130E72946284603E7841A55
:100DB0006CEB030301209A4615E702383C4455E7E3
:100DC00002383C44EDE6023ABC4433E7AEF1020E91
:100DD0003B44D2E602389C4474E70239BC44C9E77C
:100DE000AAF1020A1A4481E70238BC44D7E729462F
:100DF000E1E600BF704700BF844641EA000313F0FC
:100E0000030349D1403A23D30B6803604B68436026
:100E10008B688360CB68C3600B6903614B69436176
:100E20008B698361CB69C3610B6A03624B6A43625E
:100E30008B6A8362CB6AC3620B6B03634B6B436346
:100E40008B6B8363CB6BC36340304031403ADBD262
:100E500030320BD30B6803604B6843608B68836050
:100E6000CB68C36010301031103AF3D20C3205D386
:100E700051F8043B40F8043B043AF9D2043208D05C
:100E8000D2071CBF11F8013B00F8013B01D30B88CE
:100E900003806046704700BF082A13D38B07B1D088
:100EA00010F00303AED0C3F10403D21ADB071CBF5A
:100EB00011F8013B00F8013BA4D331F8023B20F8C4
:100EC000023B9FE7043AD9D3013A11F8013B00F8FD
:100ED000013BF9D20B7803704B7843708B788370A9
:100EE0006046704780EA010C1CF0030F37D110F008
:100EF000030C20F0030021F0030150F8042B08BF7D
:100F000051F8043B0ED08CF0030C6FF07F434FEA96
:100F1000CC0C23FA0CFC51F8043B42EA0C0243EAE5
:100F20000C0300BFA2F1013C9A4201BF2CEA020C63
:100F30001CF0803F50F8042B51F8043BF2D04FEAEC
:100F400002604FEA1222012828BFB0EB036F08BFEE
:100F50001B0AF4D003F0FF03000EC01A704710F014
:100F6000030F0AD010F8012B11F8013B012A28BF0A
:100F70009A42F4D0A2EB030070474DF8045D50F89C
:100F8000042B01F0030521F0030151F8043B022D6D
:100F900026D04DD822F07F45B5EB132FA2F1013CAE
:100FA0002CEA020C0DD11CF0803C08BF51F8043B28
:100FB0000AD185EA0205B5EB036F0CD150F8042B7A
:100FC000E8E74FEA13235BE03CF07F4C54D10B7809
:100FD0004FEA126554E04FEA126503F0FF034FE059
:100FE0004FEA0245A2F1013C4FEA15452CEA020CFA
:100FF000B5EB134F18D11CF0803C08BF51F8043BEF
:1010000007D185EA0205B5EB034F09D150F8042B4F
:10101000E6E75FEA0C4C2FD10B884FEA12452FE030
:101020004FEA03434FEA12454FEA134328E000BF5B
:1010300002F0FF05B5EB136FA2F1013C2CEA020CA4
:101040000DD11CF0803C08BF51F8043B0AD185EA61
:101050000205B5EB032F0AD150F8042BE8E74FEA5D
:1010600013630DE012F0FF0F06D051F8043B4FEA76
:10107000122523F07F4303E04FF0000020BC7047AF
:1010800005F0FF0203F0FF00012828BF904204BFD3
:101090002D0A1B0AF4D0A2EB000020BC704700BF51
:1010A0004FEA410C7FEA6C5C02D150EA013C0AD164
:1010B0004FEA430C7FEA6C5C02D152EA033C02D156
:1010C0004FF0000070474FF00100704730B44FF010
:1010D000000310F8014B11F8015B013A84EA0504A2
:1010E00043EA0403F5D1A3F101034FEAD37030BC06
:1010F00070474FF0000310F8012B013943EA020357
:10110000F9D1A3F101034FEAD37070472DE9F0073D
:1011100091E8F807B2E802105B1854EB0C04B2E84F
:1011200002104D4156EB0C06B2E802104F4158EB4D
:101130000C08B2E8021059EB01095AEB0C0A89417C
:10114000B3F1FF3374F1FF3475F1FF3576F100062A
:1011500077F1000778F1000879F101097AF1FF3A97
:1011600051F100014A425B184C414D4156F10006D5
:1011700057F1000758F1000859EB02095AEB010A30
:1011800080E8F807BDE8F00770472DE9F00791E81F
:10119000F807B2E802105B1A74EB0C04B2E8021014
:1011A0008D4176EB0C06B2E802108F4178EB0C080B
:1011B000B2E8021079EB01097AEB0C0A89414A4244
:1011C0005B184C414D4156F1000657F1000758F1AC
:1011D000000859EB02095AEB010A80E8F807BDE85C
:1011E000F00770470A462DE9F04F41EC140A92ECE3
:1011F000080A91E8390010EE101AA0FB01784FF0B0
:101200000009E3FB01894FF0000AE4FB019A4FF06B
:10121000000BE5FB01AB12EE101A4FF0000CE0FBE7
:1012200001BC4FF0000EE3FB01CE4FF00002E4FBE7
:1012300001E24FF00006E5FB012605EE107A10EE04
:10124000901A4FF00007E0FB018719EB07094FF0F8
:10125000000747EB0707E3FB01971AEB070A4FF07C
:10126000000747EB0707E4FB01A71BEB070B4FF059
:10127000000747EB0707E5FB01B712EE901A1CEBDE
:10128000070C4FF0000747EB0707E0FB01C71EEB19
:10129000070E4FF0000747EB0707E3FB01E7D21902
:1012A0004FF0000747EB0707E4FB0127F6194FF063
:1012B000000747EB0707E5FB016705EE908A11EE93
:1012C000101A4FF00008E0FB01981AEB080A4FF0E3
:1012D000000848EB0808E3FB01A81BEB080B4FF0E4
:1012E000000848EB0808E4FB01B81CEB080C4FF0C1
:1012F000000848EB0808E5FB01C813EE101A1EEBC6
:10130000080E4FF0000848EB0808E0FB01E812EB7C
:1013100008024FF0000848EB0808E3FB012816EB31
:1013200008064FF0000848EB0808E4FB016817EBDB
:1013300008074FF0000848EB0808E5FB017806EEC7
:10134000109A11EE901A4FF00009E0FB01A91BEB77
:10135000090B4FF0000949EB0909E3FB01B91CEB4C
:10136000090C4FF0000949EB0909E4FB01C91EEB28
:10137000090E4FF0000949EB0909E5FB01E913EEFD
:10138000901A12EB09024FF0000949EB0909E0FB42
:10139000012916EB09064FF0000949EB0909E3FBA7
:1013A000016917EB09074FF0000949EB0909E4FB54
:1013B000017918EB09084FF0000949EB0909E5FB31
:1013C000018906EE90AA14EE901A01F1100191E83D
:1013D000390010EE101A4FF0000AE0FB01BA1CEBC6
:1013E0000A0C4FF0000A4AEB0A0AE3FB01CA1EEBA3
:1013F0000A0E4FF0000A4AEB0A0AE4FB01EA12EB7C
:101400000A024FF0000A4AEB0A0AE5FB012A12EE33
:10141000101A16EB0A064FF0000A4AEB0A0AE0FB24
:10142000016A17EB0A074FF0000A4AEB0A0AE3FBCE
:10143000017A18EB0A084FF0000A4AEB0A0AE4FBAB
:10144000018A19EB0A094FF0000A4AEB0A0AE5FB88
:10145000019A07EE10BA10EE901A4FF0000BE0FB65
:1014600001CB1EEB0B0E4FF0000B4BEB0B0BE3FB1A
:1014700001EB12EB0B024FF0000B4BEB0B0BE4FB01
:10148000012B16EB0B064FF0000B4BEB0B0BE5FBA8
:10149000016B12EE901A17EB0B074FF0000B4BEBA2
:1014A0000B0BE0FB017B18EB0B084FF0000B4BEB39
:1014B0000B0BE3FB018B19EB0B094FF0000B4BEB14
:1014C0000B0BE4FB019B1AEB0B0A4FF0000B4BEBF1
:1014D0000B0BE5FB01AB07EE90CA11EE101A4FF0B3
:1014E000000CE0FB01EC12EB0C024FF0000C4CEB9B
:1014F0000C0CE3FB012C16EB0C064FF0000C4CEB34
:101500000C0CE4FB016C17EB0C074FF0000C4CEBE0
:101510000C0CE5FB017C13EE101A18EB0C084FF0D5
:10152000000C4CEB0C0CE0FB018C19EB0C094FF0A0
:10153000000C4CEB0C0CE3FB019C1AEB0C0A4FF07B
:10154000000C4CEB0C0CE4FB01AC1BEB0C0B4FF058
:10155000000C4CEB0C0CE5FB01BC08EE10EA11EEA4
:10156000901A4FF0000EE0FB012E16EB0E064FF026
:10157000000E4EEB0E0EE3FB016E17EB0E074FF065
:10158000000E4EEB0E0EE4FB017E18EB0E084FF042
:10159000000E4EEB0E0EE5FB018E13EE901A19EBCA
:1015A0000E094FF0000E4EEB0E0EE0FB019E1AEB03
:1015B0000E0A4FF0000E4EEB0E0EE3FB01AE1BEBDE
:1015C0000E0B4FF0000E4EEB0E0EE4FB01BE1CEBBB
:1015D0000E0C4FF0000E4EEB0E0EE5FB01CE54EC60
:1015E000173A18EE101A13EB0A0354EB0B0451EBE5
:1015F0000C0152EB0E02002040F1000013EB0B0334
:1016000054EB0C0451EB0E0152EB0E02464100204C
:10161000474158EB000859EB0A0940F10000B3EBD1
:101620000E0374F1000471F1000172EB0A0276EB13
:101630000B0677EB0C0778EB0A0879EB0C0960F1E5
:101640000000B2EB0B0276EB0C0677EB0E0778EBA3
:101650000B0879EB0E0960F100005FEAE07C7FEA9D
:101660000C0CDCF1000EB3EB0C0374EB0C0471EB0F
:101670000C0172F1000276F1000677F1000778EBB9
:101680000E0879EB0C0960F100005FEAE07CDCF108
:10169000000E13EB0C0354EB0C0451EB0C0152F154
:1016A000000256F1000657F1000758EB0E0859EBFF
:1016B0000C0940F100005FEAE07CDCF1000E13EB66
:1016C0000C0354EB0C0451EB0C0152F1000256F1E7
:1016D000000657F1000758EB0E0859EB0C095BECBC
:1016E00015AA5EEC16CA1AEB060A5BEB070B5CEB5D
:1016F000080C5EEB090E002040F100001AEB070A0F
:101700005BEB080B5CEB090C5EEB090E4341002020
:1017100044414141724140F10000BAEB090A7BF1BA
:10172000000B7CF1000C7EEB060EBB4174EB080451
:10173000B14172EB080260F10000BEEB070E73EBE3
:10174000080374EB0904B94172EB090260F100006F
:101750005FEAE0787FEA0808D8F10009BAEB080AE6
:101760007BEB080B7CEB080C7EF1000E73F10003A1
:1017700074F1000471EB090172EB080260F10000E2
:101780005FEAE078D8F100091AEB080A5BEB080B76
:101790005CEB080C5EF1000E53F1000354F1000401
:1017A00051EB090152EB080240F100005FEAE078DA
:1017B000D8F100091AEB080A5BEB080B5CEB080C8C
:1017C0005EF1000E53F1000354F1000451EB0901E6
:1017D00052EB080214EE100AA0E8005C18C080E882
:1017E0000600BDE8F08F00BF70B491E87800B2E861
:1017F00002105B1854EB0C04B2E802104D4156EB9A
:101800000C0680E878008041013070BC704770B4ED
:1018100091E87800B2E802105B1A74EB0C04B2E8AD
:1018200002108D4176EB0C0680E878008041404242
:1018300070BC70472DE9F00791E8F807B2E8021094
:101840005B1854EB0C04B2E802104D4156EB0C0649
:10185000B2E802104F4158EB0C08B2E8021059EB05
:1018600001095AEB0C0A80E8F80780410130BDE815
:10187000F00770472DE9F00791E8F807B2E8021089
:101880005B1A74EB0C04B2E802108D4176EB0C0687
:10189000B2E802108F4178EB0C08B2E8021079EB45
:1018A00001097AEB0C0A80E8F80780414042BDE864
:1018B000F00770472DE9F007524290E87800B1E850
:1018C00080071740DB1918EA020854EB080419EAEC
:1018D000020955EB09051AEA020A56EB0A0678C016
:1018E00090E87800B1E8800717407B4118EA0208C9
:1018F00054EB080419EA020955EB09051AEA020A31
:1019000056EB0A0678C080410130BDE8F007704709
:101910002DE9F007524290E87800B1E880071740BF
:10192000DB1B18EA020874EB080419EA020975EBDC
:1019300009051AEA020A76EB0A0678C090E87800F0
:10194000B1E880071740BB4118EA020874EB0804AD
:1019500019EA020975EB09051AEA020A76EB0A068A
:1019600078C080414042BDE8F007704790E8300001
:1019700091E8C000A31B1340E41AF618EB1B1340B8
:10198000ED1AFF1830C0C0C17047F0B55242FFF7E2
:10199000EDFFFFF7EBFFFFF7E9FFFFF7E7FFF0BD14
:1019A0002DE9F0073AC91668A1FB069A4FF0000C22
:1019B000E3FB06AC4FF00007E4FB06C74FF000085E
:1019C000E5FB067840F8049B56684FF00009E1FB00
:1019D00006A91CEB090C4FF0000949EB0909E3FBD0
:1019E00006C917EB09074FF0000949EB0909E4FBA9
:1019F000067918EB09084FF0000949EB0909E5FBE6
:101A0000068940F804AB96684FF0000AE1FB06CA6D
:101A100017EB0A074FF0000A4AEB0A0AE3FB067AC3
:101A200018EB0A084FF0000A4AEB0A0AE4FB068AA0
:101A300019EB0A094FF0000A4AEB0A0AE5FB069A7D
:101A400040F804CBD6684FF0000CE1FB067C18EBA5
:101A50000C084FF0000C4CEB0C0CE3FB068C19EB64
:101A60000C094FF0000C4CEB0C0CE4FB069C1AEB41
:101A70000C0A4FF0000C4CEB0C0CE5FB06AC80E8BC
:101A80008017BDE8F00770470A462DE9F04F41EC9A
:101A9000140A92EC080A91E8390010EE101AA0FB23
:101AA00001784FF00009E3FB01894FF0000AE4FBE5
:101AB000019A4FF0000BE5FB01AB12EE101A4FF04C
:101AC000000CE0FB01BC4FF0000EE3FB01CE4FF039
:101AD0000002E4FB01E24FF00006E5FB012605EE03
:101AE000107A10EE901A4FF00007E0FB018719EB17
:101AF00007094FF0000747EB0707E3FB01971AEBD5
:101B0000070A4FF0000747EB0707E4FB01A71BEBB1
:101B1000070B4FF0000747EB0707E5FB01B712EE95
:101B2000901A1CEB070C4FF0000747EB0707E0FB90
:101B300001C71EEB070E4FF0000747EB0707E3FB5B
:101B400001E7D2194FF0000747EB0707E4FB012735
:101B5000F6194FF0000747EB0707E5FB016705EEB5
:101B6000908A11EE101A4FF00008E0FB01981AEB72
:101B7000080A4FF0000848EB0808E3FB01A81BEB3C
:101B8000080B4FF0000848EB0808E4FB01B81CEB19
:101B9000080C4FF0000848EB0808E5FB01C813EEFD
:101BA000101A1EEB080E4FF0000848EB0808E0FB87
:101BB00001E812EB08024FF0000848EB0808E3FBCD
:101BC000012816EB08064FF0000848EB0808E4FB74
:101BD000016817EB08074FF0000848EB0808E5FB21
:101BE000017806EE109A11EE901A4FF00009E0FB12
:101BF00001A91BEB090B4FF0000949EB0909E3FBB5
:101C000001B91CEB090C4FF0000949EB0909E4FB91
:101C100001C91EEB090E4FF0000949EB0909E5FB6C
:101C200001E913EE901A12EB09024FF0000949EB9B
:101C30000909E0FB012916EB09064FF0000949EB01
:101C40000909E3FB016917EB09074FF0000949EBAC
:101C50000909E4FB017918EB09084FF0000949EB89
:101C60000909E5FB018906EE90AA14EE901A01F12C
:101C7000100191E8390010EE101A4FF0000AE0FB55
:101C800001BA1CEB0A0C4FF0000A4AEB0A0AE3FB0C
:101C900001CA1EEB0A0E4FF0000A4AEB0A0AE4FBE7
:101CA00001EA12EB0A024FF0000A4AEB0A0AE5FBCE
:101CB000012A12EE101A16EB0A064FF0000A4AEB40
:101CC0000A0AE0FB016A17EB0A074FF0000A4AEB29
:101CD0000A0AE3FB017A18EB0A084FF0000A4AEB04
:101CE0000A0AE4FB018A19EB0A094FF0000A4AEBE1
:101CF0000A0AE5FB019A07EE10BA10EE901A4FF0AF
:101D0000000BE0FB01CB1EEB0B0E4FF0000B4BEB7F
:101D10000B0BE3FB01EB12EB0B024FF0000B4BEB59
:101D20000B0BE4FB012B16EB0B064FF0000B4BEB00
:101D30000B0BE5FB016B12EE901A17EB0B074FF044
:101D4000000B4BEB0B0BE0FB017B18EB0B084FF090
:101D5000000B4BEB0B0BE3FB018B19EB0B094FF06B
:101D6000000B4BEB0B0BE4FB019B1AEB0B0A4FF048
:101D7000000B4BEB0B0BE5FB01AB07EE90CA11EE32
:101D8000101A4FF0000CE0FB01EC12EB0C024FF0CC
:101D9000000C4CEB0C0CE3FB012C16EB0C064FF08B
:101DA000000C4CEB0C0CE4FB016C17EB0C074FF038
:101DB000000C4CEB0C0CE5FB017C13EE101A18EB3D
:101DC0000C084FF0000C4CEB0C0CE0FB018C19EBF9
:101DD0000C094FF0000C4CEB0C0CE3FB019C1AEBD4
:101DE0000C0A4FF0000C4CEB0C0CE4FB01AC1BEBB1
:101DF0000C0B4FF0000C4CEB0C0CE5FB01BC08EE9F
:101E000010EA11EE901A4FF0000EE0FB012E16EBD7
:101E10000E064FF0000E4EEB0E0EE3FB016E17EBBD
:101E20000E074FF0000E4EEB0E0EE4FB017E18EB9A
:101E30000E084FF0000E4EEB0E0EE5FB018E13EE7A
:101E4000901A19EB0E094FF0000E4EEB0E0EE0FB50
:101E5000019E1AEB0E0A4FF0000E4EEB0E0EE3FB46
:101E600001AE1BEB0E0B4FF0000E4EEB0E0EE4FB23
:101E700001BE1CEB0E0C4FF0000E4EEB0E0EE5FB00
:101E800001CE14EE100AA0EC075A80E8C45FBDE84A
:101E9000F08F00BF70470000114B70B51C88114BCC
:101EA00006461A7882F001021A7044F3072364B2DE
:101EB00092B11C430C4DE4B22B78A34203D02046D0
:101EC00004F0D0F82C7056B1BDE870404FF4FA72AF
:101ED000064907480AF080B824EA0304EAE770BD1F
:101EE0002A0002209D00022028000220A0000220DB
:101EF0004061022038B50B4C0B48258801F038F9B9
:101F0000052300202380FFF7C7FF00F0E9FC01460E
:101F100020B1064801F02CF9258038BD044801F0B5
:101F200027F9F9E72A00022060FF050087FF050076
:101F3000ADFF050010B5A8B908F066FE07F04AF835
:101F4000044668B1CA230A4A0A490B4801F010F94D
:101F500021460A4801F00CF9CA21054801F015F99B
:101F600012F024F9BDE81040012001F06BB900BF68
:101F7000000206000E0206001702060034020600E8
:101F800001460020FFF7D6BF0D4A10B51278AAB956
:101F90000C4AD2E8AF2F8AB1037863B905F018FC78
:101FA000044658B10146084801F0E2F82046BDE871
:101FB0001040FFF7E5BF05F02DFCF1E710BD00BFB5
:101FC00032010220340102205E04060000000000FD
:101FD0002DE9F04F8BB06E462F4B02AFD3E8AF3FE9
:101FE000A3B100252D4CDFF8C0B02D4B53F82530A0
:101FF0009946986899F8011043689B6898474B4642
:10200000024640B15968274801F0B2F8B546243776
:10201000BD46BDE8F08FD9F8080007F1080A43680B
:102020000AEBC5084246DB6899F80110984702465A
:1020300008B14B46E6E7D8F80400FEF7D7F914A339
:10204000D3E90023FEF766FB80465AF8350089463F
:10205000FEF7CCF90B46024649464046FEF77AF8B1
:102060005A46CDE90001062138460CF0CFFCE36862
:10207000C0B2013308BF0123606001352046A7606C
:10208000E360FFF781FF032D04F11004ADD1BDE73C
:102090000000000080842E41340102202C00022028
:1020A000F4010600C5010600EE01060073B5044602
:1020B00001A9684603F082FF009911F008051DD1BF
:1020C0000F4BD3E8AF3FCBB1636820465B689847BE
:1020D0000C4E636832469B682946204698470A4B57
:1020E00096F8512008485A60DA689E60013208BFAD
:1020F0000122DA60FFF748FFFFF76AFF02B070BD08
:1021000034010220E00002208C00022070B5064657
:10211000154BD3E8AF3F6BB1144C204600F080FB69
:1021200040B9134D227E2978914203D0012A09D06B
:10213000022A12D0B6B1BDE8704000220D490E4807
:1021400009F04ABF0D4A0E4B9A6006220C485A60AD
:10215000FFF71AFF237E2B70ECE70A4A084B9A60C0
:102160000B22F3E770BD00BF3401022038010220CA
:102170009C0002206C0002204061022052020600F6
:102180005C00022059020600354BF7B50746187867
:102190000D46002841D0334C334E236831688B42C2
:1021A00013DA324A05EA07001188B1F5406F04BF1F
:1021B00040F604011180C10714D503215A1C226086
:1021C0002B4A2C48D15400F0D3FF226833689A423E
:1021D00006D14FF40062254B27481A8009F0F8FB1E
:1021E00003B0F0BD820706D504215A1C2260204AA4
:1021F0002248D154E7E76F0706D501215A1C226017
:102200001B4A1F48D154DEE72807E9D502215A1C92
:102210002260174A1B48D154D5E7690701D5FFF75B
:1022200075FFEA07DCD53123ADF80430164BD3E84F
:10223000AF3F002BD4D0FB0758BF3023134C01A86D
:1022400058BF8DF80430A0600CF01EFDE36860609C
:10225000013308BF01230D48E360FFF795FEBFE798
:102260003201022014000220180002202A0002205D
:1022700058010220D4FF050064010220DEFF0500A2
:10228000E8FF0500F2FF05003401022004000220EF
:10229000002310B588B08DF8043001230F4A8DF863
:1022A000083001AB92E80300039302AA04ABCDE926
:1022B00006234FF4806283E80300094B06A81A80C6
:1022C00005F036FA044630B10146064800F050FFEA
:1022D0002046FFF755FE08B010BD00BF48FF0500BF
:1022E0002A000220FCFF0500012000F0ABBF012006
:1022F00000F0A8BFF7B500240A4E0B4FA35D01A85C
:102300008DF8043005F04AFA054630B101463846EA
:1023100000F02EFF2846FFF733FE0134062CEDD1E6
:1023200003B0F0BDCEFF05007B0406002DE9F341AC
:10233000584A13780133DBB2062B137057D10124AE
:10234000554BD3E8EF2FC3E8E14F0029F9D15348AB
:1023500007F0C6FC0023ADF804308DF804400446B5
:10236000002847D14D494E4800F002FF4D4807F084
:10237000B7FC0446002876D14A49494800F0F8FEE7
:102380000024494F494EDFF8608157F824506868AF
:1023900007F0A6FCA86078B940F2A7333246414660
:1023A000434800F0E5FE6968424800F0E1FE40F273
:1023B000A731304600F0E9FE3F4B29782201D15485
:1023C0001A4401231C44032CD360DED102213B4A72
:1023D00011700021D3603A4A11703A49D36091607C
:1023E00091F851105160384A1370FFF7F1FD02B0B7
:1023F000BDE8F081354800F0BBFE636801A91B68A9
:10240000334A20469847014608B13248ACE7636832
:1024100020465B68984770B12F494FF45C73234A9C
:10242000234800F0A5FE2D4800F0A2FE4FF45C7199
:102430001E4800F0AAFE6368224A9B6800212046DD
:102440009847002892D040F27333184A224918481E
:1024500000F08EFE224800F08BFE40F273311348EC
:1024600000F093FE82E70023ADF8043001238DF8DD
:10247000043043685B6833B101A91A4A98470146A2
:1024800020B114487AE76FF08501FAE7204600F0A2
:1024900039FA75E7000002203401022082030600A9
:1024A0008A03060024040600F40106000002060068
:1024B00017020600430406002C000220040002203C
:1024C0008C000220E00002205C000220A303060032
:1024D000AD200400B50306000E020600DC03060072
:1024E000FF030600951E04002F040600017870B556
:1024F0000529044653D017D8022932D006D801291D
:102500002AD0BDE870404B4800F032BE032944D0C9
:102510000429F6D1484800F02BFEBDE8704008229F
:10252000464B1A80FFF7E6BE07293FD05ED3082945
:102530003ED0FF29E5D14168414800F019FE002254
:10254000404BD3E8EF1FC3E8E02F0028F9D16068C3
:10255000BDE87040FFF714BD3B48BDE8704000F097
:1025600007BE3A4E3A4800F003FE3578002D4FD1B1
:1025700001222946374809F0F5F94FF440622F4B04
:1025800035481A8001233370344BE2681D60344BA8
:102590001A6000F0EDFD3348DFE73348DDE73348EC
:1025A00000F0E6FDBDE87040FFF7C0BE3048D4E75C
:1025B000304800F0DDFD0023224AD2E8EF1FC2E8D8
:1025C000E03F0028F9D11D4A2B491380D1E8EF3FA5
:1025D00043F00102C1E8E02F0028F7D1DB0717D450
:1025E000BDE870400839254808F0EFB8244800F0ED
:1025F000BFFD2448E5680CF047FB22490246284607
:102600000CF0E6F828B90D4A138843F00103138053
:1026100070BD1D48E4680CF037FB1B49024620469C
:102620000CF0D6F820B9054A138823F00103EEE731
:10263000164892E7B0010600CF0006002A000220EB
:1026400048010600340102201A000600320102206F
:102650003D0006006401022065000600140002200F
:102660001800022090000600B0000600E4000600FA
:10267000030106002201060024000220406102201E
:1026800069010600800106008D0106009B0106001D
:102690008FB5474800F06CFD464803F09FFC0146AB
:1026A00010B1454800F064FD03F064FC014610B130
:1026B000424800F05DFD0F21002003F0C9FC0146F7
:1026C00010B13F4800F054FD00223E4B3E493F48C8
:1026D000C3E901123E491A6009F076FC3D493E48C3
:1026E00009F072FC3D493E4809F06EFC4FF4FA7265
:1026F00036493C4809F070FC3B4B04AC44F80C3DB7
:10270000204604F0F5FF70B1384940F25923384AA9
:10271000384800F02DFD384800F02AFD40F25921DC
:10272000334800F032FD354800F022FD4FF480625E
:10273000334B1A8006F0F8FB70B12C4940F24F334E
:102740002B4A2C4800F014FD2E4800F011FD40F2F9
:102750004F31274800F019FD2B4E0020FFF798FD60
:102760003746DFF8B48005F07DF83378CBB100212F
:10277000404609F071F9A0B9244B8DF804001B689C
:1027800020460293224B039304F0DEFF054630B14E
:102790000146204800F0ECFC2846FFF7F1FB00233F
:1027A0003B700A2009F02AF801F058FADBE700BF75
:1027B00065020600892104007A020600A6020600CE
:1027C000CF0206001C00022091220400A00002207B
:1027D000991E04000D2104006C000220F51E040067
:1027E000C000022040610220ED2404000E02060019
:1027F0000002060017020600F70206002503060085
:102800002A000220380306003201022018000220AC
:10281000580102205D030600640102200000000050
:10282000F0B5294E0546306887B0436803219B68A0
:102830009847044628B1254800F09AFC204607B086
:10284000F0BD30686A4643680321DB689847044658
:1028500008B11F48F0E70598FDF7C8FD18A3D3E9B4
:102860000023FDF757FF064604980F46FDF7BEFD0F
:1028700002460B4630463946FDF76CFC0022002329
:10288000FDF768FC134BD3E90423FDF761FC064612
:102890000F460022C5E904670F4BFEF797F858B9B9
:1028A0000E4B002230463946FEF786F8002814BF4A
:1028B000022303232B76C1E70123FBE7AFF300805C
:1028C0000000000080842E41980102209F04060031
:1028D000BB0406008001022000001440000014C068
:1028E00008B50022002310461946FDF713FF044BDC
:1028F000C3E90001C3E90201C3E90401002008BDE6
:1029000080010220014B1860704700BF980102202F
:1029100040E800F313F4803FD8B208BF6FF0150011
:10292000704770B50C254D43C66890F90B007419BB
:102930008842A8BF21464FF0200492FBF4F4B8BFB0
:10294000715902F01F0001EB8401196070BD07B5D9
:1029500001ABFFF7E6FF0123019A03FA00F01368C9
:102960000343136003B05DF804FB07B501ABFFF749
:10297000D8FF0123019A03FA00F0136823EA000349
:10298000136003B05DF804FB10F0010005D04FF0B8
:102990002003EFF3118083F3118870472DE9F8438A
:1029A0000446FF2200214FF00C0E436805890068A1
:1029B0005D4394F80AC02844E2728C4505DC00258A
:1029C0002389AB4222DCBDE8F883B5FBF3F20EFBB2
:1029D00001F7D4F80C801F2A08EB0706C8BF1F3286
:1029E0004FEA930306F10409C8BF520903F1030338
:1029F000C6E9019923F00303D4BFE17248F8070048
:102A000001F10101C8BF00EB8200D6E76268E3680C
:102A10006A4320681E1D811886509A6820464A60C5
:102A20009A68116099602A460021FFF790FF0135EE
:102A3000C6E72DE9F04F8BB0867A00AFC7E90232C6
:102A4000B3000A3303F4FF63ADEB030DE9464A46D6
:102A500043680446033323F0030342F804394FF07C
:102A6000FF3500234FF00C0C581E9E42786209DDA2
:102A70002BB110688008033020F0030050605068CC
:102A800088420BD27B6A013314D100236FF00B0014
:102A90003A6D13602C37BD46BDE8F08FE068043214
:102AA0000CFB030000F1040E4068704518BF1D4682
:102AB0000133D9E76E1CE8D0207CFFF765FF0C23BB
:102AC0006B431A1DE368386213441E68B3427AD020
:102AD000D6E900131960316859F825204B600023AE
:102AE000C6E9003323682946F31A93FBF2F2204625
:102AF000FFF73BFFA9EB890305F1010B3B6109EBF4
:102B000085057A6A0BF1FF339A4216DC237CD907DC
:102B100002D53B6A83F31188FB6800201A467B6A62
:102B200013607A6A236859F82220F31A93FBF2F3B0
:102B3000BA6813603B6D1E60ACE7236855F8042B40
:102B4000F31A93FBF2F34FF0010A9B003A69BB6161
:102B500005EB450313447B61D5F8008059460AFB19
:102B600008F3FB61F3187B60BB6920460AEB0302A4
:102B7000FFF7EDFE7B68226808F1FF389844A8EB68
:102B80000208218962684A4390450AD2E26879695D
:102B9000F8690A44111D31509168596091680B60C1
:102BA00093600AF1010ABAF1040FD5D1237CD8074A
:102BB00002D53B6A83F31188207CFFF7E5FE0BF119
:102BC000010B38629DE7013D6A1CA6F10C037FF4FE
:102BD0007CAF00269AE700002DE9F04F87B0837A9A
:102BE00000AF9B000A3303F4FF63ADEB030D044613
:102BF00043686846033323F003030360054601205E
:102C0000C7F80CD081421FD2207C0D461646FFF734
:102C1000BBFE8046002D20DAC523504A504951485A
:102C200000F0A6FA504800F0A3FAC5214B4800F086
:102C3000ACFA4FF0FF38237CDB0701D588F311880D
:102C40001C37BD46BDE8F08F2B6801309B0803336D
:102C500023F0030345F8043FD4E7FB68218953F8C8
:102C60002530D4F800B003FB06FABB60013B03EB50
:102C70000A027B6063680BEB0A094B439A420CD350
:102C80003A49A923354A374800F072FA384800F02B
:102C90006FFAA921314800F078FA324629462046D9
:102CA000FFF755FE0C23E26803FB05231A1D4BF8C2
:102CB0000A209A68C9F804209A68C2F80090C3F8FC
:102CC0000890237CDA0701D588F31188207CFFF770
:102CD0005BFE8046002DAED007F114033246294634
:102CE0002046FFF71EFE042390FBF3F37A699B0056
:102CF0001068D84000F00F000F289CD14FF0000959
:102D0000CB4626F003033B603B68208903EB0902B6
:102D1000BB68616803FB02FA41437B680AEB03006E
:102D2000814211D929462046FFF71FFE226802EB97
:102D30000A0152F80A004B68186052F80A00436012
:102D400042F80AB0C1F804B009F10109B9F1040F61
:102D5000DAD1013D96FBF9F65CE700BFD604060028
:102D6000B41D06001702060034050600170506000C
:102D70003105060008B50446084611461A46A04724
:102D800008F0EAFD00F0E4FF10B504464FF0FF3113
:102D9000204607F01FFD03460028F7D0426808339D
:102DA000D3E8EF1F21F0010CC3E8EECFBEF1000F16
:102DB000F6D1CB0700D5904708F07AFCE6E7002073
:102DC000704770B50D4604464520A047294652205D
:102DD000A04729462346BDE870405220184700000E
:102DE0000B6801330B60014B1B68184704BF0220BE
:102DF0002DE9F04F85B00E9C9B46012CB8BF0124F5
:102E0000012B0CBF3023202315468046894601261E
:102E10000A270022DFF870A0019402930AF101044E
:102E20000AB9AA451ED2B5FBF4F049463030C04776
:102E300001220136B5FBF4F10A23013F012F04FB07
:102E40001155BAFBF3FAE9D1494605F13000C04704
:102E5000BBF1030F03D1019B9C1B002C0FDC05B0C1
:102E6000BDE8F08F019BBB42E4DBBBF1020FE1D870
:102E70004946029803920136C047039ADAE7494669
:102E80002020C047013CE8E7FFC99A3B014B18608E
:102E9000704700BF04BF02202DE9F04F4FF0000A39
:102EA00006460F464FF0FF39D04689B01C46531EE8
:102EB0000393002505E06DB9252800F03D813946D2
:102EC000B047039B13F8010F03930028F3D109B017
:102ED000BDE8F08F642862D019D839280AD8312883
:102EE00051D22D283DD030283ED0252808D1394652
:102EF000B047DEE7582800F0A880632800F016816C
:102F000039462520B047039B39461878F0E77028EA
:102F100000F0918006D8692841D06C283CD0682800
:102F2000CFD0EDE775286DD017D87328E8D1256884
:102F300004F1040B2B461C4614F8010B002840F04A
:102F4000EC80B8F1030F40F000815C1BA9EB040496
:102F5000002C00F3E6805C46ABE7782875D07A2831
:102F6000DEE74FF00308ACE7B9F1000F0EDAB8F175
:102F7000000F00F0E780A0F13009B8F1000F08BFA2
:102F80004FF002089DE7B9F1000FF4DB0A2303FBC1
:102F90000909A9F13009F0E70AF1010A91E7BAF14C
:102FA000000F12D125680434002D05DA39462D2092
:102FB000B0476D4209F1FF3943462A46CDF80090EB
:102FC00039463046FFF714FF73E7BAF1010FE9D035
:102FD0004FF0000C4FF0FF3B073424F0070303F1E0
:102FE0000804D3E9002312F1004043F100018C45AD
:102FF00008BF834504D239463046FFF7E2FE58E762
:103000001546D1E7BAF1000F05D122680434CDF896
:1030100000904346D4E7BAF1010FF6D0073424F00C
:10302000070303F10804D3E90023002B08BFB2F122
:10303000004FECD3DFE739463020B04739467820DF
:10304000B0474FF008094FF00108BAF1010F27DC33
:10305000236804340793002304931022002393462B
:1030600002930693079B0BF1FF3B4FEA8B00C0F1E5
:10307000200CA0F1200123FA00F0049B03FA0CFCC1
:1030800040EA0C0023FA01F1084310F00F0013D1BD
:10309000069B13B9BBF1000F2ED14FF0300C11E09D
:1030A000073424F007031A6803F108045B680792E9
:1030B0000493D2E7059AD5E709288CBF4FF0570C47
:1030C0004FF0300C394660440592B047029B06959C
:1030D00001330293BBF1000FECD1B8F1030F7FF481
:1030E000E8AE029BC3EB4905002D7FF7E2AE3946FF
:1030F0002020B047013DF7E7531E91450593E9DBDA
:10310000B8F1010F03D139463020B047E2E7B8F1FA
:10311000020FDFD139462020F7E73946B047234672
:1031200009E739462020B047013C11E72068251DFA
:103130003946B0472C46BCE6AA46A8464FF0FF39B0
:103140000125BEE64FF00108BBE65C460546B8E641
:10315000002313B502AC44F8043D02460B46034875
:103160002146FFF799FE02B010BD00BFE12D04001B
:103170000FB407B504A951F8040B0191FFF7E8FF5C
:1031800003B05DF804EB04B07047404080F3118851
:103190004FF0050002DF704710B54FF02003EFF34A
:1031A000118483F3118800F011F80122054BC3F854
:1031B00040254FF0FF32044B9A62DA6284F31188A3
:1031C000002010BD0090034000ED00E0074AD2F857
:1031D000883043F47003C2F88830BFF34F8FBFF3D9
:1031E0006F8F034B034A1A60704700BF00ED00E089
:1031F00008BF02200090D00338B5054648B90C49F5
:103200000C4811230C4AFFF7B3FF11210A48FFF7BE
:10321000BCFF0A4C22684AB1094906481223064AF3
:10322000FFF7A6FF12210448FFF7AFFF256038BD66
:10323000A3100600170206007B0506009C01022071
:10324000D305060008B504464FF02002EFF31183C2
:1032500082F3118800F081F9204600F015FE034842
:10326000FFF786FF00F0FAFCFCE700BFED05060063
:1032700043685B6818470020704700000A4B70B530
:10328000C6B204461B683046984701280AD00A2C6B
:10329000064D03D10D212868FFF7EAFF3146286863
:1032A000FFF7E6FF204670BD0CBF0220A001022000
:1032B00010B5044C204601F039F82046BDE8104016
:1032C000FFF7E4BD7D32040008B5044806F008FDB0
:1032D000034B1860FFF7ECFF002008BD1606060040
:1032E000A001022010B54FF02003EFF3118283F309
:1032F0001188114C237823B982F311886FF077007D
:1033000010BD013BDBB2237023B182F311886FF053
:103310000F00F5E7094B0121187828B1217082F3DD
:1033200011886FF00A00EBE7197082F31188044AE4
:1033300011601870E4E700BFA6010220A501022079
:103340000450004010B54FF02002EFF3118382F3D8
:103350001188114C207880B183F311880F4AD2F87C
:103360001C34D2F8182403F0030343F4803393434E
:1033700014BF6FF07600002010BD0122227083F38D
:103380001188064BC3F80401C3F818150221C3F8CD
:1033900004139A60E2E700BFA4010220005000403D
:1033A00038B5204BD3F80851D3F80423D3F80001E3
:1033B00002F00102D3F80443D3F804111DBB78B91D
:1033C00042BBB1B940F2451317491848184AFFF7F4
:1033D000CFFEBDE8384040F245111548FFF7D5BE95
:1033E0000020C3F800011AB101220E4BC3F80823D4
:1033F00041B100220B4BC3F80421A20702D50222DF
:10340000C3F8082338BD0025C3F808510028E7D1C8
:10341000002AEDD0D3F80C3403F00113B3F1011FEF
:10342000E6D1E1E7005000409B06060017020600C7
:103430004306060008B500220121052000F072FBBA
:10344000052000F04BFB002008BD00002DE9F041F5
:103450004FF02003EFF3118283F311882D4B18787E
:103460001F46441C1C70C8B182F311883B784BB9CD
:1034700029492A4860232A4AFFF77AFE6021284812
:10348000FFF783FE274BD3F80C3403F00113B3F19D
:10349000011F0CBF00206FF076000AE0224D95F866
:1034A0000080B8F1000F06D0187082F311886FF019
:1034B0000A00BDE8F08101262E7082F31188194CB4
:1034C00021B3052000F01AFBC4F80081D4F80433BE
:1034D000C4F804632660D4F800219AB10022DB0707
:1034E00058BF0123C4F800214FF0200258BFC4F890
:1034F00008330E4B0520C3F8802100F0EFFA0023BB
:103500002B70B3E720BF40BF20BFE4E7C4F8001131
:103510002660F4E7A601022038060600170206001E
:103520004306060000500040A501022000E100E033
:1035300010B5064C0649224606481723FFF718FE29
:103540002046BDE810401721FFF71FBED806060031
:10355000B41D0600170206007047704700220F4B8B
:1035600010B4C3F840214FF02002EFF3118482F32E
:103570001188D3F8040540F24713094A1168401A2C
:1035800020F07F40B0FBF3F003FB0013136084F3E3
:1035900011885DF8044B08F053BF00BF0050014094
:1035A000A801022038B51A4806F09AFB60B34368B8
:1035B00001211B689847002440F24713154D4FF432
:1035C0000012C5F80845C5F840354FF48033C5F8FA
:1035D0004433C5F80433104B01211C600F4B1520F8
:1035E000C3F88021224600F09DFA152000F076FAFB
:1035F000012320460A4A13602B60D5F8043503F2F4
:103600004713C5F8403538BD4FF0FF30FBE700BF2A
:10361000BA060600005001404051014000E100E0C0
:10362000085001404CF66A03B0F1FF3F08BF18464E
:1036300001389842A8BF184640F2471220EAE070CD
:1036400000FB0220164B30B5984228BF18464FF0B9
:103650002003EFF3118483F31188124B1249D3F83E
:10366000043509685B1A23F07F43B3F5A27F10D3BA
:10367000B3F5A37F07D9B3FBF2F56A439B1AB3F501
:10368000A27F104401D300F24710054B984228BF97
:103690001846044B0844C3F8400584F3118830BD34
:1036A00066FFFF0000500140A80102204FF02002F9
:1036B000EFF3118382F31188074AD2F80405074A11
:1036C0001268801A40F2471220F07F40B0FBF2F0FF
:1036D00083F31188704700BF00500140A801022009
:1036E0004FF02003EFF3118283F311880549064B55
:1036F0000868D3F8043582F311881B1A23F07F433E
:1037000018447047A8010220005001400448816815
:10371000406A884203D003494FF080520A607047E4
:10372000FC60022004ED00E0002320210348C218C1
:103730000133412B82F80013F9D1704700E100E01A
:10374000084A0949936809685866996607494B68A9
:1037500043F080534B60002383F311889368986E85
:10376000704700BFFC600220A01A060000ED00E0D8
:10377000202080F3118811498A684FF028001044F6
:10378000EFF3098C80E8F01F0D4F4FF000664A6A96
:103790008A603E60506E0023536680F3118804B542
:1037A0000648806800F0B2FBBDE8044002F1280042
:1037B00090E8F01F8CF3098870470000FC6002203D
:1037C00004ED00E01EF0040F0CBFEFF30880EFF3F0
:1037D0000980816931F8021C11F0FF010229FFD034
:1037E00001B500F085FA01BD38B51E4C05461E48EE
:1037F000FFF7BEFCA36AD90402D51C48FFF7B8FC4A
:10380000A36A1A0502D51A48FFF7B2FCA36A9B0502
:103810000ED51848FFF7ACFCA16BA36A180407D5B6
:103820001548FFF7A5FC1DB1A36A23F40043A3626A
:103830000C4CA36A590502D51048FFF799FCA36AFE
:10384000DA0509D50E48FFF793FC064A0020936A73
:1038500043F47F43936238BDA36A9B04F5D50948BE
:10386000F1E700BF00ED00E0270706003E07060075
:1038700050070600640706007E070600940706004E
:10388000B0070600C907060010B51C4C1C48FFF71E
:103890006FFCA36A9A0102D51A48FFF769FCA36A74
:1038A000DB0102D51848FFF763FCA36ADC0202D5EE
:1038B0001648FFF75DFC114CA36A180302D51448A3
:1038C000FFF756FCA36A590302D51248FFF750FCD4
:1038D000A36A9A0302D51048FFF74AFC074CA36A73
:1038E000DB0302D50D48FFF743FCA36A00206FEA13
:1038F00003436FEA1343A36210BD00BF00ED00E075
:103900000B0A0600240A0600380A0600530A0600BD
:103910007E0A06009D0A0600C30A0600DE0A0600AB
:1039200038B5244C05462448FFF722FCA36AD90683
:1039300002D52248FFF71CFCA36A1A0702D52048CB
:10394000FFF716FCA36A9B070ED51E48FFF710FC75
:10395000616BA36A180607D51B48FFF709FC1DB168
:10396000A36A23F08003A362124CA36AD90702D58D
:103970001648FFF7FDFBA36A9A0602D51448FFF725
:10398000F7FBA36ADB060ED512494FF49E73124A69
:103990001248FFF7EDFB1248FFF7EAFB4FF49E7168
:1039A0000D48FFF7F2FB034A0020936A43F0FF0340
:1039B000936238BD00ED00E0F0080600070906003C
:1039C000500706003B090600540906006B09060073
:1039D000C9070600B41D06008B0906001702060081
:1039E000D109060038B52D4B05465C6801F07F43D0
:1039F000B3F17F4F05D000202946BDE8384000F0E4
:103A000045B9C807F7D4490602D52548FFF7B0FBEA
:103A1000C4F30804E21E092A35D8DFE802F0052EB7
:103A2000302B3434343434321E48FFF7A1FB1B4BA7
:103A3000DA6A920703D51C48FFF79AFBDBE7DB6ADB
:103A40005B00D8D51948FFF793FB194B1B782BB1B6
:103A50000120FFF765FF0628CED138BD154B1B7836
:103A60001BB10120FFF7C0FEF5E7134B1B889BB28B
:103A7000002BC0D0FFF708FFEDE70020E9E70020AA
:103A8000F0E70E48D8E70E480E49A4F110020F2CBB
:103A9000D8BF01460C48FFF76BFBACE700ED00E038
:103AA000270806004B080600630806008508060084
:103AB00028ED00E029ED00E02AED00E0A508060071
:103AC000F90706000E080600DC080600024A5369E2
:103AD00043F010035361704700ED00E043B2002B48
:103AE00008DB012200F01F0002FA00F0024A5B0925
:103AF00042F82300704700BF00E100E043B2002B12
:103B00000DDB012200F01F0002FA00F05B09044AFD
:103B1000203342F82300BFF34F8FBFF36F8F7047FE
:103B200000E100E070B54C1C072C05460E460ED98E
:103B30007223104A10491148FFF71AFB314610480A
:103B40000722FFF715FB72210A48FFF71EFB6BB235
:103B5000002BA8BF03F160434FEA4414B8BF094BE0
:103B6000E4B2ABBF03F5614305F00F0583F80043F2
:103B70005C5570BD0A0B0600550B060017020600C7
:103B80006C0B060014ED00E000F06EB808B572B6DC
:103B9000044B186A18B100221A6206F0CDF862B61A
:103BA00008BD00BFFC600220704700002DE9F04115
:103BB000099F05460F2F0C461646984625D11E4BE9
:103BC000984526D10A9B04223946284608F039F840
:103BD0000023A6F16801194A214421F0070122F0CF
:103BE0000102C5E91333C5E916468A61069AC1F890
:103BF00000804A60079A8A60089ACA604FF0807213
:103C0000CA61A9646B66BDE8F08107F110031E2B41
:103C1000D8D93C230A4A0B490B48FFF7A9FA394681
:103C20006FF00F030E220948FFF7A2FA3C21044867
:103C3000FFF7ABFAC6E700BF3D9D0400752D0400F9
:103C4000A00B0600E70B060017020600830C060017
:103C5000014910220A60704710ED00E0404080F3F7
:103C6000118830BF704700BF404080F311884FF08B
:103C700004007146014202D0EFF3098001D1EFF355
:103C80000880714601B5FFF7ADFE01BD38B50446A9
:103C90000D4605281AD8DFE800F003191913151787
:103CA0000D48FFF765FA07F057FEAA6901460B4871
:103CB000FFF75EFA29462046BDE8384000F01CB800
:103CC0000748EEE70748ECE70748EAE701460748F8
:103CD000FFF74EFAE7E700BFB40C0600520D0600EE
:103CE000D40C0600FA0C0600140D06002F0D060079
:103CF00001460068FFF7CABF052810B50CD007F0D1
:103D00004DFF60B107F04AFF0C490D4B002808BF7A
:103D100019460C48FFF72CFAFFF7A0FFFCE707F065
:103D20004DFF0028EED1084C0848A168FFF720FAA3
:103D3000A068BDE8104000F00BB800BF8E0D060073
:103D4000920D0600A30D0600FC600220C30D0600C4
:103D500038B504464FF02003EFF3118583F3118843
:103D6000037BDB070CD512492523124A1248FFF7C3
:103D7000FFF91248FFF7FCF925210E48FFF705FA75
:103D8000204607F03FFF0E4B9B68A3420BD10D4B23
:103D90005A68C2F3080212B92846FFF7D1FC5A68E4
:103DA00042F080525A602846BDE8384006F016BFFF
:103DB000350E0600E80D060017020600630E060029
:103DC000FC60022000ED00E001B572B60B4A106AFB
:103DD00000281EBF0021116205F0AEFF62B6EFF3AE
:103DE0000580A0F110004FEAC0000549014409C94F
:103DF0009847BDE80140034800470000FC600220EE
:103E00007CFC05000D37040000F006F800F008F80F
:103E100030BFFFF7FDBF00BF202383F31188704739
:103E200008B5164B83F30988EFF3148343F00203BC
:103E300083F31488BFF36F8F114A124B22F07F0275
:103E40009A60BFF34F8FBFF36F8FD3F8882042F48F
:103E50007002C3F888204FF00042C3F83422BFF349
:103E60006F8FB0EE400ABFF36F8F05F07FFF05F054
:103E700087FFFFF759FC05F0B5FF00BFE0BA02204D
:103E80000000040000ED00E0BFF34F8F0549064B32
:103E9000CA6802F4E0621343CB60BFF34F8F00BFE8
:103EA000FDE700BF00ED00E00400FA0508B5FFF7EC
:103EB000AFFFBDE80840FFF729BC000010B50D4B6F
:103EC00086B000930C4B0D4C01930D4B0D4A0293A1
:103ED00068462346012100F063F9002305930A4B4D
:103EE0000121E41A03A80393049400F07DF906B0BD
:103EF00010BD00BF000002200000000000000420F0
:103F000006000100000002200000022007B5002189
:103F100001A800F0C9F903B05DF804FB10B50B6807
:103F20000C7A23F01F0304F01F021A43CB686409C4
:103F300023F01F03044943F0010343EA440388606C
:103F4000CA600B6110BD00BF90ED00E030B585B0D8
:103F50009DF808200D890B684C68498965F30402B7
:103F600061F3471200938DF8082023F01F03621EAF
:103F7000134423F01F030393084B04461B68C3F349
:103F80000723013B984205DC6946FFF7C7FF20463F
:103F900005B030BD6FF01504F9E700BF90ED00E00B
:103FA0002DE9F04F0E46144680460025504F85B04F
:103FB000B54209DAD8F80490B9F1000F39D0B9F157
:103FC0001F0F05D86FF01504204605B0BDE8F08F2F
:103FD00019F01F0FF6D1D8F800A01AF01F0FF1D179
:103FE0005046FEF795FC834609EB0A000138FEF7C0
:103FF0008FFC8345E6D11BF1160FE3D0631E5B45B2
:10400000E0DBC7F808B0F968C7F808B03B6921F0F1
:104010001F0143F01F0AD8E900321A44994202F105
:10402000FF391CD1CA4508D141465FFA8BF0FFF732
:104030008DFF013508F10C08BAE74146C7F808B012
:10404000FB6822F01F0203F01F031A43FA60E0B27C
:10405000FFF77CFF10F1160FB4D0441CE9E7013BD9
:10406000CA45E0B223F01F03C7F808B006D13A6989
:10407000414602F01F0213433B61E9E7396901F051
:104080001F010B433B614146FFF760FF10F1160F24
:1040900098D0C7F808B0FA689DF80830441C62F35D
:1040A00004038DF808303B699DF808205B0863F332
:1040B00047128DF80820D8E900210A4400920AF13D
:1040C000FF3322F01F021344A3EB090323F01F0365
:1040D00003933B68E4B2C3F30723013BA342FFF61B
:1040E00071AF20466946FFF719FF0134A1E700BF11
:1040F00090ED00E00522034B5A60BFF34F8FBFF3F2
:104100006F8F704790ED00E0BFF35F8F0022014B8F
:104110005A60704790ED00E070B5194C194E226856
:104120003568C2F30722954215D940F20313164AA7
:1041300016491748FFF71CF822682946C2F30722E0
:104140001448FFF715F8104840F20311FFF71DF867
:104150004FF0FF3070BDFFF7D7FF0F4B23630024F4
:10416000A54205D10D4B1D70FFF7C4FF0020F1E7FC
:104170007168204601EB0411FFF7D0FE0134EFE730
:1041800090ED00E044050600060F0600B41D060091
:10419000170206005B0F0600AAFF4400C0010220C0
:1041A00038B50C4C0D462278FFF7FAFE2070163019
:1041B0000FD1C923084A09490948FEF7D9FF294602
:1041C0000848FEF7D5FFBDE83840C9210248FEF790
:1041D000DCBF38BDC0010220060F0600B41D06007A
:1041E00017020600AB0E06002DE9F84F0E460746F3
:1041F0000025DFF8B080254CB54201DBBDE8F88F23
:10420000D7F804A0BAF1000F2DD0D7F800B0584667
:10421000FEF77EFB81460AEB0B000138FEF778FBC8
:104220001423814518BF6FF01500194A6B431278AB
:10423000C0B2824203F8080018D9A0604344A060CD
:10424000E068197B60F3040119732169E268187B47
:1042500022F01F025A602269490861F3471022F0D8
:104260001F0218731A6101350C37C5E7D923094AB3
:1042700009490A48FEF77CFF31460948FEF778FFF6
:10428000BDE8F84FD9210348FEF77FBF90ED00E06D
:10429000C0010220060F0600B41D0600170206002A
:1042A000D70E0600AC01022070B5164B0C461D78E7
:1042B00000222B46064614480168C1F307218B42B1
:1042C0001BDB124911F8040BFFF728FE2A46214692
:1042D0003046FFF765FE163013D1E8230C4A0D492E
:1042E0000D48FEF745FF21460C48FEF741FFBDE8AB
:1042F0007040E8210648FEF748BF83600261013341
:10430000DAE770BDC001022090ED00E0AC010220B0
:10431000060F0600B41D0600170206007E0E0600FA
:104320004FF0FF307047002070470000014B1860CD
:10433000704700BF14BF0220F8B506460D460024A2
:10434000064FAC4208DA3B6898470A28305504F11A
:10435000010401D00D28F4D12046F8BD10BF022081
:104360002DE9F04106460D4604460A4FA31B9D4227
:1043700002DC2846BDE8F0812378A0460A2B02D152
:104380003B680D2098473B6898F800000134984737
:10439000ECE700BF14BF022008461146FFF7CCBF70
:1043A00008461146FFF7DCBF4FF0FF307047002092
:1043B00070470120704700207047002070474FF47D
:1043C000005300204B60704708B505210148FFF7F6
:1043D000C7FFFEE78F0F0600074910B50B68C4182A
:1043E0000648C0F1005202F5802294423ABFC0183C
:1043F0000C604FF0FF3010BDC4010220ACCA022097
:1044000005F094BC7047000024218379044A01FB25
:1044100003231B6AC01A034BC0105843704700BFE8
:1044200064CA0220ABAAAAAA10B524248379094A37
:1044300004FB0323DB690A685C6823689A4294BF23
:104440000A600B60FFF7E0FFD4E9002302FB0030B5
:1044500010BD00BF64CA022010B50278A2F130037B
:10446000D9B2092905D9A2F14103052B1AD8A2F125
:10447000370342781B01A2F13001CCB2092C18D8C5
:104480000B4482781B01A2F13001CCB2092C1DD85B
:104490000B44C0781B01A0F13002D1B2092922D807
:1044A000D01810BDA2F16103052B29D8A2F1570342
:1044B000DFE7A2F14101052902D8373A1344E0E7CA
:1044C000A2F1610105291BD8573AF7E7A2F1410192
:1044D000052902D8373A1344DBE7A2F16101052927
:1044E0000ED8573AF7E7A0F14102052A02D837382B
:1044F0001844D6E7A0F16102052A01D85738F7E73A
:104500000020CEE72DE9F84F0A780646222A01F16D
:10451000010934D04FF00009624B19604846BDE8EC
:10452000F88F5C2914BF0132023201341178204621
:10453000222903D011B1601CF3D100205A4A013066
:10454000126890470746002800F0A98004464FF003
:104550000A0A4FF009084FF00D0B99F80020222AA3
:1045600000D07AB90022227099F800203761222AFF
:104570004FF0040208BF09F10109F260CEE74A4694
:104580000024D3E75C2A09F1010C03D02270013426
:10459000E146E2E799F801206E2A19D007D8622A8D
:1045A00004F101030CD0662A10D0227012E0742AA4
:1045B00012D0752A13D0722AF7D184F800B009E01E
:1045C000082222701C460CF1010CE1E70C22F8E7EE
:1045D00084F800A00134F6E784F80080FAE709F1D6
:1045E0000200FFF739FFA0F55C42B2F5806F054687
:1045F00009F1050CE7D30028E5D0A0F55842B2F543
:10460000806F3AD299F806205C2ADCD199F807200D
:10461000752AD8D109F10800FFF71EFFA0F55C4309
:10462000B3F5806F09F10B0CCDD2204BC0F309001C
:1046300003EA8525284300F58035B5F5803F23BF83
:1046400005F03F0363F07F03E370032324BF0423DB
:10465000AD0905F03F0004F1030E60F07F000EF19C
:10466000FF320EF8010CAD0905F03F0060F07F004D
:10467000541E02F8010CAD0903E07F2809D801237C
:1046800001340B4AD25C013B154304F8015C1C4425
:1046900099E7B0F5006FD0D2A21C0223E4E781466F
:1046A0003CE700BFC80102201CBF022000FC0F0035
:1046B000C40F06000346184623B102780133013ABD
:1046C0001F2AF8D9704710B530B103682BB1846840
:1046D00018190AF0D9FA204410BD1846FCE700006A
:1046E000064B10B51B6828209847044618B12822AD
:1046F00000210AF0FDF8204610BD00BF1CBF0220BB
:10470000F8B505460C4609B9002411E004227549A4
:1047100020460AF0E7FA18B90223EB60043407E0F8
:104720000522714920460AF0DDFA18B9E86005341F
:104730002046F8BD04226D4920460AF0D3FA18B984
:104740000123EB606B61E9E72378222B05D1214639
:104750002846BDE8F840FFF7D5BE2D2B05D0A3F1C4
:104760003002092A1DD8012302E04FF0FF33013443
:104770002278302A08BF01342278313A082A4FF0D3
:10478000000209D80A2014F8011B303900FB02127C
:10479000217830390929F6D953436B610323EB6043
:1047A000C6E75B2B36D10523601CEB60FFF782FF69
:1047B000037804465D2B01D10134B9E7FFF790FF80
:1047C0000646A86000289FD02046FFF773FF0146E9
:1047D0003046FFF795FFFFF76DFF0446002893D0A2
:1047E00003782C2B04D05D2BE6D0414B1C608BE76B
:1047F000FFF776FF0546002886D030604660601CD3
:10480000FFF758FF01462846FFF77AFFFFF752FFF0
:104810002E46E2E77B2BE8D10623601CEB60FFF716
:1048200049FF037804467D2BC6D0FFF759FF0646A3
:10483000A86000283FF468AF2046FFF73BFF014621
:104840003046FFF75FFEFFF735FF00283FF45CAF0F
:10485000002433693461336203783A2B02D0244B4D
:10486000186065E70130FFF725FF01463046FFF786
:1048700047FFFFF71FFF074600283FF445AF0378C7
:104880002C2B03D07D2B29D1441C51E7FFF728FFA7
:10489000054600283FF438AF30604660781CFFF7CB
:1048A00009FF01462846FFF72DFEFFF703FF00280A
:1048B0003FF42AAF2B692C612B6203783A2B02D08C
:1048C0000B4B186020E70130FFF7F4FE0146284645
:1048D000FFF716FFFFF7EEFE2E46CCE7044B1860FD
:1048E00012E700BFCB0F0600D00F0600D60F060060
:1048F000C8010220F8B5054668B30668F6B18368BA
:1049000042685C18A24201DB1E4417E0013C44EA05
:10491000640444EAA40444EA241444EA242444EA4F
:1049200024440E4B01341B68204698470C4F064622
:1049300030B93B6828689847C5E900663046F8BD3D
:10494000D5E90012FCF758FA3B6828689847C5E992
:104950000064AB68D8E70646F0E700BF1CBF022042
:1049600018BF022070B506460AF08EF9064B441CAB
:104970001B6820469847054618B122463146FCF789
:104980003BFA284670BD00BF1CBF0220000000009B
:10499000F8B5D0E9066705460C46002200233046EC
:1049A0003946FBF7F5FF80B154B102212046FFF7ED
:1049B000A1FF044610B152490AF008F92046F8BD9B
:1049C000504B02201B689847F3E76869FBF70EFD20
:1049D00032463B46FBF7BCFB41EC100B08F0F0F90C
:1049E0000022494B51EC100BFBF7E6FF00B33CA350
:1049F000D3E9002330463946FBF7DEFFC0B1002281
:104A0000424B30463946FBF7E1FF88B15CB11521D6
:104A10002046FFF76FFF04460028CFD06A693C4963
:104A20000AF03CF8CAE7374B15201B689847F2E7B5
:104A300074B340212046FFF75DFF04460028BDD037
:104A400047EC106B08F0C8F932463B4651EC100BAE
:104A5000FBF77EFB41EC100B08F0B2F900222A4B69
:104A600051EC100BFBF7A8FFB8B147EC106B08F046
:104A7000A7F91DA3D3E9002351EC100BFBF792FF1C
:104A800058B132463B46234920460AF007F895E7DD
:104A90001C4B40201B689847CFE747EC106B08F091
:104AA0008FF913A3D3E9002351EC100BFBF77AFF26
:104AB00018B132463B461849E6E747EC106B08F060
:104AC0007FF90DA3D3E9002351EC100BFBF788FF0E
:104AD0000028EED132463B461049D5E7AFF30080BF
:104AE0000000C0FFFFFFDF4144F3C2E4E4E9634C90
:104AF0008DEDB5A0F7C6B03E0000000065CDCD41FC
:104B0000B41D06001CBF02200000B03C0000E0C144
:104B1000DE0F0600E10F0600E60F0600E90F0600B3
:104B20002DE9F0470346064688460022194611F84B
:104B3000014BCCB95ABB9C1BE11CB8F1000F21D032
:104B40004046FFF7D7FE054658B12227431C0770A1
:104B5000314618460AF03AF8034600222344075526
:104B60005A702846BDE8F087631E1E2B08D9222CF8
:104B700006D0A4F15C035C425C4122430B46D5E7BE
:104B80000124FAE7414B08461B689847DBE796B9D2
:104B9000B8F1000F0AD003214046FFF7ABFE0546EF
:104BA0000028DED03A490AF011F8DAE7374B032043
:104BB0001B689847F3E7B1463778DFF8D8A017B1FC
:104BC000651C1AD12C46E11CB8F1000F23D04046D9
:104BD000FFF790FE05460028C3D022235C274FF044
:104BE0006608DFF8B490441C0370013E16F8013FDC
:104BF000B3B9222263702270B3E73946504609F0F8
:104C00006FFF20B1A51C19F8017F2C46D7E71F2F95
:104C100098BFA51DF7E71D4B08461B689847D9E7C5
:104C20001F2B04F1010006D9222B04D05C2B02D0EB
:104C300023700446DAE7277032780C2A16D009D898
:104C4000092A1AD00A2A15D0082A19D16223A01CD1
:104C50006370EEE7222A06D05C2A04D00D2A0FD119
:104C6000A01C7223F4E7A01C6270E2E7A01C84F889
:104C70000180DEE7A01C6E23EAE7A01C7423E7E7AF
:104C8000494609F00BFFA01DD3E700BF1CBF02205F
:104C9000EC0F0600EF0F0600F70F06002DE9F04FAE
:104CA00080468A4616461C460025076885B077B9B7
:104CB000ADB97CB103212046FFF71CFE824610B13E
:104CC000744909F083FF504605B0BDE8F08F013507
:104CD0003F68ECE7704B03201B689847EEE7002C19
:104CE0004BD0A368012120460193FFF703FE10B9C2
:104CF0004FF0000AE7E75B23002E0370D8F800505E
:104D000014BF4FF002084FF001084FF02C0BA368BE
:104D100008F101090133A3600AF1010A6DB902210A
:104D20002046FFF7E7FD0028E2D05D2345700370C1
:104D30002368019A1A449246C5E7234632465146F3
:104D4000284600F0ADF82046FFF7BDFC2B68A060B8
:104D50006BB149462046FFF7CDFD0028C8D080F84A
:104D600000B036B9431C1F70A3684344A3602D688C
:104D7000D4E72022831C4270F5E7DFF81C91AB00DA
:104D80000293A800D9F800309847CDF80C90074658
:104D90000028ADD04FF0050BAA00214609F0A8FD70
:104DA000D8F80090A7F10408CDF804800AF1010AB0
:104DB000B9F1000F1ED02CB1029B3D463B441C466E
:104DC000364E5AE0324623465146484600F068F8CF
:104DD000019A42F8040F019250B109F055FF331CBB
:104DE00018BF012302339B448344D9F80090DFE7C6
:104DF0000124FAE7002CDFD1039B58461B68984733
:104E000082460028D8D05B238146DFF890B009F8AD
:104E1000013B6B1E4470019358F8040F09F034FFF6
:104E2000D8F80010024602904846FBF7E5FF029BC7
:104E30009944019B9C4209D04FF02C0389F8003023
:104E40000EBB09F10109002389F80030DBF80030BE
:104E5000D8F8000001349847A542DDD1DBF80030D6
:104E6000384698475D2389F80030002389F80130DF
:104E700029E755F8040B00B19847A5423368F8D1EB
:104E80003846984734E7202309F1020909F8013C24
:104E9000D9E700BFDB0F06001CBF022018BF0220AD
:104EA00010B5002852D0047B7BB3062C4ED8DFE827
:104EB00004F00F1804212642480005211846FFF788
:104EC00019FD044610B1224909F080FE204610BDAC
:104ED00006211846FFF70EFD04460028F6D01D49AE
:104EE000F2E705211846FFF705FD04460028EDD03E
:104EF0001949E9E71946BDE81040FFF749BD1946D1
:104F0000BDE810400069FFF70BBE062C1ED8DFE895
:104F100004F0090B040D0F1117000D48BDE81040F7
:104F2000FFF720BD0B48F9E70B48F7E70021E2E760
:104F30000021E5E70023BDE810400830FFF7AEBED2
:104F40000023BDE81040083000F008B80024BDE799
:104F5000CB0F0600D00F0600D60F06002DE9F04F4C
:104F600080468B46154600271C46036889B05BB90E
:104F7000AFBB74B15DB10BF104012046FFF7BAFC81
:104F8000044678B9002415E001371B68EFE70321D8
:104F9000F3E7AE4B1B681DB10BF104009847EFE738
:104FA0000320FBE77B23037045B9431C7D221A7065
:104FB00000225A70204609B0BDE8F08F0A22831CF7
:104FC000427009251A460BF1FF31D01A814203DCE9
:104FD0000029A8BF5B18E9E702F8015BF5E7002CA0
:104FE00000F09480002D0CBF012702272046791C79
:104FF000D4F80890FFF77EFC0028C3D07B23037011
:10500000F5B9431C00224FF0090A1A70A368D8F8BA
:1050100000603B44A3600BF10108AEB9002D67D0DE
:105020000BF102012046FFF765FC0028AAD0002DF5
:1050300069D17D2303700023437024684C44B9E791
:105040000A22831C4270DDE765B141462046FFF726
:1050500051FC002896D003461A1A904545DCA368F7
:105060004344A3602146306AFFF75AFD2046FFF70C
:105070002AFB3946A0602046FFF73CFC002881D07F
:105080004FF03A0303700DB180F801A0A3682A46DF
:105090003B444146A36030462346FFF701FF2046CC
:1050A000FFF711FB2B1C18BF01233268A060002AF8
:1050B00018BF01332046591C0093FFF71BFC002842
:1050C0003FF460AF3268009B1AB12C22013000F827
:1050D000012C1DB10A22013000F8012C00220270BF
:1050E000A26836681344A36097E703F801ABB3E7FF
:1050F000022197E703F8011B1A1A9345FADC2BEA01
:10510000EB79484495E703460921F5E7DFF83CA130
:105110004FEA8709DAF800304846984706460028E3
:105120003FF430AFDAF8003048469847009020B995
:10513000474B30461B6898473CE74A462146304675
:1051400009F0D6FB4A462146009809F0D1FB0BF145
:105150000103D8F80080039325B30BF10804002D58
:105160000BF1030308BF00234FF0000A009A02333B
:10517000043A0292321F01920592029A0693049217
:10518000B8F1000F10D1BAF1000F36D0304D002425
:10519000A846A7422B6846D1009898472B6830460E
:1051A0009847EFE60724DAE70021D8F82000FFF758
:1051B000B7FC049B2A4643F8040F0493814600235E
:1051C00003994046FFF76CFE059A42F8040F0592DA
:1051D000B9F1000F0ED068B109F056FD07904846AE
:1051E00009F052FD069B1C44079B1C440444D8F85C
:1051F0000080C5E74FF0010AF9E7144B20461B6811
:10520000984704460028C1D07B230370C5B900F13C
:105210000108002388F80030039B23EAE37304931A
:105220001DB343461AE0009A52F8240000B1984793
:1052300056F82400D8F8003000B198470134A8E7A8
:105240000A2300F102084370E3E700BF1CBF0220FD
:1052500018BF02204FF0090203F8012B0399A3EBBA
:1052600008029142F6DC049B9844029B53F8040F19
:10527000029309F009FD029B8146024619684046E7
:10528000FBF7BAFD3A2208EB090308F80920002DC4
:1052900040D103F10109019B484653F8041F0193D3
:1052A00009F094FC019B186809F0EEFC7B1E9A45FE
:1052B00018BF2C2309EB00081CBF09F8003008F1C7
:1052C000010825B10A2308F1010808F8013C002370
:1052D000029ADFF8689088F800301068D9F800303A
:1052E0009847019AD9F8003010680AF1010A9847E6
:1052F000574595D1D9F8003000989847D9F8003033
:1053000030469847BDB97D2388F80030002388F8DF
:1053100001304FE64FF0090203F102095A70BAE773
:1053200003F8011BA3EB08029345F9DCBBF1000F66
:10533000A8BFD844E7E743460921F3E718BF022096
:105340002DE9F84320B9081C18BF0120BDE8F883F7
:10535000002937D08946471E17F8016F08F056FF1D
:1053600030444378C84603F00303012B08BF2036BE
:1053700019F8015B08F04AFF2B46284442783C7834
:1053800002F00302012A08BF20339E4216D008F023
:105390003DFF2044437898F8005003F00303012BAD
:1053A00008BF203408F032FF29462844437803F030
:1053B0000303012B08BF2031601AC7E7002CCBD1B3
:1053C0002046C3E70120C1E710B50A490A4A20B9BF
:1053D0000A4B0B600A4B136010BD0368074C002B8F
:1053E00008BF23460B6043680549002B08BF0B46E6
:1053F000F1E700BF1CBF022018BF022029E2040011
:1054000039E2040070B504460E4D04B970BDE3687E
:105410002668D90503D4A06808B1FFF7F3FFE36855
:10542000DA0503D4206908B12B689847E3689B0527
:1054300003D4206A08B12B68984720462B68984708
:105440003446E2E718BF02202DE9F84305460E4630
:1054500091460027FFF744F9DFF850800446C8F86A
:10546000007060B12846FFF725F901462046FFF796
:1054700047F9054630B92046FFF7C4FF2C462046C1
:10548000BDE8F883B9F1000F0BD0FFF713F90378EB
:10549000054633B12046FFF7B5FF3C46C8F800503B
:1054A000EDE7002EEBD03560E9E700BFC801022030
:1054B00000221146FFF7C8BF00231A461946FFF71E
:1054C000EFBC38B50D46846824B12946206AFFF741
:1054D00037FF08B9204638BD2468F5E749B183682D
:1054E00013B98160704713461A68002AFBD119600E
:1054F0004B60704770B505460E46144672B1106A8F
:1055000010B1074B1B6898473046FFF72BFA21462E
:1055100020622846BDE87040FFF7E0BF70BD00BFC5
:1055200018BF022008B5FFF7DBF808B10223C360FB
:1055300008BD13B58DED000BFFF7D2F8044650B14E
:105540009DED000B032380ED060BC36051EC100BA7
:10555000FBF750FA6061204602B010BD38B5054631
:10556000FFF7BEF8044628B10423C3602846FFF7BE
:10557000F9F92061204638BD08B5FFF7B1F808B148
:105580000523C36008BD08B5FFF7AAF808B10623D4
:10559000C36008BD2DE9F04180460F460025FFF7A6
:1055A000EBFF2C4606460EB1BC4202DB3046BDE89E
:1055B000F08158F82400FAF719FF41EC100BFFF7BF
:1055C000B8FF1CB9B06001340546ECE728604560BF
:1055D000F9E704F0B4BE04F0B7BE00000348044B82
:1055E0000360044B4360FFF7EFBE00BFCC01022015
:1055F000D7550400D3550400002208B511462A20CF
:10560000FEF790FA0EF0BEFD002008BD684620F0BF
:1056100007018D4601B5FEF7C7FA11F05DFAFEF7F6
:10562000B5FAFEF773F8BDE8014085467047684655
:1056300020F007018D4601B5FEF7B6FA0EF0F4FE34
:10564000FEF7A4FAFEF762F8BDE801408546704710
:10565000684620F007018D4601B5FEF7A5FA0FF068
:10566000E7FAFEF793FAFEF751F8BDE801408546E8
:105670007047002070472F2810B5044672D027DCF1
:10568000162809D012DC092806D009DC022803D02C
:10569000052801D0012817D1FEF7B2FE046010BD25
:1056A0000D28F9D00E28F7D00C28F4E72A2849D085
:1056B00005DC23283DD0292840D01828EBE72C28EA
:1056C00048D043DB2D2849D0FEF79AFE162333E05D
:1056D0006928E1D016DC362850D009DC322845D0C4
:1056E000332847D03028EFD1FEF78AFE702323E01D
:1056F000392847D03C2849D03828E5D1FEF780FE2C
:105700007F2319E07E284DD009DC732842D07D2804
:1057100044D07028D8D1FEF773FE75230CE08028A2
:105720004AD044DB8128CFD1FEF76AFE40F2D47321
:1057300002E0FEF765FE0B230360B0E7FEF760FEB4
:105740006B23F9E7FEF75CFE6D23F5E7FEF758FEE5
:105750007B23F1E7FEF754FE7C23EDE7FEF750FED6
:105760005F23E9E7FEF74CFE6A23E5E7FEF748FE14
:105770007323E1E7FEF744FE7223DDE7FEF740FE08
:105780006823D9E7FEF73CFE8023D5E7FEF738FE15
:105790007423D1E7FEF734FE7723CDE7FEF730FE22
:1057A0008C23C9E7FEF72CFE40F2D173C4E7FEF765
:1057B00027FE40F2D273BFE7FEF722FE40F2D3731A
:1057C000BAE700004FF08052014BC3F80021704748
:1057D00000E100E04FF08052014BC3F88021704798
:1057E00000E100E04FF00052014BC3F80021704788
:1057F00000E100E04FF00052014BC3F880217047F8
:1058000000E100E008B51D2000220621FEF78AF91C
:10581000BDE808401D20FEF761B908B51C20002234
:105820000621FEF77FF9BDE808401C20FEF756B9B7
:1058300008B5FFF7F2FFBDE80840FFF7E3BF00201F
:10584000704710F0400318BF0223820748BF43F09F
:10585000080318467047112814D005DCC0B106288B
:1058600015D06FF07A00704740F2111398420BD0B8
:1058700040F2012398420BD0B0F5817FF1D14FF473
:1058800082707047022070474FF487707047012084
:105890007047000008B50248FDF7AEFC002008BDC7
:1058A0000010060038B5044604B938BD6069E569E2
:1058B00004F045FD204604F042FD2C46F4E770B5A7
:1058C000044618461546FFF7BCFF2A460346204605
:1058D000BDE8704011F07ABD70B504461846154613
:1058E000FFF7AFFF2A4603462046BDE8704011F09F
:1058F000B9BDF0B591B004460D46164600214022D0
:10590000684608F0F5FF04230022AA420CDB324669
:105910002946684611F05CFE002223461646012700
:10592000AA421BDB11B0F0BD54F83210E05A4DF81A
:105930003210C10748BF3DF8031002F1010244BF15
:1059400041F001012DF80310470742BF3DF8031055
:1059500041F002012DF803100833D6E70DEBC20128
:10596000C988DE80CC0748BFDF808C0748BFDC8851
:1059700002F1010244BF44F00404DC804C0748BF3C
:10598000DC8803F1080344BF44F0080423F8024C08
:10599000090742BF33F8021C41F0200123F8021C22
:1059A000BEE711F0A1BD11F0E7BC012816D0B0F59B
:1059B0008D7F1DD1013905291AD8DFE801F00307D1
:1059C000090B150D02231360002070470523FAE729
:1059D0000623F8E70723F6E70123F4E7142905D0A7
:1059E000192903D0042903D10423ECE71160EBE764
:1059F0004FF0FF307047F0B5012985B006460C46E0
:105A000017461D4602D0B1F58D7F1FD103AA394636
:105A10002046FFF7CAFF002818DB0A9B3046009398
:105A2000039A2B46214611F0B3FD064658B955B1ED
:105A3000012C08D1042F06D12868FFF71CFEFEF7C1
:105A4000DFFC03682B60304605B0F0BDFEF7D8FCE4
:105A50006D234FF0FF360360F5E70B890222438088
:105A6000034630B523F8042B01F1100202F11004B3
:105A700052F8045BA24243F8045BF9D10B6A037548
:105A800030BD2DE9F041002514468AB0064688460F
:105A90002022294602A81F46019508F029FF64B379
:105AA0002022294602A808F023FFA3680493A388B4
:105AB000022B06D0662B05D0012B40F093800223E9
:105AC00000E00A23E0680393FFF7C5FE05907B30F2
:105AD00000F08B8002AA01AB4146304611F074FD04
:105AE0000023019E3B6098460546002857D0386841
:105AF000FFF7D8FE00233B6053E02246EBE720206F
:105B000004F022FC0446002866D07268B3680A2AB2
:105B1000C0E906550560836017D0662A17D0022AAF
:105B200066D101236360F368022B41D011DCFBB125
:105B3000012B3FD06FF07A03E360002363612046BE
:105B400004F0FDFB6FF00605D1E70223EAE71346F8
:105B5000E8E7B3F5877F09D040F201218B4207D0F7
:105B6000B3F5827FE6D14FF4817301E040F2111367
:105B7000022AE36020D1082004F0E6FB606140B314
:105B80000823236173691A89DB684280012243601C
:105B90000280B8F1000F22D13C60A046F669002EC9
:105BA000ADD1019811F012FD28460AB0BDE8F08190
:105BB0001123DDE70623DBE70A2AC0D1182004F011
:105BC000C3FB606128B1182371692361FFF745FFAA
:105BD000DFE7204604F0B3FB6FF0090587E7C8F85C
:105BE0001C40DAE76FF00805DEE76FF00605DBE73B
:105BF00004F0A5FB6FF0080579E72422F0B50A70E0
:105C0000428804460A810A220B464A6001F11006C6
:105C1000021D00F11407354610685168083203C5AB
:105C2000BA422E46F7D1227D1A62F0BD2DE9F0432B
:105C30008DB0149C05460E46174698466CB918461A
:105C4000FFF7FFFDCDE9004403463A4631462846BA
:105C500011F0A0FB0DB0BDE8F0832388012B10D11B
:105C600063881021ADF81430022304936368404622
:105C700006938DF80C10FFF7E4FD03AB0191009340
:105C8000E2E7022B0CD10DF10C0949462046FFF743
:105C9000B4FF4046FFF7D5FD2423CDE90093D3E7B9
:105CA000FEF7AEFB862303604FF0FF30D2E72DE90D
:105CB000F04380468DB01846DDE914469146FFF763
:105CC000C0FD034654B9CDE900444A46404611F0B0
:105CD000ADFB054628460DB0BDE8F08324220CAD8F
:105CE00045F8282D03AF019500974A46404611F02C
:105CF0009DFB049B0546022B09D1BDF8143063803F
:105D000001232380069B636008233360E2E70A2BAC
:105D1000E0D139462046FFF7A0FE1823F5E710B57D
:105D20000A888AB0012A04460B460ED149881022FF
:105D3000ADF80C1002215B6802918DF804200493E9
:105D400001A911F0BFFB0AB010BD022A07D101A9B9
:105D50001846FFF752FF242201A92046F1E7FEF77B
:105D60004FFB862303604FF0FF30ECE7F0B50827C8
:105D700085B0164604AA0C4642F80C7D0DEB0701CF
:105D800011F0C2FB051E1ADB039B022B0AD1BDF8E2
:105D900010303760638001232380059B63602846B1
:105DA00005B0F0BD0A2B06D1182302A933602046A6
:105DB000FFF753FEF3E7FEF723FB862303604FF064
:105DC000FF35ECE77FB50C46012C054611461E4613
:105DD00002D0B4F58D7F0FD103AA2046FFF7E5FD71
:105DE000002809DB089B039A009321463346284686
:105DF00011F0B2FB04B070BDFEF702FB6D2303602F
:105E00004FF0FF30F6E710B584B2022C0AD0662CB2
:105E100009D0012C12D0FEF7F3FA6A2303604FF089
:105E2000FF3010BD0A241046FFF715FD10F17B0F5F
:105E3000024605D1FEF7E4FA7B23EFE70224F2E7FE
:105E40002046BDE8104011F085BA10B50A888AB026
:105E5000012A04460B460ED149881022ADF80C10D9
:105E600002215B6802918DF80420049301A911F0CE
:105E700061FB0AB010BD022A07D101A91846FFF73D
:105E8000BCFE242201A92046F1E7FEF7B9FA8623D9
:105E900003604FF0FF30ECE72DE9F3410024254685
:105EA0001A4E1B4F30687A5D43680021D3F8088092
:105EB00001ABC047E8B10024164BD3E8EF2FC3E88D
:105EC000E14F0029F9D1144B144D1A78D2B9144B73
:105ED0001B682BB12968A14202D061402046984737
:105EE0000A22104910482C6006F076F802B0BDE88E
:105EF000F081019B13B90123AB401C430135042DF4
:105F0000D0D1D9E700221A70EAE700BFF8010220D9
:105F1000401006000402022020BF0220FC010220E3
:105F2000D4010220D8010220406102202DE9F8436B
:105F30000746884600240D4E0D4D27FA04F328FA33
:105F400004F21A43D20705D40134042CF5D1002001
:105F5000BDE8F883306803F0010342680021D2F8FD
:105F600004902A5DC8470028EED0F1E7F80102202E
:105F70004B100600F8B50E4803F0B2FE0D4D286038
:105F800090B100240C4E2868325D436800211F68E0
:105F90000123B847034648B90134042CF3D1BDE8C6
:105FA000F8400F21FFF7C2BF6FF012031846F8BD8B
:105FB00044100600F80102204B100600054BD3E800
:105FC000AF3F00B10360044811B102685A400A6053
:105FD000036070470402022000020220F8B5154B4E
:105FE000154E1860154803F07BFE3060F0B10025B7
:105FF000134F30687A5D436800211C684FF480734A
:10600000A047044680B90135042DF2D10D490E4850
:1060100005F0DAFF22460C490C4805F0DDFF044686
:1060200010B90146FFF7CAFF2046F8BD6FF0120411
:10603000FAE700BFD4010220F80102204410060054
:1060400040100600995E0400D80102204061022041
:1060500040EA010333F00F0301D1FFF767BF6FF090
:10606000150070470F21FFF7F3BF43689B6A03B128
:106070001847704770B54FF0FF31184804F0C8F961
:10608000174B184C1D68184B1E6823684BB91749ED
:1060900017487E23174AFDF76BF87E211548FDF758
:1060A00074F82368DB6A4BB9134911487F23114AFE
:1060B000FDF75EF87F210F48FDF767F82368324649
:1060C000DC6A0E4900232846A047044804F048FA39
:1060D000BDE870400A4B1868FFF7C7BF2C030220C9
:1060E00024BF02209C010220080302209C1006000D
:1060F000170206004F100600A71006000802022033
:10610000F0030220012230B5344B87B034481A70B6
:1061100003F0E6FD334D286018B96FF00D0007B0AD
:1061200030BD43689B68002B4DD12A685368002B13
:106130004DD12D4C23684BB92C492D4819232D4A9C
:10614000FDF716F819212B48FDF71FF823681B6887
:106150004BB9294926481A23264AFDF709F81A217E
:106160002448FDF712F8236840F201221B68002141
:10617000662098470122214B1860214B9A80214AC2
:1061800018601368013003F101031360C5D00024C7
:106190001D4804F037F91D4B1D4A1C60C3E901245A
:1061A0000A234FF45272CDE902431A491A4BCDE942
:1061B0000444CDE90044194805F0BCFD2868FFF708
:1061C00054FF2046ABE798470028AED0A5E79B6C6C
:1061D000002BAED0124910469847AAE7EC030220E4
:1061E00016060600F00302209C0102209C10060007
:1061F000170206004F100600B810060024BF022048
:106200001C030220280302202C0302200C0302207E
:1062100075600400588E022035630400400302209C
:10622000256204004368F7B55B6C054603B19847E7
:106230006B685B6B6BB12846984750B1344C354E58
:106240006B689B692BB101220DF107012846984725
:1062500008B903B0F0BD22689DF80710531C22292D
:10626000236018D07F2901D0082918D102B1013A42
:10627000022B38BF022300272748023B87542360A4
:106280003378002BDCD1254B1B78032BD8D8DFE8E3
:1062900003F012123038307880F001003070B3F51E
:1062A000807F03D94FF480732360C9E7002BFBD0B4
:1062B000194B9954E4E71A4AD35C8B42C0D1194B6D
:1062C00018684368DB6A03B198471749D1E8EF3F84
:1062D00043F00102C1E8E02F0028F7D1DB0703D427
:1062E0000839124804F071FA114B22681A60002331
:1062F000DAE7094B1A4412F8013C002BA0D00A2916
:10630000DCE7054B1A4412F8013C0D2B98D1F6E757
:10631000180302202403022008020220EC030220BA
:10632000ED100600F0030220140302204061022059
:10633000080302202DE9F043344ED3B04FF4A47289
:106340000021684608F0D4FA3446314F314B1D68BD
:1063500033684BB9304931484D23314AFCF708FFC7
:106360004D212F48FCF711FF23689B694BB92D493C
:106370002A484E232A4AFCF7FBFE4E212848FCF708
:1063800004FF23684FF0FF329B692946264898474F
:106390004FF0FF31384604F03BF8244BD3F800802F
:1063A00023684BB91C491D4869231D4AFCF7E0FED0
:1063B00069211B48FCF7E9FE23685B6A4BB91C495D
:1063C00016486A23164AFCF7D3FE6A211448FCF7E4
:1063D000DCFE23684FF4A4725D6A694640234046A0
:1063E000A8478046384604F0BBF8B8F1000FADDD91
:1063F0000025DFF840904545A8D0D9F800001DF8E9
:106400000510436801355B689847F4E79C0102205A
:106410002C030220280302209C100600170206000D
:106420004F100600CB1006001C03022024BF0220E0
:10643000DC100600F003022010B51C688C420DD25F
:10644000091B01290AD0115D2244090201805278FA
:1064500002341143018000201C6010BD6FF0150054
:10646000FBE7F0B5002426461D688D4210D210F8D7
:1064700005C001350CF07F07A7401CF0800F04F128
:1064800007043E44E4B2F0D100201D601660F0BD68
:106490006FF01500FBE710B59A42029C02D86FF02E
:1064A000150010BD90F85400042808BFC85C03F123
:1064B000010304BF00F0010020709A42EFD9CB5CC9
:1064C00000206370EDE72DE9FF411C469B7D0DF137
:1064D00010086FF30003A37548F80C2D02780546E9
:1064E00062F34103A37503780246C3F341032372A9
:1064F0000DF10E0043460E46FFF79EFF00230746B0
:10650000C4E9003300BB019BBDF80E20F11A914293
:106510000DD30AB1E918216013440193237A626014
:1065200043B9019A0023964212D2C4E903336FF0B3
:10653000150709E043462A46314604F11400FFF7E7
:106540007BFF0028EDD00746384604B0BDE8F08157
:10655000B61AC4E90333F7D01544C4E90356F3E788
:1065600037B51D4602AC44F8042D234602462846A2
:10657000FFF762FF03B030BD37B51D4602AC44F8EB
:10658000042D234602462846FFF756FF03B030BDD0
:1065900037B51D4602AC44F8042D23460246284672
:1065A000FFF74AFF03B030BD37B51D4602AC44F8D3
:1065B000042D234602462846FFF73EFF03B030BDB8
:1065C00073B506461C4602A840F8042D0346324621
:1065D00020460D46FFF730FF48B9019B9D4208D386
:1065E000ED1AC4E9010002D01E44C4E9016502B0FD
:1065F00070BD6FF01500FAE737B51D4602AC44F8E0
:10660000042D234602462846FFF716FF03B030BD8F
:1066100010B540F2FA741368A3420ED8C3F5FF64B4
:106620000334012C09D0040ACC541368194448706F
:10663000002013680233136010BD6FF01500FBE7F4
:10664000F8B5064640F2FA7013680F4683421546C5
:1066500017D87068C3F5FF630333841CA34213D3B8
:1066600080B2FFF7D5FF044648B91068D6E900129A
:106670003844FAF7C1FB2B68726813442B6020463C
:10668000F8BD6FF01504FAE76FF00B04F7E770B58B
:106690000B4600240134DB09A4B2FBD1E4431568A6
:1066A0002E1928550C4604F07F0598B2E40900F134
:1066B000010018BF65F07F0535540133002CF2D17D
:1066C0000131166011FA80F070BD2DE9F34100240C
:1066D00088461E46089F0094154622B3036840F280
:1066E000FB72053321461846019308F001F96A460A
:1066F00001462846FFF78CFF054688B90099B1F19D
:10670000805F0AD201AA4046FFF7C1FF019B3860B3
:106710003360284602B0BDE8F0814FF0FF30F5E766
:106720003C603460F5E76FF01505F2E72DE9F743BB
:106730000F460021036C90F855400546904690F8AE
:1067400054004E4A4E4E0533042808BF16461846DC
:1067500040F2FB720193009108F0CAF86A460146C4
:106760003046FFF76DFFC4F34004034670B9DDE91E
:10677000002140F2FA76B24288BF6FF0150395F817
:1067800054009FBF8854009A01320092DDF80090B7
:1067900009F101020092002B65D16A460199782027
:1067A000FFF736FF034600285DD16A46019905F1DF
:1067B0004C00FFF745FF064600285DD1E86A6400FB
:1067C000F0B16A460199FFF73BFF034600284AD122
:1067D000EB6A95F855201B7A02F00102DB0044F0C9
:1067E000040403F0180344EA42141C432B6B019980
:1067F0006A4663B31846FFF723FF0346002832D1E9
:10680000686A48B16A460199FFF71AFF034650BB10
:10681000A86AF8B944F0800495F85400C31E5842A1
:1068200058412B6C994489F805400099B1F1805F7B
:106830001FD2400001AA40F01000FFF728FF019B83
:10684000C8F800003B60304603B0BDE8F083FFF7B6
:10685000DFFED2E76A460199FFF7F2FE44F0C0047A
:1068600003460028D8D000221E46C8F800203A600F
:10687000E9E74FF0FF30E2E70346F4E704110600D2
:10688000F4100600F7B51F46002300930B7A0C4660
:10689000164613B18B8A002B54D0036C40F2FB7266
:1068A000053300211846019308F022F86A46014694
:1068B0002046FFF7C5FE054640B9237A5BB940F292
:1068C000FA72009B93420ED96FF015000023054623
:1068D0003B6033602DE06A460199A08AFFF798FE7D
:1068E0000028F3D1EBE72269C3F5FF610331914240
:1068F00025D30198E1681844FAF77EFA00992369D4
:106900001944B1F1805F009116D2A37D01AA03F072
:106910000100C3F3400343F0300343EAC003207A8D
:10692000400000F006001843FFF7B1FE019B3860FD
:106930003360284603B0F0BD4FF0FF30F6E76FF04C
:106940000B00C3E76FF01505F3E707B5098800935F
:1069500013460A4640210844FFF7B7FE03B05DF82E
:1069600004FB0000024B00200B6002231360704701
:10697000F01006002DE9F74F0D4600211F46EB8869
:1069800016460091002B3AD0036C40F2FB7205339F
:106990001846019307F0ACFF6A460146E888FFF706
:1069A00037FE044698BB80464FF00C0940F2FA7A55
:1069B00009FB08FB28686A4601995844FFF740FE26
:1069C000044620BB2B685B44197ADDE9003253454D
:1069D0001BD8D1540099AB8808F101080131434517
:1069E0000091E5D8B1F1805F02D34FF0FF3003E0B2
:1069F00001AA8220FFF74BFE3860019B09E06FF08F
:106A00001504204603B0BDE8F08F6FF01504002395
:106A10003B603360F5E72DE9F7430E4600219846C9
:106A2000036C1746053340F2FB7218460091019340
:106A300007F05EFF6A460146F088FFF7E9FD04466D
:106A4000F0B905464FF00C0930686A4609FB0500AD
:106A50000199FFF7F5FD0135044688B9B388AB42CB
:106A6000F2D80099B1F1805F02D34FF0FF3003E01C
:106A700001AAA220FFF70BFEC8F80000019B02E06C
:106A80000023C8F8003020463B6003B0BDE8F08327
:106A9000024B00200B6002231360704710110600A8
:106AA00000232DE9F04F80468A4616468FB00DF13F
:106AB000380949F8283D0393049FB74243D2039B0A
:106AC0000AEB07050593012305AA0493F11B4B4626
:106AD0002846FFF7C6FC002840F08680DDE9042444
:106AE0001444B4F5006F2DD807EB040BB3457DD8E3
:106AF0001AF807300D9003F0F003502B50D026D831
:106B0000302B39D0402B42D0202B25D107AB8DF82C
:106B1000180000932946134640462246FFF7BBFC67
:106B2000054690BB9DF81D202AB9D8F83C3043F0AB
:106B30000403C8F83C300D92002206A9404600F03C
:106B4000E3F94DB1264630460FB0BDE8F08F702B0B
:106B500038D004D8602B2CD0CDF810B0ACE7902BF7
:106B600039D0B02BF8D1082321468DF818302846AB
:106B700007ABFFF741FD07E0022321468DF81830EF
:106B8000284607ABFFF79FFC05460D95D4E7032386
:106B900021468DF81830284607ABFFF7E1FCF3E7F4
:106BA000042321468DF81830284607ABFFF7E4FC94
:106BB000EAE7052321468DF81830284607ABFFF792
:106BC000E7FCE1E7062321468DF81830284607AB9D
:106BD000FFF7EAFCD8E7072321468DF8183028464E
:106BE00007ABFFF7EDFCCFE73446ABE73C46A9E740
:106BF00070B5104C054623684BB90F490F48212347
:106C00000F4AFCF7B5FA21210D48FCF7BEFA2368BC
:106C10005B684BB90B4909482223094AFCF7A8FADB
:106C200022210748FCF7B1FA23682846BDE87040E6
:106C30005B6818479C0102209C10060017020600A2
:106C40004F100600121106002DE9F0412D4C056A87
:106C5000236806462F884BB92B492C4819232C4A08
:106C6000FCF786FA19212A48FCF78FFA23681B687B
:106C70004BB9284925481A23254AFCF779FA1A21E5
:106C80002348FCF782FA236838461B680622012154
:106C9000984700280746706005DAFDF7B1FB0068E9
:106CA0004042BDE8F0812B88356A012B236814BF70
:106CB0004FF018084FF008084BB913491348452303
:106CC000134AFCF755FA45211148FCF75EFA236890
:106CD0005B694BB910490D4846230D4AFCF748FA49
:106CE00046210B48FCF751FA236842465B69294666
:106CF00038469847002803DA7068FFF779FFCCE739
:106D00000020CEE79C0102209C100600170206001E
:106D10004F100600B8100600241106002DE9F84FA8
:106D200080468946174600241D4DBC4201D30020F1
:106D300031E0D8F8043009EB040A1E46194BA7EBE2
:106D4000040B1B684BB9184918487E232A46FCF7E8
:106D50000FFA7E212846FCF718FA124B1B68DB6AF3
:106D60004BB9134911487F232A46FCF701FA7F21CA
:106D70002846FCF70AFA0B4B30461B685A46DB6A7A
:106D800051469C4600236646B047002805DAFDF7C9
:106D900037FB00684042BDE8F88F0444C5E700BFF8
:106DA0004F1006009C0102209C10060017020600EE
:106DB000A71006002DE9F041184C0F462368154630
:106DC0004668D2F800804BB9154916486923164A1F
:106DD000FCF7CEF969211448FCF7D7F923685B6A00
:106DE0004BB912490F486A230F4AFCF7C1F96A21CF
:106DF0000D48FCF7CAF9236842465C6A39464023CD
:106E00003046A047002805DAFDF7FAFA006840424C
:106E1000BDE8F08128600020FAE700BF9C01022055
:106E20009C100600170206004F100600DC1006003A
:106E300008B54068FFF7DCFE002804DAFDF7E0FA49
:106E40000068404208BD0020FCE700000378024AC9
:106E50001B01D358184700BF3811060010B4044B6B
:106E6000047803EB04135B685DF8044B184700BF1C
:106E70003811060010B4044B047803EB04139B682C
:106E80005DF8044B184700BF381106000278024B2A
:106E900003EB0213DB68184738110600014803F0C2
:106EA0005FBB00BFF8030220030706D410F0040FF5
:106EB0000CBF6FF07F00002070476FF00F0070472D
:106EC0004FF0FF31014803F0A3BA00BFF8030220DE
:106ED00037B50025036C0446C56333B102A941F8F8
:106EE000043D084803F0C8F82564636C3BB102A96F
:106EF00041F8043D034803F0BFF80023636403B086
:106F000030BD00BF0C04022070B5446B05460E4630
:106F100044B1FFF7C3FF31462846A047BDE87040A3
:106F2000FFF7CEBF70BD00000F4B10B51A6888B0D8
:106F3000904204BF00221A60C36B044613F014038E
:106F400013BF01238DF800306FF06E03079114BF5B
:106F50008DF800300793FFF7BBFF012269462046FA
:106F6000FFF7D2FF08B010BDF403022010B50446AD
:106F7000FFF78CFF002806DB2046BDE810406FF0CD
:106F80007001FFF7D1BF10BDC36B70B513F0120FC6
:106F900005460E4609D0FFF779FF041E03DB314694
:106FA0002846FFF7C1FF204670BD6FF00C04FAE7DA
:106FB00038B5C36B044643F00803C363FFF74EFFC5
:106FC000E36B054623F00803E36338B1014620462E
:106FD000FFF7DAFF6FF00405284638BD05F01EFB09
:106FE000A063F9E710B50024084803F00BFAFFF797
:106FF00067FF074B4FF400621C60064902230648F6
:1070000002F09AFFFFF74AFF204610BDF803022066
:10701000F4030220280402200C04022037B50446A1
:1070200010B3FFF74DFF58220021204607F060FC07
:107030000423002584F8543002232A4684F855306E
:1070400001A90A4802F0A6FFA842A8BF019D00229C
:10705000256401A9054802F09DFF0028B4BF002364
:10706000019B6364FFF71AFF03B030BD0C040220DC
:1070700073B50446002845D0C36C002B42D0FFF7FF
:107080001FFF224B1A681E464AB12046FFF720FF19
:107090006FF00B05FFF702FF284602B070BD1C60C1
:1070A000236C002BF1D0636C002BEED02046FFF751
:1070B000CDFEF8B9E36B01AA43F00203E36369462E
:1070C0002046FFF733FB90B9DDE90012E36B204661
:1070D00043F00803E363FFF7C1FEE36B054623F0CB
:1070E0000803E36318B905F099FAA063D2E72046D4
:1070F000FFF73CFF2046FFF7EBFE00236FF06E0525
:107100003360C7E76FF01505C6E700BFF403022040
:1071100073B50E460546D0B1C9B1FFF7D1FEE86B95
:10712000FFF7C2FE044668B901AB6A4631462846FD
:10713000FFF7A8FB044628B9DDE900122846FFF74F
:1071400037FF0446FFF7AAFE204602B070BD6FF07D
:107150001504F9E773B50E460546D0B1C9B1FFF77E
:10716000AFFEE86BFFF7A0FE044668B901AB6A46C4
:1071700031462846FFF7E9FB044628B9DDE900124D
:107180002846FFF715FF0446FFF788FE204602B0A9
:1071900070BD6FF01504F9E737B50546D8B1FFF7B4
:1071A0008FFEE86BFFF780FE044678B901AA6946B6
:1071B0002846FFF7D7FB044640B9DDE90012284610
:1071C000FFF7F6FE044608B91023EB63FFF766FEEF
:1071D000204603B030BD6FF01504F9E773B50E46D5
:1071E0000546D0B1C9B1FFF76BFEE86BFFF75CFE57
:1071F000044668B901AB6A4631462846FFF7BAFB38
:10720000044628B9DDE900122846FFF7D1FE0446FE
:10721000FFF744FE204602B070BD6FF01504F9E799
:1072200073B50E460546D0B1C9B1FFF749FEE86B0C
:10723000FFF73AFE044668B901AB6A463146284674
:10724000FFF7E9FB044628B9DDE900122846FFF7FD
:10725000AFFE0446FFF722FE204602B070BD6FF07D
:107260001504F9E737B50546C0B1FFF729FEE86B0D
:10727000FFF71AFE044660B901AA69462846FFF7DF
:1072800007FC044628B9DDE900122846FFF790FE06
:107290000446FFF703FE204603B030BD6FF015042F
:1072A000F9E7000038B5FFF70BFE0D4B1C6834B151
:1072B000E36BDB0607D500212046FFF765FEFFF7ED
:1072C000EDFD002038BDA56B05F0A8F9054B5B1B53
:1072D0001844054B9842F2D82046FFF7C3FFEEE76B
:1072E000F4030220402BFEFF3F2BFE7F73B50446C4
:1072F000002849D0FFF7E4FDE36B13F0100605D03A
:1073000000212046FFF740FE054614E09B0738D5D4
:10731000A36C02AAC3F5006142F8041D616C20460B
:107320001944FFF7A7FD051E0ADA15F10B0F26D049
:107330002046FFF71BFEFFF7B1FD284602B070BDE7
:1073400001990029DDD0A26C20460A44A264616C38
:10735000FFF7A6FBA26C0146904207D96FF004012B
:107360002046FFF711FE6FF00405E4E7121AA2644D
:10737000002AE0D0606C014407F058FADBE735469C
:10738000D9E76FF00C05D6E76FF01505D5E70000DB
:1073900070B5104C054623684BB90F490F4821239F
:1073A0000F4AFBF7E5FE21210D48FBF7EEFE2368AF
:1073B0005B684BB90B4909482223094AFBF7D8FE01
:1073C00022210748FBF7E1FE23682846BDE870400C
:1073D0005B6818479C0102209C10060017020600FB
:1073E0004F100600121106002DE9F341154C984686
:1073F000236805460E4617464BB9134913485723D1
:10740000134AFBF7B5FE57211148FBF7BEFE236870
:10741000DB694BB90F490D4858230D4AFBF7A8FE0D
:1074200058210B48FBF7B1FE2368CDF80080DC69DA
:1074300032463B464FF48D712846A04702B0BDE866
:10744000F08100BF9C0102209C100600170206007C
:107450004F100600581106002DE9F041484D076A0B
:107460002B6804463E884BB9464947481923474A8A
:10747000FBF77EFE19214548FBF787FE2B681B684A
:107480004BB9434940481A23404AFBF771FE1A2181
:107490003E48FBF77AFE2B684FF481721B6801218E
:1074A000304698470028606005DAFCF7A9FF0068BD
:1074B0004042BDE8F081042304F108020521FFF7F2
:1074C00093FF002803DA6068FFF762FFEDE72269A7
:1074D000002A31D1A269002A39D1E669002E41D1B2
:1074E0003B886668012B2B680CBF4FF008084FF0F3
:1074F0001808276A4BB9234923484523234AFBF739
:1075000037FE45212148FBF740FE2B685B694BB9EC
:1075100020491D4846231D4AFBF72AFE46211B48E9
:10752000FBF733FE2B6842465B6939463046984785
:107530000028C8DB0020BCE7E368002BCAD09B0012
:1075400003216068FFF750FF0028C3DABBE76369D7
:10755000002BC2D09B0001216068FFF745FF002887
:10756000BBDAB0E73046D4F8048007F08DFB324632
:10757000034602214046FFF737FF0028B0DAA2E7B2
:107580009C0102209C100600170206004F10060006
:10759000B8100600241106002DE9F84F80468946F0
:1075A000174600241D4DBC4201D3002031E0D8F81D
:1075B000043009EB040A1E46194BA7EB040B1B68A9
:1075C0004BB9184918487E232A46FBF7D1FD7E2186
:1075D0002846FBF7DAFD124B1B68DB6A4BB91349EF
:1075E00011487F232A46FBF7C3FD7F212846FBF77E
:1075F000CCFD0B4B30461B685A46DB6A51469C4615
:1076000000236646B047002805DAFCF7F9FE00685B
:107610004042BDE8F88F0444C5E700BF4F100600A4
:107620009C0102209C10060017020600A71006000D
:107630002DE9F041184C0F46236815464668D2F8EC
:1076400000804BB9154916486923164AFBF790FD8F
:1076500069211448FBF799FD23685B6A4BB912490D
:107660000F486A230F4AFBF783FD6A210D48FBF799
:107670008CFD236842465C6A394640233046A04769
:10768000002805DAFCF7BCFE00684042BDE8F08146
:1076900028600020FAE700BF9C0102209C10060031
:1076A000170206004F100600DC10060008B54068FF
:1076B000FFF76EFE002804DAFCF7A2FE00684042E5
:1076C00008BD0020FCE70000014B1878704700BFA0
:1076D00028140220044B1870044B1B6813B109B125
:1076E00008461847704700BF281402202C140220B7
:1076F00038B50D4C0546237883B903688BB100F08B
:10770000E3FE50B900F03FF938B900F0F3FF20B9BB
:10771000064B2A681A600123237038BD6FF00C00F5
:10772000FBE76FF01500F8E7281402202C14022064
:10773000044B1B78012B01D801F0A4B86FF00C00AA
:10774000704700BF281402201FB50446F0B1124B49
:107750001B78072B1DD810220021684607F0C8F8B7
:1077600042F24B5302930123204669468DF80C30B8
:1077700000F00EF9044630B9684601F007F90446F6
:10778000019802F0DCFD204604B010BD6FF0150436
:10779000F9E76FF00C04F6E7281402207FB50B4BD5
:1077A0001B780C2B0FD81422002101A807F0A0F899
:1077B00005230C2001A98DF80430FFF78BFF002072
:1077C00007B05DF804FB6FF00C00F9E72814022005
:1077D00030B50F4B85B01B7805460C2B11D898B1EE
:1077E00001A900F0B5F9044640B9EB6801A803937C
:1077F00001F03CF90446029802F0A1FD204605B0D4
:1078000030BD6FF00C04F9E76FF01504F6E700BF28
:107810002814022030B50F4B85B01B7805460C2B81
:1078200011D898B101A900F093F9044640B9EB686A
:1078300001A8039301F01DF90446029802F07FFDB0
:10784000204605B030BD6FF00C04F9E76FF0150469
:10785000F6E700BF28140220014B197800F036BE6D
:107860002814022001F024B970B50D460121064606
:10787000D0E900044008084402F06CFD80B1002308
:10788000326859008A420CD8D10707D5144414F83D
:10789000012C1201D2B240F823200133C5E9003097
:1078A00070BD14F81320214449781201D2B201F0BE
:1078B0000F010A4440F823200133E1E738B543ECD7
:1078C000102B04460D46FDF734FE024628B1204633
:1078D0002946FDF70FFE002038BD6FF00B00FBE7D7
:1078E00038B5044610460D46FDF738FE024628B16D
:1078F00020462946FDF7FEFD002038BD6FF00B0045
:10790000FBE708B1FDF7DDBD704738B50546084611
:107910000C4607F0B9F921460246284607F0E2F97D
:10792000B0FA80F0400938BD38B504460D46FDF781
:10793000F9FD024628B120462946FDF7DBFD00206F
:1079400038BD6FF00B00FBE738B50D46044610B1AB
:10795000C368042B04D000236FF001006B6038BDB6
:10796000006907F091F92860013002F0EDFC6860D1
:1079700030B12A682169013207F0FAF90020EEE7F8
:107980006FF00B00EBE708B5FDF728FE002008BDFF
:107990002DE9F04F85B00091044648B95C495D4837
:1079A000A0235D4AFBF7E4FBA0215B48FBF7EDFB5E
:1079B000009B4BB959495748A123574AFBF7D8FBBD
:1079C000A1215548FBF7E1FB2046002310F8042BCA
:1079D000CDE90233524B02A953F832300193FFF73D
:1079E00043FFFDF7D0FD0646FDF7CDFD8246FDF7CE
:1079F000CAFD8146FDF7C7FD8046FDF7C4FD05467B
:107A0000FDF7C1FD0746DDE90210FDF7C3FD834622
:107A10005EB1BAF1000F08D0B9F1000F05D0B8F18E
:107A2000000F02D00DB107B1E8B93046FDF7EAFC0E
:107A30005046FDF7E7FC4846FDF7E4FC4046FDF7FD
:107A4000E1FC2846FDF7DEFC3846FDF7DBFC584636
:107A5000FDF7D8FC039802F072FC6FF00B0420468F
:107A600005B0BDE8F08F2F4B00222F492846FFF7C5
:107A700025FF019A04462D492846FFF731FF0444AB
:107A80000298F8F7A3FC0B46024629492846FFF75F
:107A900015FF284A044428494046FFF721FF2A469B
:107AA000044426494046FDF725FD019A1F49384602
:107AB000FFF716FF5A46224904443846FDF71AFDDF
:107AC000424620494846FDF715FD3A461E494846BC
:107AD000FDF710FD4A461D495046FDF70BFD3046A7
:107AE00052461549FDF706FD3046002C9ED1FDF7A4
:107AF000E3FC0546039802F022FC3046FDF782FCC9
:107B0000009B28465D6007F0BFF8009B1860A6E761
:107B10000513060017020600A91206001A13060034
:107B2000D81306000000F03F301306003A13060099
:107B30004113060048130600551306005B130600A8
:107B4000621306006A130600721306008013060013
:107B5000F8B50F46064648B92C492D48EC232D4A66
:107B6000FBF706FBEC212B48FBF70FFBB3684BB987
:107B700029492748ED23274AFBF7FAFAED21254842
:107B8000FBF703FB73684BB924492148EE23214AD4
:107B9000FBF7EEFAEE211F48FBF7F7FA4FB9204941
:107BA0001B48EF231B4AFBF7E3FAEF211948FBF7C9
:107BB000ECFAFDF7E8FC0546B8B11A4B32781A49E1
:107BC00053F82220FFF78CFEB26804461749284676
:107BD000FFF786FE164A044416492846FFF780FE42
:107BE0002418284604D0FDF70DFC6FF00B040AE0C2
:107BF000FDF762FC06462846FDF704FC7E60304631
:107C000007F042F838602046F8BD00BF1F1206009A
:107C100017020600A91206003512060055120600CA
:107C20001A1306008C1306006B1206007112060070
:107C3000761206007B12060070B505460C4659B94F
:107C40003E493F484FF487733E4AFBF791FA4FF4A1
:107C500087713C48FBF799FA5DB93B49384840F2D7
:107C60000F13384AFBF784FA40F20F113548FBF73F
:107C70008CFA6B685BB9354931484FF48873314AE7
:107C8000FBF776FA4FF488712E48FBF77EFA2B68E3
:107C90005BB92F492A4840F211132A4AFBF768FAC8
:107CA00040F211112748FBF770FA6868FDF700FCF5
:107CB0000646B0B12749FFF724FE27490546FFF7DE
:107CC00020FE2649002808BF2846FFF71AFE214952
:107CD000FFF717FE10B1C368042B05D03046FDF73F
:107CE00091FB6FF001000BE005691D492846FFF785
:107CF0000CFE30B1062323703046FDF783FB0020D5
:107D000070BD18492846FFF700FE08B10723F2E7C7
:107D100015492846FFF7F9FD08B10823EBE7134999
:107D20002846FFF7F2FD08B10923E4E71049284689
:107D3000FFF7EBFD0028DFD00A23DCE7A5110600E2
:107D400017020600A912060005130600C41106005A
:107D5000DE11060055130600EE1106006A13060038
:107D6000F611060048130600FF1106001012060067
:107D7000181206002DE9F04F044685B0894659B91E
:107D80007B497C4840F245137B4AFBF7F1F940F20E
:107D900045117948FBF7F9F9FDF7F5FB0746FDF7C3
:107DA000F2FB8046FDF7EFFB0646FDF7ECFB0546D0
:107DB00027B1B8F1000F01D006B150B93846FDF730
:107DC00021FB4046FDF71EFB3046FDF71BFB284616
:107DD0005AE0A01F042800F2B980DFE800F0033A5F
:107DE00081B78800654A66493046FFF779FD654AE4
:107DF000044665492846FFF773FD64490444284654
:107E0000FFF792FD624904442846FFF78DFD0444C4
:107E10002A4660493046FDF76DFB32465E494046D2
:107E2000FDF768FB384642465749FDF763FB384685
:107E3000002CC4D1FDF740FB05463846FDF7E2FAB9
:107E400025B3C9F80450284606F01EFFC9F8000003
:107E50008AE0FDF798FB82465048FDF77FFB83469A
:107E6000BAF1000F00D0A0B93846FDF7CBFA404672
:107E7000FDF7C8FA3046FDF7C5FA2846FDF7C2FA05
:107E80005046FDF7BFFA5846FDF7BCFA6FF00B04F9
:107E90006AE0434B002243495046FFF70FFD5A4624
:107EA000044641495046FDF725FB00223F4B40491F
:107EB0005046FFF703FD3F4A044433492846FFF785
:107EC0000FFD5246044431492846FDF713FB002CB0
:107ED0009ED05046FDF796FA5846FDF793FA97E77D
:107EE000354A29492846FFF7FBFC044690E7334A08
:107EF00025492846FFF7F4FC244904462846FFF7A5
:107F000013FD2F4904443046FFF70EFD6946044433
:107F100002A800F081FDFDF736FB824600283FF401
:107F20004DAF039A2749FFF7DBFC019A0444264929
:107F30005046FFF7D5FC5246044415492846FDF744
:107F4000D9FA002C3FF464AF5046C6E73846FDF737
:107F500059FA4046FDF756FA3046FDF753FA2846DF
:107F6000FDF750FA6FF08504204605B0BDE8F08FAC
:107F70001A13060017020600A9120600871206004F
:107F80008C120600F6110600551306005B1306005E
:107F9000921206006A13060080130600991206006A
:107FA0000000F03F301306003A13060000001840AE
:107FB0004113060048130600FF11060018120600C0
:107FC00072130600A1120600A51206002DE9F04169
:107FD00088461746044658B9444945484FF4EC735F
:107FE000444AFBF7C5F84FF4EC714248FBF7CDF873
:107FF00063685BB940493E4840F2D9133D4AFBF7FC
:10800000B7F840F2D9113B48FBF7BFF823685BB9DA
:108010003A4937484FF4ED73364AFBF7A9F84FF465
:10802000ED713448FBF7B1F8B8F1000F0BD13449CA
:108030002F4840F2DB132F4AFBF79AF840F2DB118E
:108040002C48FBF7A2F85FB92E4929484FF4EE738C
:10805000284AFBF78DF84FF4EE712648FBF795F8A8
:108060006068FDF725FA0546F0B12749FFF749FC9E
:1080700026490446FFF745FC2549002808BF20464D
:10808000FFF73FFC20490646FFF73BFC2149044629
:108090003046FFF736FC06461CB110B1E368042BEE
:1080A00005D02846FDF7AEF96FF0010411E01A493A
:1080B0002069FFF72AFC0028F3D018493046FFF763
:1080C00020FC4146FFF740FC044628B12846FDF756
:1080D00099F92046BDE8F08111493046FFF711FCBF
:1080E0003946FFF731FC0446F0E700BF05130600F0
:1080F00017020600A9120600C4110600DE110600D0
:108100006F1106008A11060055130600EE110600D5
:108110006A1306009212060018120600A112060049
:10812000A5120600002070477FB51422002101A887
:1081300006F0DEFB082301A901208DF80430FFF7CB
:10814000C9FA002007B05DF804FB10B586B00446FC
:108150001422002101A806F0CBFB062362688DF8EB
:10816000043003AB92E8030083E80300FFF7ACFAA6
:1081700001A9FFF7AFFA002006B010BD1FB510220D
:108180000021684606F0B4FB41F6852302930123E3
:10819000694606208DF80C30FFF7ECFD044650B917
:1081A000684600F0F3FB0446019802F0C8F800218D
:1081B0000620FFF78FFA204604B010BD07B54068CF
:1081C0000DF10701FFF738FD28B99DF80730062BA0
:1081D00001D1FFF7D3FF03B05DF804FB10B58AB0FF
:1081E0001022002101A806F083FB012301A907202A
:1081F00003938DF81030FFF7BDFD0446A8B901A820
:1082000000F0C4FB0446029802F099F81422002101
:108210000DEB020006F06CFB02238DF814300623F0
:1082200005A907200893FFF755FA20460AB010BDAC
:1082300010B58AB01022002101A806F059FB41F6C2
:10824000D2630393012301A90A208DF81030FFF7B0
:1082500091FD044698B901A800F098FB04460298E5
:1082600002F06DF8142200210DEB020006F040FB35
:10827000032305A90A208DF81430FFF72BFA2046B6
:108280000AB010BD10B5446886B00DF10701204654
:10829000FFF7D2FC48B99DF80730072B07D00A2B0F
:1082A00008D0062B01D1FFF769FF06B010BDFFF71C
:1082B00095FFFAE702AA04A92046FFF787FE0028E7
:1082C000F3D102A904A800F091FBFFF7B1FFECE79E
:1082D00030B545688BB00DF103012846FFF7ACFCC3
:1082E000044660B99DF80330063B042B07D8DFE84D
:1082F00003F003091E450C00FFF740FF044620462B
:108300000BB030BDFFF76AFFF8E701AA05A92846C0
:10831000FFF75CFE04460028F1D101A905A800F092
:1083200065FBFFF785FF044600F0B8FBE7E7102286
:10833000002101A806F0DCFA012301A9082003931B
:108340008DF81030FFF716FD04460028D7D101A89C
:1083500000F01CFB0446029801F0F1FF14220021FA
:108360000DEB020006F0C4FA02238DF81430062348
:108370000720089305A9FFF7ADF9C0E714220021F3
:108380000DEB020006F0B4FAFF2305A98DF81430B6
:108390000F20F0E77FB5016859B9142201A806F053
:1083A000A7FA04230C200DEB03018DF80430FFF72E
:1083B00091F9002007B05DF804FB08B541F22E6387
:1083C00042689A4203D100210520FFF783F900207B
:1083D00008BD41F22E62436810B5934205D10021D9
:1083E0000520FFF777F900240BE041F6D2629342B3
:1083F000F9D100F021FB044618B901460B20FFF724
:1084000069F9204610BD000010B5044686B0002171
:10841000142201A806F06CFAFF2321688DF80430BD
:1084200039B101A90F20FFF755F90024204606B005
:1084300010BD0420FFF74EF9064800F0A7FA0446E5
:1084400020B1022001A9FFF745F9EFE70146052019
:10845000F9E700BFD014060007B540680DF1070129
:10846000FFF7EAFB38B99DF80730062B03D100F07F
:1084700003FBFFF783FE03B05DF804FB10B5036850
:1084800086B053B1FF2301A902208DF804300024E7
:10849000FFF720F9204606B010BD012301A90220F4
:1084A0008DF80430FFF716F900F05EFA0446002854
:1084B000F0D101460320FFF70DF9EBE700207047EC
:1084C0000020704700207047002070470F2910B52A
:1084D00008D8BDE810400B4B027A53F8213053F80E
:1084E0002230184740F20313074A08490848FAF7B0
:1084F0003FFE40F203110448FAF747FE6FF0150003
:1085000010BD00BF8C15060008150600B41D06003E
:108510001702060030B50D4687B0044668B3102236
:10852000002102A806F0E4F9154B8DF80850D3F8A5
:1085300088200092D3F88C20019222681AB16168D9
:1085400009B1CDE90312A2683AB1ADF81420694629
:108550000C48FEF7DDFD07B030BDD3F89820511C64
:1085600088B230B1C3F89810D3F89830ADF8143011
:10857000EDE70232C3F89820F6E76FF01500EAE75E
:10858000781402209014022000232DE9F0418CB0D1
:10859000CDE90333CB69074602930B780C46082BD1
:1085A00034D8DFE803F0305A0554333333444D00F8
:1085B00000254FF00C082D4E08FB05F3F21851680A
:1085C000A26860688A4228BF0A46995906F08AFB69
:1085D000F8B9274B53F825308DF82C30238B0A93AC
:1085E000236909936369089303238DF8103008AB5E
:1085F0000393237B012B06D1238B0CA921F82C3D5F
:108600003846FEF7A7FD02A8FFF726F90CB0BDE833
:10861000F0810135032DCFD1238B07932369069376
:108620006369059305238DF8103005ABE0E740F250
:10863000D2428B88934212D101238DF81030E2E7A9
:1086400040F2D2438A889A42E0D10723F5E7042317
:108650008DF810308B880393D5E70923EDE742F2BC
:108660003D229342D2D10223E7E700BF4416060021
:108670006816060010B5084CD4F8900008B101F057
:108680005EFED4F8880008B101F059FE0023C4E969
:108690002433C4E9223310BD7814022070B5124C83
:1086A00004F118063046FEF7B9FC04F17003A36329
:1086B0000E480F4B6066E36406F0E6FA042384F884
:1086C0006C300023C4E90F33012304F12005A066B8
:1086D00023760FCC0FC594E8030085E803003046ED
:1086E000BDE87040FEF7C4BC781402206414022078
:1086F00089850400002130B54A4C85B040F2012242
:108700006620C4E92411C4E922110EF023FE051EDF
:1087100009DA45494548FB23454AFAF729FDFB217B
:108720004348FAF732FD0722424928460EF068FE18
:10873000072809D040493D48FE233D4AFAF718FD75
:10874000FE213B48FAF721FD0F22694628460EF02C
:10875000A3FE0F280BD03949344840F20113344AA4
:10876000FAF706FD40F201113148FAF70EFD002339
:10877000334A8DF80F3014216B46324806F046F923
:1087800028460EF0F9FD58B12F49284840F207134A
:10879000274AFAF7EDFC40F207112548FAF7F5FCF5
:1087A000284B2A4A27212A4806F030F9262803D0E8
:1087B0006FF00B0005B030BD224B264A342126480D
:1087C00006F024F93328F3D11E4B244A34212448DF
:1087D00006F01CF93328EBD11A4B224A34212248E7
:1087E00006F014F93328E3D1164B204A2E212048F5
:1087F00006F00CF92D28DBD1124B1E4A2B211E4806
:1088000006F004F92A28D3D100230222A360C4E988
:1088100000230123E360194B2361194B6361FEF7C9
:10882000E1FBC7E7781402201D17060017020600B7
:10883000BD1606002F170600371706004A17060058
:108840005B17060064140220621706006B1706000F
:10885000481502208117060030140220A4170600D4
:1088600014150220C71706009A150220EA17060001
:10887000CE150220071806006F15022028BF02201F
:10888000211806000023012270B52E4C8AB0CDE9D4
:108890000232CDE9042323684BB92B492B4893239B
:1088A0002B4AFAF765FC93212948FAF76EFC2368F6
:1088B0005B6B4BB9274925489423254AFAF758FCA6
:1088C00094212348FAF761FC236802AA5D6B00211A
:1088D00001AB2148A847054600282CD1019B002B5D
:1088E0002CD01A69082A29D15B695A681B4B5A6730
:1088F0001B4A1A67FFF7D2FE05462368019E4BB953
:10890000114912489B23124AFAF732FC9B21104866
:10891000FAF73BFC23689B6B4BB912490B489C232D
:108920000B4AFAF725FC9C210948FAF72EFC23682C
:1089300030469B6B984728460AB070BD6FF0010522
:10894000DBE700BF9C0102209C1006001702060016
:108950004F1006008C16060021180600781402201D
:10896000010022B3A416060007B56B46054A92E83B
:10897000030083E8030019460348FEF72FFC03B009
:108980005DF804FB50FF05009014022030B504464A
:1089900087B008B3057B012D21D81022002102A841
:1089A00005F0A6FF0C236B430E49CA18CB58009361
:1089B00053680193137A8DF8083023681BB16268FD
:1089C0000AB1CDE90323A36869460748ADF814301E
:1089D000FEF79EFB07B030BD6FF01500FAE76FF0B1
:1089E0008500F7E7741606009014022038B5054696
:1089F0000C46FFF73FFE6A68064BC3F888202A68DA
:108A0000C3F88C206268C3F890202268C3F89420D1
:108A100038BD00BF78140220064BD3F8882042608E
:108A2000D3F88C200260D3F89020D3F894304A60B9
:108A30000B607047781402207FB50A4801A9D0F86E
:108A4000903018300393C36F049301238DF81430D2
:108A500003AB0193044B0293FEF7C0FB07B05DF834
:108A600004FB00BF7814022001003D220121FFF722
:108A700051BD0021FFF74EBD07B56B46054A92E890
:108A8000030083E8030019460348FEF7C9FB03B05F
:108A90005DF804FB58FF05009014022008B5FFF7AD
:108AA000E9FDBDE808400148FEF776BB90140220BE
:108AB00008B50348FEF71AFCBDE80840FEF7F2BB14
:108AC0009014022038B513460C4661B9074D18467C
:108AD00095F851202946F8F78FF995F8512080F83C
:108AE0005120204638BD6FF08500FBE7EC1A0220CC
:108AF0002DE9F04F8DB003F091FD4FF4FA654FF67C
:108B0000FF74B0FBF5F0B0FBF4F3C3EB0343C01A02
:108B1000F7F75CFC41EC100B04F0E6F965A3D3E930
:108B2000002351EC100BF7F7CBFC64A3D3E900232F
:108B3000F7F710FBCDE90A0103F070FDB0FBF5F08B
:108B4000B0FBF4F4C4EB0444001BF7F73FFC41EC2A
:108B5000100B04F0D5F85BA3D3E9002351EC100B04
:108B6000F7F7AEFC59A3D3E90023F7F7F3FA0F4662
:108B7000064603F053FD4FF47A73B0FBF3F0484C14
:108B8000484923780A68484D9B1A0344DBB23B2BC3
:108B900023700860DFF83C811BD93C21B3FBF1F264
:108BA00001FB123323702B780133DBB23B2B2B708C
:108BB0000FD9B3FBF1F001FB1033182198F8002016
:108BC0002B70531CDBB2B3FBF1F201FB123388F8BC
:108BD00000300022DDE90A010023F7F7E3FE002858
:108BE0004FD0DDE90A214FF0530901F10043CDE9EF
:108BF0000A230022002330463946F7F7D3FE002827
:108C000042D007F100431F464FF0570A9DED0A7B03
:108C10004FF0000B8DED027BCDE908ABCDE9066787
:108C2000CDF81090227898F8003001922A785121DE
:108C300000921E481E4A05F0E9FE1C4B5A469B4610
:108C400003F1520013F8011F2A2920D19DED0A7B60
:108C50008DED027BCDE908A2CDE90667CDF8109035
:108C6000227898F8003001922A78512100920F481A
:108C70000F4A05F0CBFE8BF8510000200DB0BDE887
:108C8000F08F4FF04E09B4E74FF0450ABEE783423C
:108C900001D04A40D6E70022D8E700BFAFF30080FA
:108CA0002EBF0220E81A02202DBF0220EC1A02205B
:108CB0005C1806009A9999999999A93FE17A14AE9E
:108CC00047B5B8409A9999999999B93FFCA9F1D2B9
:108CD000CD0890402CBF02200B7870B5012B0D46BB
:108CE000164684680CD14FF0FF31074801F090FB25
:108CF0002B8805482663A38601F032FC002070BD56
:108D00006FF08500FBE700BF401B022070B50646F0
:108D100086B0FAF7E5FC05F041FE0C480024B56882
:108D200001F070FB6FF00503CDE90444CDE9024387
:108D3000CDE90064064B4FF4806205F1380105F57A
:108D4000876002F0F7FF204606B070BD401B02208E
:108D5000558D040070B5054686680A4C4FF4FA60DC
:108D600002F04CFD4FF0FF31204601F051FB336B18
:108D70001BB106F1340128469847204601F0F0FB6C
:108D8000ECE700BF401B022070B5104C054623687D
:108D90004BB90F490F4821230F4AFAF7E9F921216E
:108DA0000D48FAF7F2F923685B684BB90B4909489B
:108DB0002223094AFAF7DCF922210748FAF7E5F9F4
:108DC00023682846BDE870405B6818479C01022074
:108DD0009C100600170206004F1006001211060034
:108DE00010B5114C23684BB9104911481923114A89
:108DF000FAF7BEF919210F48FAF7C7F923681B687B
:108E00004BB90D490A481A230A4AFAF7B1F91A214F
:108E10000848FAF7BAF9236840F20122BDE8104089
:108E20001B680021662018479C0102209C10060048
:108E3000170206004F100600B810060070B5134C5C
:108E4000054623680E464BB9114912486923124A58
:108E5000FAF78EF969211048FAF797F923685B6AE7
:108E60004BB90E490B486A230B4AFAF781F96A217C
:108E70000948FAF78AF9236831465C6A2846A4460D
:108E8000BDE8704000238022604700BF9C010220A3
:108E90009C100600170206004F100600DC100600AA
:108EA000F0B51B4CA1B0236805460F4616464BB9DA
:108EB000184919487E23194AFAF75AF97E211748AA
:108EC000FAF763F92368DB6A4BB9154912487F2327
:108ED000124AFAF74DF97F211048FAF756F923683C
:108EE0003246DC6A394600232846A04786420BD129
:108EF00069462846FFF7A2FF012805D902226946E4
:108F0000084805F065FC08B16FF0040021B0F0BD21
:108F10009C0102209C100600170206004F1006005C
:108F2000A7100600E81806002DE9F041A0B0FFF7F1
:108F300057FF431C04463ED00A222049FFF7B0FFEA
:108F4000054630B12046FFF71FFF284620B0BDE898
:108F5000F08109221A492046FFF7A2FF05460028A2
:108F6000F0D1184E184FDFF8688069462046FFF7A9
:108F700065FF18B90A2002F041FCF6E709226946AC
:108F8000304605F025FC0028DCD00822694638462A
:108F900005F01EFC0028D5D009226946404605F0A0
:108FA00017FC0028CED008226946084805F010FCBE
:108FB0000028DFD1C6E76FF00D05C6E7DD18060013
:108FC000A3180600B7180600C1180600D41806003A
:108FD000CA18060038B5FFF703FF431C054609D041
:108FE00009220649FFF75CFF04462846FFF7CCFE3E
:108FF000204638BD6FF00D04FAE700BFAD1806003B
:10900000D0B514460F460646F7F7F4FC2060F7F794
:10901000EDF902460B4630463946F7F799F804A3B6
:10902000D3E90023F7F74CFAF7F7E4FC6060D0BD12
:109030000000000080842E4183680878012801BF69
:109040001A630A8800209A8618BF6FF0850070475F
:109050000020704738B5144610292FD8DFE801F0FA
:10906000090D14182E2E2E2E2E2E2E2E2E282C2E9E
:109070002A00144BD3E9000102E0124BD3E90201AC
:10908000FFF7BEFF002038BD0E4BD3E90401F7E720
:109090000C4DD5E90001FFF7B3FFD5E9020104F15A
:1090A0000802FFF7ADFFD5E9040104F11002E7E77C
:1090B000054BDFE7054BDDE7054BDBE76FF0850090
:1090C000E1E700BF581B0220681E0220701B02202F
:1090D000781B022008B503F0A1FA4FF6FF73B0FB2E
:1090E000F3F3C3EB0343C01AF7F770F941EC100B2D
:1090F00003F0FAFE0022054B51EC100BF7F7E0F9F4
:1091000000220023F7F726F808BD00BF0000344016
:1091100030B56FF005030024856887B04FF4007206
:1091200005F13801CDE90243CDE90004064BCDE954
:10913000044405F50E7002F0FDFDFAF7D1FA05F0D2
:109140002DFC204607B030BD4D91040070B504469B
:10915000856805F134064FF47A7002F04FFB2B6BF3
:10916000002BF8D0314620469847F4E70000000075
:10917000F8B5102900F2A680DFE801F009203040A0
:10918000A4A4A4A4A4A4A4A4A46890A47D00544C62
:10919000FFF7A0FF2068F7F729F9524B0022064697
:1091A0000F46F7F78DF9504BC3E90001304607F140
:1091B0000041F7F71FFC20600020F8BD484CFFF786
:1091C00089FF2068F7F712F9464B002206460F4642
:1091D000F7F776F9444BC3E90201E7E7404CFFF7A4
:1091E00079FF2068F7F702F93E4B002206460F464A
:1091F000F7F766F93C4BC3E90401D7E7FFF76AFFCD
:10920000394C374DC4E90001012002F0F7FAFFF7AD
:1092100061FFC4E90201012002F0F0FAFFF75AFFF2
:109220002868F7F7E3F800222E4B06460F46F7F7BB
:1092300047F9C4E90001C4E90201C4E90401304668
:1092400007F10041F7F7D6FB2860B5E705F0AEFB64
:10925000F7F7CCF81EA3D3E90023F7F75BFA002257
:10926000224BF6F775FF224B0022F6F773FF214BD6
:10927000C3E90001A0E705F099FBF7F7B7F814A3DD
:10928000D3E90023F7F746FA0022184BF6F760FF00
:10929000194B0022F6F75EFF184BE9E705F086FB55
:1092A000F7F7A4F80AA3D3E90023F7F733FA00226B
:1092B0000E4BF6F74DFF08A3D3E90023F6F74AFF5C
:1092C0000F4BD5E76FF0850077E700BFAFF3008065
:1092D0000000C0FFFFFFCF41CDCCCCCCCC8C5840A0
:1092E00030BF022000003440581B02200000F03F35
:1092F00000003540681E022000004A40701B02201A
:10930000781B022010B504688068A46801292468CD
:10931000C06903D158406060002010BD00334FF099
:10932000010118BF0123D04000F0010091408342A9
:1093300014BFA160E160EFE770B504688068A468BD
:10934000C069256801296E692C696D6880EA04008E
:1093500084EA050404EA060480EA04001CBFD04045
:1093600000F001001860002070BD000070B51646C6
:1093700084680D4661B922491C23224A2248F9F724
:10938000F7FE2248F9F7F4FE1C211E48F9F7FDFE0E
:109390006B6863B91E491D231A4A1B48F9F7E8FE9A
:1093A0001C48F9F7E5FE1D211648F9F7EEFE236883
:1093B0005BB100229D4213D12B685AB962682360C9
:1093C000954200D1636000232B6076B9002070BD08
:1093D0000B46EFE7136063689D4208BF6260F2E7E7
:1093E00019681A460029F3D13EB123682B606068E2
:1093F00025600028EAD16560E9E76FF01500E6E72F
:109400007E190600341906001702060087190600A7
:1094100096190600A819060008B5034A034B40F246
:10942000DD11034804F0B2FEFC180600D419060052
:10943000E21906001F2808B501D9FFF7EDFF084B18
:1094400003EB8000D0F8003223F44033C0F8003240
:10945000D0F8003243EA0141C0F8001208BD00BF55
:10946000002584402DE9F041036801F01F049B684A
:109470000D461B79484E44EA43140023D6F80423D2
:109480008768D2B203F5A27156F82110C1F3042106
:109490008C4266D122FA03F1C90762D59A0002F123
:1094A000804202F54432D2F8101521F00101C2F8D1
:1094B0001015012202FA03F3C6F8083320460021F2
:1094C000FFF7B8FFB868E84010F0010047D0F8682F
:1094D000E84010F0010042D07869E84010F001083F
:1094E0004BD0BB69EB40DB073FD43B69FA69EB40EB
:1094F00022FA05F503F0010305F00105AB420CBFAC
:1095000002250125002202F5A27356F8230010F06F
:1095100003002CD1930003F1804303F54433D3F8C7
:109520001015240221F4473121F44071C3F81015BD
:10953000D3F8101504F4F85444EA05450D431749CF
:10954000C3F8105541F82200D3F8101541F001017D
:10955000C3F81015012303FA02F2C6F80423BDE88C
:10956000F0810133082B8DD1A8E70325CAE701322A
:10957000082AC8D16FF01200F1E73B69FA6920466A
:10958000534023FA05F515F0010F0CBF032102210A
:10959000FFF750FF4046E2E7001003400011034090
:1095A00001292DE9F04118BFD4B2064612BF254665
:1095B0001F2500244FF001088768AC4202D9002023
:1095C000BDE8F081FB6808FA04F223EA0203FB60BD
:1095D00021463046FFF746FF0028F1D10134E4B2BE
:1095E000EBE7000008B5094B1A786AB90121312070
:1095F00019700521FAF796FA3120FAF76FFA4FF051
:109600000042034BC3F80423002008BD701E022053
:10961000001003402DE9F74F8046856803F4704041
:10962000B0F5804F1E4649D02CDCB0F5805F3DD0B0
:10963000B0F5405F3ED060BB06F44077B7F5807F61
:109640003ED0A7F5007463426341012919BFD4B22B
:10965000A1464FF01F0900244FF0010B06F0010C4A
:109660004FEA4C0747EA0C0747EA0020DFF8D0A092
:1096700040EA830706F00203A14523D2002003B08D
:10968000BDE8F08FB0F5E04F16D005DCB0F5A04F87
:109690000ED06FF01500F2E7B0F5404F04D0B0F5F2
:1096A000504FF6D10720C7E70620C5E70120C3E7E2
:1096B0000320C1E70420BFE70520BDE70220BBE788
:1096C0000323C2E7D8F800209268117904F01F0242
:1096D00042EA41121F2A01DDFFF79EFE80324AF85E
:1096E0002270A9680BFA04F2002B25D01143A9605F
:1096F0006969B0064CBF114391436961A96970065D
:109700004CBF11439143A961296970074CBF1143B4
:1097100091432961E96930064CBF0A4321EA0202FC
:10972000EA61214640460193FFF79CFE0028A6D13E
:109730000134E4B2019B9FE721EA0201D7E700BFB1
:10974000002584402DE9F047524F3E68012E74D128
:10975000B0464FF0000A504A93681268DC69D2F8AC
:109760000890D3E902251540D3E905210A4325EAEB
:109770000205D9F800201B6912695C40544025EAB3
:109780000404002D46D13D60002301279E46434D31
:10979000DFF814C1D5F8042307FA03F111420FD002
:1097A00003EB0C0292001168012909D103F5A270A4
:1097B00055F82000C2F800E0C0F3042081400C43BB
:1097C0000133082BE6D1002C39D0334883681D685B
:1097D000ADB380462F68DFF8D490DFF8D4A0AB6833
:1097E0001C4213D06B6863B951463D234A462C484E
:1097F000F9F7BEFC2B48F9F7BBFC3D214846F9F7C9
:10980000C4FC6B682246294640469847BFB13D4696
:109810003F68E4E715EA080F0AD099F804300AF027
:109820001F00002140EA4310FFF704FE25EA080567
:109830000AF1010A4FEA4808A3E70024A4E7012E31
:109840000ED10027144B9D681B68D3F80880D5E91A
:1098500002341C40D5E90532134324EA03040CB951
:10986000BDE8F087264212D02B69EA6998F804C057
:109870005340FB4013F0010F07F01F000CBF032102
:10988000022140EA4C10FFF7D5FD24EA0604013717
:109890007600E4E77C110340B4C9022000100340C5
:1098A00017020600A819060040C40010341906006B
:1098B000C819060001292DE9F04118BFD4B20646A7
:1098C00012BF25461F2500244FF001088768AC42CF
:1098D00002D90020BDE8F081FB6808FA04F21343C6
:1098E000FB6021463046FFF7BDFD0028F2D1013470
:1098F000E4B2ECE783681A7D72B10268926812687C
:10990000D2F8201141B14FF48071C2F8081301213F
:10991000D16000221A7570479A680AB1D86810475A
:109920007047000070B54B79012B23D18B79032B45
:1099300020D1CC792CB1012C1CD103689B689B7978
:10994000C3B10A7912B1022A14D10E2247F61226A7
:1099500003689B681D680B68B3426BD027D8B3F5CA
:10996000965F61D012D8B3F5167F4DD005D8B3F508
:10997000967F74D06FF0850052E0B3F5966F50D0AB
:10998000B3F5166FF6D14FF41D233FE0B3F5615FD9
:109990004CD004D8B3F5165FECD1324B36E0B3F5BA
:1099A000964F45D0B3F5E14FE4D12F4B2EE0B3F500
:1099B000E13F48D012D84DF6C026B3423DD005D87D
:1099C000B3F5164FD6D14FF41D031FE0B3F5614F29
:1099D00036D0B3F5963FCDD1244B17E0B3F5E12F48
:1099E00037D008D8B3F5613F30D0214EB342C1D152
:1099F0004FF080630AE0B3F5612F2DD01D4EB342C6
:109A0000B8D14FF0805301E04FF41C33C5F8243532
:109A10008368224303C9C5F86C2583E8030000204E
:109A200070BD4FF49E23F1E7134BEFE7134BEDE7C7
:109A3000134BEBE74FF40003E8E74FF46503E5E76A
:109A40004FF46B03E2E74FF0EB73DFE74FF06C731B
:109A5000DCE74FF0E863D9E74FF07063D6E74FF4E7
:109A6000A033D3E70050270000C0750000903A01F2
:109A700090D0030040420F0000B0130000F03A0005
:109A800000A04E000B46826892E8030083E80300C2
:109A900000207047036882689B681B68D3F8100138
:109AA00038B1527D00200A700122C3F810011A60FB
:109AB00070474FF0FF30704782B002AA02F8011DD4
:109AC000002103689B681B68C3F82011C3F8442574
:109AD0000122C3F848259A60D3F820110029FBD051
:109AE000DA6002B0704703689B681B68D3F82401F2
:109AF00018B1D3F88004C3F8800470470368F0B548
:109B00009E6800243568D5F82031ABB18768B088ED
:109B100023469042A8BF1046C5F8204183423A69C7
:109B200006DB0123C5F84425C5F84805AB60F0BD48
:109B3000CC5CD4540133F1E71846F8E703689B681E
:109B40001A68D2F8103143B183680020C2F81001BE
:109B500001205B7D0B7010607047184670474FF412
:109B6000807103689B681A688368C2F80413002236
:109B70001A757047012283681A75704703689B68DD
:109B80001B68D3F8200118B1D3F80403C0F30020F8
:109B9000704703689B681B68D3F81001003018BF3A
:109BA00001207047102203689B681B68C3F80423D8
:109BB0007047102203689B681B68C3F8082370472E
:109BC0004FF4007203689B681B68C3F80423704756
:109BD0004FF4007203689B681B68C3F80823704742
:109BE000012070478368C3E90212704708B5036813
:109BF00002469B681968D1F80433DB0505D4D1F817
:109C0000040310F0100006D108BDFFF7B7FF0028CD
:109C1000F5D00120F8E71046FFF7BBFF003018BF72
:109C20000120F1E770B50646002201210820F9F76E
:109C300079FF0820F9F752FF4FF000523368B568FA
:109C40009B6803211C681A4B1D209A600022C3F8F0
:109C50007412C3F87022C4F80C051C20C4F8140553
:109C60004FF000609860C3F86C12C3F868221B23A1
:109C7000C4F808351A232946C4F810353046FFF7D2
:109C800051FE98B90823C4F8003505F11503C4F84E
:109C90001001C4F8343501232A69C4F8383523602B
:109CA000C4F84425C4F84805A360E36070BD00BF54
:109CB0000025844070B50026084B53F82040013041
:109CC00053F82050A54200D870BD236820465B6839
:109CD000984700B166600C34F4E700BF8C1A0600A8
:109CE000104B70B505461E460F4C9C4204D10E4CDD
:109CF000B44209D1002412E062681AB122681268E5
:109D0000AA420CD00C34F0E763680BB90C34EFE7CF
:109D1000236828461968F7F7E5F80028F6D12046A9
:109D200070BD00BFFCC902203CC90220014B9868ED
:109D300054307047FC600220F9F70EBC08B50A4D9C
:109D40004FF02002EFF3118382F3118802F0F4FA4E
:109D5000012104460228D8BF084602F02BFB2C62E2
:109D6000F9F77CFFECE700BFFC6002200248034AE1
:109D70000021121A04F0BCBD00000220D478022099
:109D800008B50648064A0749121AF7F735F8BDE83C
:109D90000840054A05490648F7F72EB8E0BE0220FC
:109DA000ACCA0220344F060000000000344F060009
:109DB0000000022008B50220FFF77CFF0748F9F7F2
:109DC000D7F90320FFF776FF02F010F8F8F760FCF0
:109DD000034A137B23F00103137308BDB41A060072
:109DE000601F022080B5394BB2B083F3088800248D
:109DF000E022374B012783F82220DC771C765C7643
:109E00009C765A6A334E42F4E0225A62F9F75EFEBB
:109E1000F9F71EFF07ABAC222146184604F068FD97
:109E2000B06020468DF82970FFF744FF3846FFF7F1
:109E300041FF01F031FC284B284DCDE90473072385
:109E40004FF40052CDE90243CDE90044244B2549AB
:109E50002846756201F0BCFE6B7B23F0040213F010
:109E60001B0F6A7304D1AB6913B9284601F074F86B
:109E70001D4B0024059301220F231C4FCDE9033213
:109E80001B494FF4A0723846CDE901440094194BA8
:109E900001F09EFE7B7BF76023F004037B73164B7F
:109EA000C6E90633FAF70AF8B560144B83F309885C
:109EB00062B661B684F311880848FAF727F823469A
:109EC000224621460648F8F755FF00BFE0BA0220B7
:109ED00000ED00E0FC600220A41A0600601F0220D2
:109EE000B59D0400A0910220A91A0600B41E02200C
:109EF000A0B102203D9D040014610220A0B1022007
:109F000070B500240A4B0B48834201D3002070BD7A
:109F100000211A699D685C61A94201D11C33F3E7F5
:109F20005E6901311660DE685A613244F4E700BFB1
:109F3000FCC9022034CA0220F8B51E46C368044694
:109F40009B070D4617460CD00E4950230E4A0F486A
:109F5000F9F70EF90E48F9F70BF950210A48F9F70D
:109F600014F90023C4E90267C4E9053325619E4260
:109F700002D1C4E90044F8BD626901332A60656119
:109F80003D44F4E7CD1B06008B1B060017020600BC
:109F9000FC1B0600F8B504460D4616464FF020039C
:109FA000EFF3118783F31188284801F053FE60B95D
:109FB00027494C23274A2848F9F7DAF82748F9F7C0
:109FC000D7F84C212348F9F7E0F8E3689B070CD059
:109FD00023496423234A2048F9F7CAF82248F9F7AD
:109FE000C7F864211F48F9F7D0F86369DBB12B602B
:109FF00063691B686361A3690133A361002413488B
:10A0000001F03AFE60B919495C23124A1248F9F787
:10A01000AFF81748F9F7ACF85C210E48F9F7B5F836
:10A0200087F3118810E01EB92E606FF00B04E6E78D
:10A03000224633463946054801F0DCF9044618B992
:10A040000C4B9B685B692B602046F8BD0C200220FE
:10A05000371B0600F41A0600170206004C1B060008
:10A06000CD1B06008B1B0600FC1B0600611B0600B7
:10A07000781B0600FC60022070B504460D464FF0C8
:10A080002003EFF3118683F31188214801F0E2FDEC
:10A0900060B920494C23204A2048F9F769F8204844
:10A0A000F9F766F84C211C48F9F76FF8204601F0E3
:10A0B0005FFA80B100212A6881664261427BD20644
:10A0C00003D183690BB900F047FF3146BDE870400A
:10A0D0000F4800F04BBD2B6862690D481A602B6871
:10A0E0006361A369013BA36101F0C6FD60B90D493D
:10A0F0005C23094A0948F9F73BF80B48F9F738F8A7
:10A100005C210548F9F741F886F3118870BD00BF5E
:10A110000C200220371B0600F41A06001702060066
:10A120004C1B0600611B0600781B060038B5074C67
:10A13000074DAC4201D3002038BD04F11403204682
:10A14000C4E90533F8F72AFC1C34F2E734CA0220CC
:10A1500050CA02202DE9F04F064685B00D4617463D
:10A160001C46EFF305830D2B05D8002B5BD0374B36
:10A170005B681A0557D4002C48D10022344B904616
:10A18000F31A344A9B1002FB03FA06F1140B5FFA30
:10A190008AFA009503AB02AA39463046F8F749FC23
:10A1A00010F10B0F0BD1009503AB02AA39463046D4
:10A1B000F8F73FFC10F10B0F08BF6FF00B006B7945
:10A1C000029A85F804A062F303036B716B68039A2B
:10A1D00062F31F336B60B0B1ACB110F10C0F12D150
:10A1E0004FF02003EFF3118083F311882246594684
:10A1F00001F0EEF8631CCCD002F0C4F9B8EB000417
:10A20000C7D56FF00A0005B0BDE8F08F12493923B9
:10A21000124A1348F8F7ACFF1248F8F7A9FF3921A2
:10A220000E48F8F7B2FF002CA7DD02F0ABF94FF4AF
:10A23000004C002180460C484FF4A0220023CCFBA8
:10A240000401F6F7FFFB18EB000297E700ED00E0D2
:10A2500034CA0220B76DDBB65B1C06001A1C060070
:10A260001702060031050600FFFF040070B50478F0
:10A2700002684178204DC4EBC404A400120B01F025
:10A280000F012819F8F7A8FC4FF02003EFF311860F
:10A2900083F31188194801F0DDFC60B918494C239B
:10A2A000184A1948F8F764FF1848F8F761FF4C217D
:10A2B0001448F8F76AFF04F11400284401F0D6F9B5
:10A2C00028B13146BDE870400C4800F04FBC0B4847
:10A2D00001F0D2FC60B90E495C230A4A0A48F8F73B
:10A2E00047FF0C48F8F744FF5C210648F8F74DFF9C
:10A2F00086F3118870BD00BF34CA0220F4600220CA
:10A30000371B0600F41A0600170206004C1B060055
:10A31000611B0600781B060007B504228A1804D2C8
:10A3200000236946FFF716FF18B1002003B05DF85F
:10A3300004FBDDE900321A6000980430F6E710B142
:10A340000438FFF793BF704701460148FFF7E4BFA9
:10A3500034CA022070B5A0FB014535B92046FFF78D
:10A36000F3FF064618B9304670BD0026FBE72246CB
:10A37000294604F0BDFAF6E7034B01469B68186EC8
:10A3800008B1FFF7C9BF7047FC60022010B5EFF3BA
:10A3900005830D2B04D883B1134B5B681B050CD4CC
:10A3A0001249FB23124A1348F8F7E2FE1248F8F765
:10A3B000DFFEFB210E48F8F7E8FE104CA268D27BC6
:10A3C000012A0CD10E49FC23094A0A48F8F7D0FEAD
:10A3D0000948F8F7CDFEFC210548F8F7D6FEA2683B
:10A3E000D37B013BD37310BD00ED00E0371D0600A9
:10A3F000EF1C06001702060031050600FC60022073
:10A40000431D06000023C0E90000C0E90233704785
:10A41000F8B504460E46FFF7B9FFE368484A4BB16A
:10A42000A1689068814212D09EB900F019FD6FF0CA
:10A430000F050AE0916891F90E100133E36093680B
:10A440002161A36000F00CFD00252846F8BD2169BC
:10A45000F3E790F90E5091F90E309D42A8BF1D46CA
:10A4600025EAE5754FF02003EFF3118783F3118898
:10A47000344801F0EFFB60B933494C23334A344888
:10A48000F8F776FE3348F8F773FE4C212F48F8F7BB
:10A490007CFEA06890F90E309D4202DA294600F059
:10A4A000D7FF334622463946264800F0A3FF05462B
:10A4B00010B900F0D5FCC8E7236825699C4207D095
:10A4C00033B193F90E309D42A8BF1D4625EAE575CC
:10A4D0004FF02003EFF3118683F31188194801F040
:10A4E000B9FB60B918494C23184A1948F8F740FEDF
:10A4F0001848F8F73DFE4C211448F8F746FEA068CE
:10A5000090F90E309D4202D0294600F0A1FF0D487F
:10A5100001F0B2FB60B910495C230C4A0C48F8F713
:10A5200027FE0E48F8F724FE5C210848F8F72DFEB8
:10A5300086F3118800F094FC6FF00A0585E700BFF0
:10A54000FC600220F8600220371B0600F41A0600A7
:10A55000170206004C1B0600611B0600781B060054
:10A56000C36870B5044663B94149DC23414A424897
:10A57000F8F7FEFD4148F8F7FBFDDC213D48F8F710
:10A5800004FE3F4BA2689B689A420CD03D49DD23F4
:10A59000384A3948F8F7ECFD3848F8F7E9FDDD218D
:10A5A0003448F8F7F2FDFFF7F1FEE368012B05D020
:10A5B000013BE360BDE8704000F052BC4FF0200367
:10A5C000EFF3118683F311882F4801F043FB60B944
:10A5D0002E494C232E4A2848F8F7CAFD2D48F8F793
:10A5E000C7FD4C212A48F8F7D0FDA068216990F9F1
:10A5F0000E30994201D000F02BFF204600F0B8FF4A
:10A600000546A060F8B1437BDB0603D183690BB933
:10A6100000F0A2FC1C4801F02FFB60B91E495C232E
:10A620001B4A1548F8F7A4FD1C48F8F7A1FD5C216A
:10A630001748F8F7AAFD86F311880023AB6695F951
:10A640000E302361B6E7E0600F4801F015FB60B9FA
:10A6500011495C230E4A0848F8F78AFD0F48F8F7BD
:10A6600087FD5C210A48F8F790FD86F31188A1E781
:10A67000B81C0600791C060017020600310506000A
:10A68000FC600220CF1C0600F8600220371B060089
:10A69000F41A06004C1B0600611B0600781B06001E
:10A6A0002DE9F84304460D469046994600F1080608
:10A6B0004FF02003EFF3118783F31188304601F048
:10A6C000C9FA60B930494C23304A3148F8F750FD97
:10A6D0003048F8F74DFD4C212C48F8F756FDB9F1FC
:10A6E000000F2AD00820FFF747FEB0B9304601F02E
:10A6F000C3FA60B928495C23244A2548F8F738FD95
:10A700002648F8F735FD5C212048F8F73EFD87F331
:10A7100011886FF00B00BDE8F8830123C0F80480B6
:10A720000360036803F003035DB922681343036009
:10A730006368206073B960600CE0C8F80090404620
:10A74000EFE72A6832F0030215D16268036062B94C
:10A75000C4E90000042104F10C0002F0C1FA304603
:10A76000394600F003FA0020D5E7136803F003032D
:10A7700003431360DFE7134303602B6803F0030315
:10A7800018432860E6E700BF371B0600F41A0600EE
:10A79000170206004C1B0600611B0600781B060012
:10A7A00010B5044630B10268930703D0446809B17C
:10A7B000FFF7C5FD204610BD0023C0E900338360CC
:10A7C00000F10C03C0E9033370470A4600234168D7
:10A7D000FFF766BF2DE9F04F044689B00F4600F140
:10A7E00008054FF02003EFF3118883F31188284602
:10A7F00001F030FA60B95F494C235F4A5F48F8F7CF
:10A80000B7FC5F48F8F7B4FC4C215B48F8F7BDFC97
:10A81000206810B30368626823F00303904208BF06
:10A82000636023600121FFF7BBFF0646284601F065
:10A8300023FA60B953495C234F4A5048F8F798FC13
:10A840005148F8F795FC5C214B48F8F79EFC88F3DB
:10A850001188304609B0BDE8F08F28469FB901F055
:10A860000BFA60B947495C23434A4448F8F780FC37
:10A870004548F8F77DFC5C213F48F8F786FC88F3F3
:10A8800011880026E5E701F0F7F960B93D495C233E
:10A89000394A3A48F8F76CFC3B48F8F769FC5C2108
:10A8A0003548F8F772FC88F311880022234604210A
:10A8B00003A801F0DFFF7A1C02D001F0AFFE83464F
:10A8C0004FF00009DFF8B080DFF8B0A0069BA7EBDF
:10A8D00009026FF31033012103A8069302F020F858
:10A8E00008B10B30CDD14FF02003EFF3118283F389
:10A8F00011882846019201F0ADF960B91D494C2339
:10A9000042465046F8F734FC1D48F8F731FC4C211C
:10A910004046F8F73AFC206838B10368626823F0D3
:10A9200003039042236008BF63600121FFF738FFF3
:10A930000646284601F0A0F960B912495C23424658
:10A940005046F8F715FC1048F8F712FC5C21404619
:10A95000F8F71BFC019B83F31188002E7FF479AF7D
:10A960007B1CB3D001F05AFEA0EB0B094F45ADDACA
:10A9700087E700BF371B0600F41A0600170206001F
:10A980004C1B0600611B0600781B0600437BDB06A0
:10A9900003BF8069B0FA80F04009002070470000D2
:10A9A000EFF305800D2809D828B1054B586880F4CD
:10A9B0000060C0F3C02080F0010070470120FAE77A
:10A9C00000ED00E008B5F8F771FE054B054A1B687D
:10A9D0000021184410611846BDE8084001F0EABCA7
:10A9E00038610220FC600220036810B504465BB9A0
:10A9F000064907484FF4C273064AF8F7B9FB4FF40B
:10AA0000C2710448F8F7C1FB206810BDF51D0600AF
:10AA100017020600B61D060090F90E0091F90E30DF
:10AA20009842ACBF0020012070470000F8B50746EF
:10AA30000D464FF02003EFF3118483F311881C4877
:10AA400001F008F960B91B494C231B4A1B48F8F771
:10AA50008FFB1B48F8F78CFB4C211748F8F795FB48
:10AA600000224FF400460021164B17481A61C6FB1E
:10AA700007014FF4A0220023F5F7E4FF134B186001
:10AA8000134B1D60FFF79EFF094801F0F5F860B910
:10AA900010495C23084A0948F8F76AFB0E48F8F7A2
:10AAA00067FB5C210448F8F770FB84F31188F8BD5C
:10AAB00030610220371B0600F41A06001702060058
:10AAC0004C1B0600FC600220FFFF040038610220DE
:10AAD00034610220611B0600781B060038B504466D
:10AAE0004FF02003EFF3118583F31188184801F02C
:10AAF000B1F860B917494C23174A1848F8F738FBE2
:10AB00001748F8F735FB4C211348F8F73EFB04F1E2
:10AB10000800FFF769FF214600F0E8F8637B0C4866
:10AB200023F00203637301F0A7F860B90D495C23B9
:10AB3000094A0A48F8F71CFB0B48F8F719FB5C2197
:10AB40000548F8F722FB85F311880023A36038BD80
:10AB500030610220371B0600F41A060017020600B7
:10AB60004C1B0600611B0600781B060010B5024650
:10AB70000C46FFF715FFA8B1104601F07DF860B94B
:10AB800012497323124A1348F8F7F2FA1248F8F7F9
:10AB9000EFFA73210E48F8F7F8FA2046BDE81040A6
:10ABA000F8F7CEBD104601F067F860B907495C239D
:10ABB000074A0848F8F7DCFA0748F8F7D9FA5C21A1
:10ABC0000348F8F7E2FA84F3118810BD611B060010
:10ABD000F41A060017020600781B060008B50246A4
:10ABE000FFF7DEFE20B1BDE808401046F8F7A8BD2B
:10ABF00082F3118808BD4FF02003EFF3118083F337
:10AC00001188FFF7EBBF000038B54FF02003EFF3DA
:10AC1000118583F31188284801F01CF860B9274991
:10AC20004C23274A2748F8F7A3FA2748F8F7A0FA51
:10AC30004C212348F8F7A9FAEFF305830D2B04D82C
:10AC400083B1224B5B681B050CD42149FB23214AAD
:10AC50001C48F8F78DFA2048F8F78AFAFB211D48BE
:10AC6000F8F793FA1D4CA268D27B012A0CD11C493B
:10AC7000FC23184A1348F8F77BFA1748F8F778FAD4
:10AC8000FC211448F8F781FAA268D37B013BD37307
:10AC9000094800F0F1FF60B912495C23084A0948ED
:10ACA000F8F766FA1048F8F763FA5C210448F8F7F9
:10ACB0006CFA85F3118838BD30610220371B06001D
:10ACC000F41A0600170206004C1B060000ED00E017
:10ACD000371D0600EF1C060031050600FC6002204F
:10ACE000431D0600611B0600781B0600124B10B5C1
:10ACF00003F1280282420C4605D19B688B4202D1A7
:10AD00004B7BDB0617D10D4B1B689C420BD10C49CA
:10AD10000C4840F275230C4AF8F72AFA40F27521E4
:10AD20000948F8F732FAD4E900231A602268536020
:10AD30000023C4E9003310BDFC600220B01A0600F5
:10AD40007C1D060017020600B61D060038B5044635
:10AD50004FF02003EFF3118583F311881B4800F0B7
:10AD600079FF60B91A494C231A4A1B48F8F700FAD0
:10AD70001A48F8F7FDF94C211648F8F706FA04F1DD
:10AD80000800FFF731FE2146FFF7B0FF637B0F4855
:10AD900023F00203637300F06FFF60B910495C2376
:10ADA0000C4A0D48F8F7E4F90E48F8F7E1F95C2190
:10ADB0000848F8F7EAF985F31188002304F1180030
:10ADC000A360BDE8384001F071BA00BF30610220D5
:10ADD000371B0600F41A0600170206004C1B06007B
:10ADE000611B0600781B06000368984214BF1846D2
:10ADF0000020704738B5154C024604F12800FFF7D3
:10AE0000F3FF054600B9E568CAB9A36863B91049FC
:10AE10007F23104A1048F8F7ABF91048F8F7A8F963
:10AE20007F210C48F8F7B1F9A3685A7BD20606D106
:10AE3000AA6922B9DA897F2A01D9636238BDA36879
:10AE4000AB4201D0FFF7BEFD6562F7E7FC60022070
:10AE50000C1E0600B61D060017020600310506008E
:10AE600038B5304CA268D27B72B92F4940F2192311
:10AE70002E4A2F48F8F77CF92E48F8F779F940F276
:10AE800019212A48F8F781F9EFF305830D2B04D82F
:10AE900093B1294B5B681B050ED4284940F21A2355
:10AEA000224A2348F8F764F92248F8F761F940F29A
:10AEB0001A211E48F8F769F94FF02003EFF31185C6
:10AEC00083F311881E4800F0C5FE60B91D494C236C
:10AED0001D4A1748F8F74CF91C48F8F749F94C2176
:10AEE0001948F8F752F9A2680120D37B0133D373D4
:10AEF000FFF780FF124800F0BFFE60B914495C23E1
:10AF0000114A0B48F8F734F91248F8F731F95C2187
:10AF10000D48F8F73AF985F31188BDE83840FFF796
:10AF20006ABE00BFFC6002208E1D0600B61D060032
:10AF3000170206003105060000ED00E0371D06008F
:10AF400030610220371B0600F41A06004C1B060075
:10AF5000611B0600781B0600F8B504464FF020037D
:10AF6000EFF3118583F311882D4800F073FE60B96B
:10AF70002C494C232C4A2D48F8F7FAF82C48F8F7BE
:10AF8000F7F84C212848F8F700F92A4B1B689C4237
:10AF90000BD12949254840F25F23284AF8F7E8F801
:10AFA00040F25F212548F8F7F0F8254A02F1280120
:10AFB000D2E90A308B420BD053B194F90E6093F969
:10AFC0000E70B7420ADC984202D01B68002BF6D103
:10AFD000C4E90010D36A1C60D46205E05A68C4E971
:10AFE00000325A6814605C60637B002043F04003C9
:10AFF0006373FFF7FFFE0A4800F03EFE60B9114997
:10B000005C23094A0948F8F7B3F80F48F8F7B0F895
:10B010005C210548F8F7B9F885F31188F8BD00BF41
:10B0200030610220371B0600F41A060017020600E2
:10B030004C1B0600B01A06007C1D0600B61D06005B
:10B04000FC600220611B0600781B060050F8103CD3
:10B0500070B50446A0F11805002B39D04FF020033D
:10B06000EFF3118683F31188214800F0F3FD60B9F6
:10B0700020494C23204A2148F8F77AF82048F8F76D
:10B0800077F84C211C48F8F780F8A4F11000FFF77E
:10B09000ABFC2946FFF72AFE14F80B3C144823F0BA
:10B0A000020304F80B3C00F0E7FD60B915495C238E
:10B0B000114A1248F8F75CF81348F8F759F85C2180
:10B0C0000D48F8F762F886F31188002344F8103C25
:10B0D00014F80B3C284623F0040304F80B3CFFF75C
:10B0E00055FC20B12846BDE87040FFF735BF70BD64
:10B0F00030610220371B0600F41A06001702060012
:10B100004C1B0600611B0600781B0600F8B50446C0
:10B110004FF02003EFF3118583F31188304800F0DE
:10B1200099FD60B92F494C232F4A3048F8F720F891
:10B130002F48F8F71DF84C212B48F8F726F8214640
:10B140002C48FFF7D3FD2C4B1B689C420BD12B499D
:10B15000264840F25F232A4AF8F70AF840F25F21B6
:10B160002748F8F712F8274A02F12801D2E90A30F5
:10B170008B420BD053B194F90E6093F90E70B74225
:10B180000ADC984202D01B68002BF6D1C4E90010FB
:10B19000D36A1C60D46205E05968C4E9003159687B
:10B1A0000C605C60637B906843F040036373031B37
:10B1B00058425841FFF71EFE094800F05DFD60B996
:10B1C00011495C23084A0948F7F7D2FF0F48F7F7FF
:10B1D000CFFF5C210448F7F7D8FF85F31188F8BD4D
:10B1E00030610220371B0600F41A06001702060021
:10B1F0004C1B060024610220B01A06007C1D0600CC
:10B20000B61D0600FC600220611B0600781B0600CC
:10B2100010B51449144C8B68226893424FF0000219
:10B22000226003D1BDE81040FFF7CCBB0F4A126883
:10B23000BAB1DA897F2A14D80D4A93F90E40126800
:10B2400094420EDB0B4A126893420AD09A6942B9C3
:10B250000A69824203DC1846FFF758FFE2E7121A38
:10B260000A6110BDFC6002202C61022038610220BE
:10B2700034610220B01A060070B504464FF0200376
:10B28000EFF3118683F311881B4800F0E3FC60B9EB
:10B290001A494C231A4A1B48F7F76AFF1A48F7F76E
:10B2A00067FF4C211648F7F770FF637B5B060FD5ED
:10B2B000164D214605F12800FFF718FDA868637BAD
:10B2C000021B23F04003504263735041FFF792FD8D
:10B2D000094800F0D1FC60B90D495C23084A0948CF
:10B2E000F7F746FF0B48F7F743FF5C210448F7F7F1
:10B2F0004CFF86F3118870BD30610220371B0600B9
:10B30000F41A0600170206004C1B0600FC6002201F
:10B31000611B0600781B060070B504460D461646F4
:10B32000FFF7AAFF637B43F002036373002D2DD068
:10B33000214BA5601B689C420BD12049204840F25C
:10B340005F23204AF7F714FF40F25F211D48F7F70B
:10B350001CFF2B689D420CD05BB194F90E2093F931
:10B360000E1091420CDC69688B4202D01B68002BE6
:10B37000F5D16B68256063606B681C606C6005E0EC
:10B380005A68C4E900325A6814605C60731C12D0B9
:10B390004FF4004500210C484FF4A022C5FB0601E4
:10B3A0000023F5F74FFB0949421C04F11800BDE8E2
:10B3B000704000F0DBBE70BDB01A06007C1D0600B8
:10B3C00017020600B61D0600FFFF04004DB0040082
:10B3D00010B50446054B9868054B1860FFF79CFFB5
:10B3E0002046BDE81040F8F7ABB900BFFC60022072
:10B3F0002C61022038B505460C4611460E4A90686D
:10B400000E4A10601A46FFF787FF284600F034FC0A
:10B4100060B90B4973230B4A0B48F7F7A9FE0B4899
:10B42000F7F7A6FE73210748F7F7AFFE2046BDE801
:10B430003840F8F785B900BFFC6002202C6102207B
:10B44000611B0600F41A060017020600781B0600AE
:10B45000F8B504460D464FF02003EFF3118683F351
:10B460001188374800F0F6FB60B936494C23364A5C
:10B470003648F7F77DFE3648F7F77AFE4C2132481A
:10B48000F7F783FE2046FFF781FA6DB207460028E2
:10B4900052D021462F48FFF729FC2F4BA5731B687C
:10B4A0009C420BD12D49294840F25F232C4AF7F7E3
:10B4B0005FFE40F25F212A48F7F767FE294A02F152
:10B4C0002801D2E90A308B420BD053B194F90E50C7
:10B4D00093F90EC0AC450ADC834202D01B68002BF6
:10B4E000F6D1C4E90010D36A1C60D46205E05A6842
:10B4F000C4E900325A6814605C600120FFF77AFCEE
:10B500000F4800F0B9FB60B917495C230E4A0F4899
:10B51000F7F72EFE1548F7F72BFE5C210A48F7F7E0
:10B5200034FE86F311884FB10E4B9B68DB7B2BB941
:10B53000BDE8F840FFF75FBBA573E1E7F8BD00BFCA
:10B5400030610220371B0600F41A060017020600BD
:10B550004C1B060024610220B01A06007C1D060068
:10B56000B61D0600FC600220611B0600781B060069
:10B5700038B504464FF02003EFF3118583F31188AB
:10B58000334800F067FB60B932494C23324A3348F4
:10B59000F7F7EEFD3248F7F7EBFD4C212E48F7F7B1
:10B5A000F4FD2046FFF720FC0446294800F064FB28
:10B5B00060B92C495C23284A2848F7F7D9FD2A4866
:10B5C000F7F7D6FD5C212448F7F7DFFD85F31188F6
:10B5D000002C3AD04FF02003EFF3118583F311884C
:10B5E0001B4800F037FB60B91A494C231A4A1B4824
:10B5F000F7F7BEFD1A48F7F7BBFD4C211648F7F7E1
:10B60000C4FD04F10800FFF7EFF92146FFF76EFBD8
:10B61000637B0F4823F00203637300F02DFB60B9D6
:10B6200010495C230C4A0D48F7F7A2FD0E48F7F7C6
:10B630009FFD5C210848F7F7A8FD85F311880023DA
:10B6400004F11800A36000F031FE204638BD00BFB1
:10B6500030610220371B0600F41A060017020600AC
:10B660004C1B0600611B0600781B060070B50646E1
:10B6700000253468A64200D00CB9284670BD20468B
:10B68000FFF764FB2046FFF781F901250028F0D081
:10B690002046FFF761FCECE70021044B084603F16C
:10B6A0002802C3E90A22FFF7C1B900BFFC600220EB
:10B6B000F8B5EFF305830D2B04D893B1404B5B68CD
:10B6C0001B050ED43F4940F267333F4A3F48F7F726
:10B6D0004FFD3F48F7F74CFD40F267313A48F7F726
:10B6E00054FD3C4D3C4EA968326891425DD04FF00C
:10B6F0002003EFF3118783F31188384800F0AAFA8A
:10B7000060B937494C23374A3048F7F731FD36489E
:10B71000F7F72EFD4C213348F7F737FDA96833487A
:10B72000FFF7E4FAAC6833689C420BD130492748F4
:10B7300040F25F23244AF7F71BFD40F25F212248C5
:10B74000F7F723FDD5E90A31284A93420BD053B1CC
:10B7500094F90E0093F90E6086420ADC994202D0F9
:10B760001B68002BF6D1C4E90021EB6A1C60EC6277
:10B7700005E05A68C4E900325A6814605C60012030
:10B78000FFF738FB154800F077FA60B919495C23D8
:10B79000144A0E48F7F7ECFC1748F7F7E9FC5C2170
:10B7A0001048F7F7F2FC87F311884FF02003EFF30E
:10B7B000118083F31188BDE8F840F7F7C1BF00BFDF
:10B7C00000ED00E0371D0600B61D0600170206005A
:10B7D00031050600FC600220B01A0600306102202C
:10B7E000371B0600F41A06004C1B060024610220D9
:10B7F0007C1D0600611B0600781B06002DE9F34145
:10B800000446EFF305830D2B04D893B1434B5B68DB
:10B810001A050ED4424940F27E33424A4248F7F7B5
:10B82000A7FC4248F7F7A4FC40F27E313D48F7F709
:10B83000ACFC631C67D13E4940F27F33394A3A4839
:10B84000F7F796FC3948F7F793FC40F27F3135481B
:10B85000F7F79BFC4FF40045002136484FF4A02237
:10B860000023C5FB0401F5F7EDF8461C00F0D2FEFD
:10B87000002302AD341845F8043D4FF02003EFF3E8
:10B88000118883F31188284600F0E4F960B92A4949
:10B890004C232A4A2448F7F76BFC2948F7F768FC41
:10B8A0004C212648F7F771FC264F274BB8681860E3
:10B8B000FFF7E2FCB86832461830244900F056FC25
:10B8C000284600F0D9F960B9214973231B4A16486C
:10B8D000F7F74EFC1F48F7F74BFC73211748F7F7B3
:10B8E00054FC4046F7F72CFF00F094FE201A002885
:10B8F00011DD4FF47A716422002380FB0101F5F71A
:10B90000F1F8044603E0002CA4D1FFF7D1FE204655
:10B9100002B0BDE8F0810024F9E700BF00ED00E0CF
:10B92000371D0600B61D0600170206003105060089
:10B930006B1D0600FFFF0400371B0600F41A06000B
:10B940004C1B0600FC6002202C6102204DB004005C
:10B95000611B0600781B0600014B9868704700BF0A
:10B96000FC60022070B504460E46154662B91249C5
:10B970004623124A1248F7F7FBFB1248F7F7F8FB89
:10B9800046210E48F7F701FCB5420CD20E49472379
:10B990000A4A0B48F7F7ECFB0C48F7F7E9FB47219D
:10B9A0000648F7F7F2FB04F11003C4E90265C4E9A5
:10B9B0000044C4E9043370BD681E06002B1E060057
:10B9C00017020600741E06008B1E0600A21E06004B
:10B9D00070B504464FF02003EFF3118683F311880E
:10B9E000184800F037F960B917494C23174A18482E
:10B9F000F7F7BEFB1748F7F7BBFB4C211348F7F7E7
:10BA0000C4FB2046FFF7B4FD054670B1437BDB065F
:10BA100003D183690BB9FFF79FFA0023AB66314668
:10BA2000BDE870400748FFF7A1B8D4E902329A4256
:10BA300018BF01330221A36004F1100001F050F996
:10BA4000EDE700BF3C610220371B0600F41A060038
:10BA5000170206004C1B060070B505460E46EFF3B4
:10BA600005830D2B04D88BB1304B5B681B050DD4BF
:10BA700066B12F498C232F4A2F48F7F779FB2F48BF
:10BA8000F7F776FB8C212B48F7F77FFB4FF020036D
:10BA9000EFF3118483F31188294800F0DBF860B9D3
:10BAA00028494C23284A2448F7F762FB2748F7F730
:10BAB0005FFB4C212448F7F768FBAB68B3B1013B4F
:10BAC000AB601F4800F0D8F860B921495C231E4ADA
:10BAD0001948F7F74DFB1F48F7F74AFB5C211A4856
:10BAE000F7F753FB84F31188002070BDAEB91448FA
:10BAF00000F0C2F860B916495C23134A0E48F7F704
:10BB000037FB1448F7F734FB5C210F48F7F73DFB90
:10BB100084F311886FF00F00E7E733462A46214689
:10BB2000BDE870400648FFF765BC00BF00ED00E0CF
:10BB3000C71E06002B1E0600170206003105060070
:10BB40003C610220371B0600F41A06004C1B06005D
:10BB5000611B0600781B060010B5084C4FF0FF3340
:10BB60004FF480622046064900F00AFA04F11400FE
:10BB7000044900F02BF8002010BD00BF40610220F6
:10BB8000E0BA0220ED1E0600437BDB0603BF80699E
:10BB9000B0FA80F04009002070470000EFF3058004
:10BBA0000D2807D838B1044B586880F40060C0F302
:10BBB000C02070470120704700ED00E0024B9B68F9
:10BBC000187B00F001007047FC6002207047000005
:10BBD00030B587B00E9D044604950D9D03950C9DD0
:10BBE00002950B9D01950A9D0095F7F7DFFF044B29
:10BBF0009B6813B9236607B030BD1B6EFAE700BF20
:10BC0000FC600220036D10B5044603B1984720463E
:10BC1000FFF7BAFF38B12046FFF72EFB637B43F0F6
:10BC20000803637310BD637B9B0702D52046FEF7B4
:10BC300055FFA369002BF1D004F1180000F036FB8A
:10BC4000ECE70373002342738173C373C0E90633C7
:10BC500070470000074B0268197D1AB102F0030219
:10BC60008A4204D09B680B43036001207047002088
:10BC7000704700BFFC600220064A117D936802688D
:10BC80000B439A424FF0000306BF036001201846A1
:10BC9000704700BFFC60022038B504464FF0200317
:10BCA000EFF3118583F311881B48FFF7D3FF60B9C9
:10BCB0001A494C231A4A1B48F7F75AFA1A48F7F759
:10BCC00057FA4C211648F7F760FA637B5A0713D4EA
:10BCD0001148FFF7D1FF60B914495C23104A11489D
:10BCE000F7F746FA1248F7F743FA5C210C48F7F7E2
:10BCF0004CFA85F3118838BD23F0040363732046A2
:10BD0000FFF742FF10B12046FFF726F92946BDE8AC
:10BD100038400148FEF72ABF04620220371B0600A4
:10BD2000F41A0600170206004C1B0600611B0600F1
:10BD3000781B06002DE9F04186B004460E461746F2
:10BD40009846119DEFF305830D2B04D893B1204B3A
:10BD50005B681A050ED41F4940F2AD131E4A1F48F6
:10BD6000F7F706FA1E48F7F703FA40F2AD111A4842
:10BD7000F7F70BFA00230593109B3A4604930F9BA9
:10BD8000314603930E9B204602930D9B01930C9B1F
:10BD900000934346FFF71CFF6B1C03D035B92046C8
:10BDA000FFF77AFF204606B0BDE8F0814FF4004669
:10BDB00000210C484FF4A0220023C6FB0501F4F734
:10BDC00041FE0949421C04F1180000F0CFF9E9E7EF
:10BDD00000ED00E0371D0600F61E06001702060003
:10BDE000361F0600FFFF04004DB004002DE9F04FA0
:10BDF000284E294DB04687B0B54205F130040FD327
:10BE0000FEF702FF4FF400490027234C234EDFF8D2
:10BE100090A0444521D307B0BDE8F04FFFF720B80C
:10BE200054F8043C059354F8103C049354F8143C23
:10BE3000039354F8183C029354F81C3C019354F8B3
:10BE4000203C009354E90A2354E90C01FFF7C0FE9B
:10BE500054F8303CDD642546CEE7616A4B1C04D0C3
:10BE6000256821B92846FFF717FF3034D1E7B346DC
:10BE7000BC46C9FB01BC4FF4A022002358466146D2
:10BE8000F4F7E0FD5146421C05F1180000F06EF990
:10BE9000EBE700BFFCC90220FCC90220FFFF040041
:10BEA0004DB0040000B501F10803D3E8EF2F42F0D4
:10BEB000010CC3E8EECFBEF1000FF6D1D30703D4D7
:10BEC0005DF804EBFEF781BC5DF804FBA0F10C010A
:10BED0000069FFF7E7BF0000C36970B5044663B9A6
:10BEE00023493523234A2448F7F742F92348F7F733
:10BEF0003FF935211F48F7F748F904F10805D5E85F
:10BF0000AF3FDB072FD50021E269136813B96FF04B
:10BF1000150070BD9C4221D12368566823F00300B0
:10BF200091B9B442106000D15060236803F003035C
:10BF300023600020E061D5E8EF3F23F00103C5E86E
:10BF4000E23F002AE5D0F6E70B68B44203F00303B2
:10BF500043EA00030B6008BF5160E6E71868194622
:10BF600020F00303D2E704F10C0000F09FF9E0E7B2
:10BF7000A51F0600651F0600170206003105060012
:10BF80002DE9F041054686B098460E461746FEF765
:10BF900013FC002005F11404CDE90400CDE90208EA
:10BFA000CDE900503146064B3A462046FFF7C2FE27
:10BFB0002046044906B0BDE8F041FFF707BE00BFC8
:10BFC000892D04005B1F06000023C0E90031C0E991
:10BFD00002330361C36170472DE9F84305460E46FD
:10BFE000914600F1C0074FF02003EFF3118883F36F
:10BFF00011883846FFF72EFE60B930494C23304A8D
:10C000003048F7F7B5F83048F7F7B2F84C212C482C
:10C01000F7F7BBF8F469D4B1AC424BD13046FFF727
:10C020005BFF041E15DA3846FFF726FE60B9274984
:10C030005C23234A2348F7F79BF82548F7F798F83D
:10C040005C211F48F7F7A1F888F311881DE0002D47
:10C05000E4D0F561B9F1000F1AD13846FFF70CFEB4
:10C0600060B91A495C23164A1648F7F781F8184850
:10C07000F7F77EF85C211248F7F787F888F3118804
:10C0800031462846FFF70EFF00242046BDE8F8831E
:10C090004FF4004500210F484FF4A0220023C5FBB8
:10C0A0000901F4F7CFFC0C49421C06F10C0000F02A
:10C0B0005DF8B8E76FF06F04B5E700BF371B060007
:10C0C000F41A0600170206004C1B0600611B06004E
:10C0D000781B0600FFFF0400CDBE0400034B1B6865
:10C0E0000BB9F7F7E3BA0020704700BF08620220DF
:10C0F00038B5104B1B78002B0F4B18BF4FF0FF309B
:10C100001C6808BF6FF000409C420AD04CB1A56883
:10C11000FFF7E4FF281A00280ADBA468FFF7DEFF18
:10C12000201A064B1B6913B19842A8BF184638BDA8
:10C130000020F6E70C6202204CBF0220FC600220C7
:10C14000036840B1084A5268904204D01BB19A6813
:10C1500081680A449A604268136003685A60002349
:10C16000C0E90033704700BF4CBF022003682DE9CF
:10C17000F04704460E46154663B140494D23404AF8
:10C180004048F6F7F5FF4048F6F7F2FF4D213C48EE
:10C19000F6F7FBFF012DB8BF0125E6604FF0200345
:10C1A000EFF3118883F311883848FFF753FD60B926
:10C1B00037494C23374A3348F6F7DAFF3648F6F763
:10C1C000D7FF4C213348F6F7E0FFFFF787FF334EE8
:10C1D00028443568A060B54248D0294FDFF8C8A090
:10C1E000DFF8A09040E0AB68002B0CDA51465623F4
:10C1F0003A464846F6F7BCFF2348F6F7B9FF562102
:10C200003846F6F7C2FFAA68A3689A4226DDD31A19
:10C21000AB606B68C4E900536B681C606C6033688A
:10C22000B34206D09C4204D1FFF762FF0021F7F72A
:10C23000F9F91648FFF720FD60B919495C23154A42
:10C240001048F6F795FF1748F6F792FF5C21114862
:10C25000F6F79BFF88F31188BDE8F0879B1AA3606F
:10C260007368AB4202D02D68002DBCD17368266084
:10C27000636073681C607460D1E700BF0220060031
:10C28000C11F0600170206003105060018620220D1
:10C29000371B0600F41A06004C1B06004CBF022098
:10C2A000611B0600781B06002220060038B50446F4
:10C2B0004FF02003EFF3118583F311881748FFF740
:10C2C000C9FC60B916494C23164A1748F6F750FFC7
:10C2D0001648F6F74DFF4C211248F6F756FF236833
:10C2E00013B96FF0150403E02046FFF729FF00247F
:10C2F0000A48FFF7C1FC60B90D495C23094A0A48A6
:10C30000F6F736FF0B48F6F733FF5C210548F6F7E2
:10C310003CFF85F31188204638BD00BF186202201B
:10C32000371B0600F41A0600170206004C1B060015
:10C33000611B0600781B060038B54FF02003EFF3B1
:10C34000118583F311881448FFF784FC60B9134901
:10C350004C23134A1348F6F70BFF1348F6F708FF70
:10C360004C210F48F6F711FFFFF7C2FE04460A48BA
:10C37000FFF782FC60B90D495C23094A0948F6F7CA
:10C38000F7FE0B48F6F7F4FE5C210548F6F7FDFED4
:10C3900085F31188204638BD18620220371B06003D
:10C3A000F41A0600170206004C1B0600611B06006B
:10C3B000781B060070B504460D464FF02003EFF3DE
:10C3C000118683F311881748FFF744FC60B91649BA
:10C3D0004C23164A1648F6F7CBFE1648F6F7C8FE69
:10C3E0004C211248F6F7D1FEFFF782FEA04205DD90
:10C3F000012803DD29462046F7F714F90948FFF71D
:10C400003BFC60B90C495C23084A0948F6F7B0FECA
:10C410000A48F6F7ADFE5C210448F6F7B6FE86F34F
:10C42000118870BD18620220371B0600F41A06003E
:10C43000170206004C1B0600611B0600781B060055
:10C440002DE9F04B0446FEF7E3FE4FF02003EFF337
:10C45000118583F311884148FFF7FCFB60B940491F
:10C460004C23404A4048F6F783FE4048F6F780FEEA
:10C470004C213C48F6F789FE3D4F3E4EB946DFF869
:10C4800000813460D8F8004032684445D7E900BCE8
:10C4900005D024B1A368934223DD9B1AA360002436
:10C4A0001BEB02004CEBE271C9E900013460FFF7BD
:10C4B0001FFE2146F7F7B6F82848FFF7DDFB60B905
:10C4C0002D495C23274A2848F6F752FE2B48F6F7F9
:10C4D0004FFE5C212348F6F758FE85F31188BDE82E
:10C4E000F08B1BEB03004CEBE371D31A336000239A
:10C4F000C7E90001A3602046FFF722FE1748FFF7B7
:10C50000BBFB60B91C495C23164A1748F6F730FE9E
:10C510001A48F6F72DFE5C211248F6F736FE85F331
:10C520001188E368204698474FF02003EFF3118508
:10C5300083F311880948FFF78DFB0028A2D14C2313
:10C54000084A07490848F6F713FE0848F6F710FEB0
:10C550004C210448F6F719FE94E700BF1862022048
:10C56000371B0600F41A0600170206004C1B0600D3
:10C570001062022008620220611B0600781B060080
:10C580004CBF02202DE9F0414FF02003EFF311865C
:10C5900083F311881748FFF75DFB60B916494C23F8
:10C5A000164A1748F6F7E4FD1648F6F7E1FD4C2168
:10C5B0001248F6F7EAFDF7F779F8134BD3E900458F
:10C5C00027180C4845F10008FFF756FB60B90F49E2
:10C5D0005C230A4A0A48F6F7CBFD0D48F6F7C8FD7A
:10C5E0005C210648F6F7D1FD86F3118838464146AE
:10C5F000BDE8F08118620220371B0600F41A06001D
:10C60000170206004C1B060010620220611B060088
:10C61000781B060008B5FFF7B5FF08BD08B5FFF7A2
:10C62000F9FF4FF47A7164220023A0FB0101F4F7B3
:10C6300059FA08BD2DE9F84314240F46904604FB2F
:10C640000104414DDFF83C91404E002F01DABDE876
:10C65000F8830023A360637B03F00F03042B39D816
:10C66000DFE803F0452A03381C00236963B9384921
:10C6700096232A463046F6F77BFD3648F6F778FDD6
:10C6800096212846F6F781FD226882B363681A6016
:10C69000226853600023C4E9003328E02369002B9B
:10C6A000F2D12D499A232A463046F6F761FD2B48F0
:10C6B000F6F75EFD9A21E4E72369002BE4D12849CF
:10C6C0009E232A463046F6F753FD2648F6F750FDDE
:10C6D0009E21D6E74946A5232A463046F6F748FD6F
:10C6E0002148F6F745FDA5212846F6F74EFD1F48DF
:10C6F000FFF7C2FA60B91E495C231E4A3046F6F7BE
:10C7000037FD1D48F6F734FD5C211A48F6F73DFD6C
:10C7100088F311884FF02003EFF3118883F3118819
:10C720001248FFF797FA60B914494C23114A304672
:10C73000F6F71EFD1248F6F71BFD4C210D48F6F7E3
:10C7400024FD013F143C80E79120060017020600FB
:10C75000CF200600E9200600FE2006001A21060070
:10C760002B210600482106005F2106001C620220E2
:10C77000611B0600F41A0600781B0600371B060032
:10C780004C1B0600B41D0600836870B505460E46B6
:10C7900053B31C6874B91B4940F25B131A4A1B4817
:10C7A000F6F7E6FC1A48F6F7E3FC40F25B11164890
:10C7B000F6F7EBFC0022AB681A71637B9A0713D57E
:10C7C000236A02331AD02046FEF7C0FA082E0CBFA7
:10C7D0006FF003030023A366637BDB0604D1A36928
:10C7E00013B92046FEF7B8FB0020EB68A860C3F33E
:10C7F0000432164366F31033EB6070BD6FF00A002D
:10C80000FBE700BF1C22060091200600170206006D
:10C8100041220600F8B51746D0E9002390420446AD
:10C820000D4606D163682C606B6063681D606560AF
:10C8300019E0002BF6D09B6839681868FEF7ECF811
:10C840000028EFD12668B442ECD0002EEAD0B368BD
:10C8500038681968FEF7E0F830B17368C5E900631D
:10C8600073681D607560F8BD63689E42DAD03668F3
:10C87000EBE70000F8B504460F461D46164662B1C8
:10C880001F492A231F4A2048F6F772FC1F48F6F773
:10C890006FFC2A211B48F6F778FC0F2F0CD91C4996
:10C8A0002B23184A1848F6F763FC1A48F6F760FC81
:10C8B0002B211448F6F769FC65B917492C23114A56
:10C8C0001148F6F755FC1548F6F752FC2C210D4897
:10C8D000F6F75BFC0022637BA26067F303036373DC
:10C8E000E368256162F31033E360C3F3074366F343
:10C8F0004103A373E38962F38F03E381F8BD00BFB3
:10C9000075210600912006001702060095210600F9
:10C91000BB210600DF210600EF21060002220600EF
:10C920002DE9F04F054687B08A469046EFF3058320
:10C930000D2B04D883B19F4B5B681B050CD49E491B
:10C94000C1239E4A9E48F6F713FC9E48F6F710FC5A
:10C95000C1219A48F6F719FC65B99B49C223974A49
:10C960009748F6F705FC9948F6F702FCC221934870
:10C97000F6F70BFCBAF1000F0CDC9549C3238F4A84
:10C980008F48F6F7F5FB9348F6F7F2FBC3218B4887
:10C99000F6F7FBFB904B2C469B684FF00009029387
:10C9A00001234FF0FF36DFF838B28C4F8DF80C3092
:10C9B000D14538DB4FF02003EFF3118483F3118866
:10C9C0008748FFF747F960B986494C23834A7C487A
:10C9D000F6F7CEFB8448F6F7CBFB4C217F48F6F701
:10C9E000D4FB9DF80C30002B40F0168128462246DF
:10C9F0003146FFF71FFE7A48FFF73EF960B97B49E1
:10CA00005C23764A6E48F6F7B3FB7948F6F7B0FB3D
:10CA10005C217248F6F7B9FB84F3118800242046A4
:10CA200007B0BDE8F08F4FF02003EFF3118283F3DE
:10CA3000118858460192FFF70DF960B969494C23F6
:10CA40003A465F48F6F794FB6748F6F791FB4C21AE
:10CA50003846F6F79AFB637B03F00F03042B26D8C6
:10CA6000DFE803F0071F0325190023699B68002BEB
:10CA70002ED1B8F1000F37D09DF80C30002B33D0F9
:10CA8000637B03F00F03042B00F28680DFE803F0E2
:10CA9000597144845D0023691B68002BE9D004228E
:10CAA00017E023699B68002BE3D0012211E050239B
:10CAB000424A50494248F6F75BFB617B4E4801F021
:10CAC0000F01F6F755FB50213C48F6F75EFBD0E727
:10CAD00002220021E368A160C3F30430024362F341
:10CAE0001033E3608DF80C105846FFF7C5F860B9B5
:10CAF0003E495C233A463248F6F73AFB3C48F6F7A3
:10CB000037FB5C213846F6F740FB019B83F3118825
:10CB100009F1010914344BE7236963B937497523D7
:10CB2000264A2748F6F724FB3548F6F721FB7521FE
:10CB30002248F6F72AFB2146206902AA1030FFF7A7
:10CB400069FE02ABA3600136CEE7236963B92D49C4
:10CB500079231A4A1A48F6F70BFB2B48F6F708FB1D
:10CB600079211648F6F711FB206902AA21460C30FC
:10CB7000E5E7236963B925497D23104A1048F6F794
:10CB8000F7FA2348F6F7F4FA7D210C48F6F7FDFA98
:10CB900002AA21462069D2E78423084A1549084899
:10CBA000F6F7E6FA1B48F6F7E3FA84210348F6F7AE
:10CBB000ECFAC6E700ED00E0371D06009120060004
:10CBC0001702060031050600312006004720060046
:10CBD0005620060065200600FC600220F41A0600BC
:10CBE0001C620220371B06004C1B0600611B06005E
:10CBF000781B0600B41D060074200600CF20060036
:10CC0000E9200600FE2006001A2106002B2106005E
:10CC1000482106005F21060000238DF80C30B8F192
:10CC2000000F15D12748FFF727F860B926495C2384
:10CC3000264A2748F6F79CFA2648F6F799FA5C2127
:10CC40002248F6F7A2FA84F311886FF00A04E6E6A8
:10CC500004AA214643461B48CDE90422FEF7CAFB3D
:10CC600004464FF02003EFF3118783F31188154832
:10CC7000FEF7F0FF60B918494C23144A1448F6F740
:10CC800077FA1648F6F774FA4C211048F6F77DFA51
:10CC900028463A463146FFF7CDFC0A48FEF7ECFF3E
:10CCA00060B909495C23094A0948F6F761FA09485D
:10CCB000F6F75EFA5C210548F6F767FA87F3118804
:10CCC000ADE600BF1C620220611B0600F41A0600DC
:10CCD00017020600781B0600371B06004C1B0600D7
:10CCE000036898420AD0D3E90002106018684260D5
:10CCF00000221846C3E90022FFF746BD704770477F
:10CD000051EC100B2C4A21F00043934200B585B042
:10CD100020DD2A4A934209DD10EE102A0B46F3F774
:10CD200017FA41EC100B05B05DF804FB684600F003
:10CD30003BF900F00300012817D002282FD028B3B8
:10CD400001209DED021B9DED000B01F0BDF851ECA3
:10CD5000100BE6E79FED161B00F052FB51EC100B99
:10CD600041EC100B05B05DF804FB9DED021B9DED41
:10CD7000000B01F0A9F810EE100A53EC102B03F190
:10CD8000004141EC100B05B05DF804FB9DED021B6A
:10CD90009DED000B00F034FB51EC100BC1E79DED55
:10CDA000021B9DED000B00F02BFBE4E7AFF30080CE
:10CDB0000000000000000000FB21E93FFFFFEF7FC3
:10CDC00051EC100B10EE102A21F0004343EC102B15
:10CDD000704700BF0000000051EC100BC1F30A5374
:10CDE0002DE9F041A3F2FF350C4610EE106A0F4614
:10CDF000132D1DDC002D3DDB394B43FA05F801EA0C
:10CE00000803034319D034A3D3E90023F3F7A2F9AD
:10CE100000220023F3F7E4FDD0B3002C04DA4FF432
:10CE2000801343FA05F52F4427EA080400262FE073
:10CE3000332D06DDB5F5806F30D041EC100BBDE829
:10CE4000F081A3F213434FF0FF3828FA03F818EAF1
:10CE5000000FF2D020A3D3E90023F3F77BF90022DF
:10CE60000023F3F7BDFD98B1002C28DB26EA080665
:10CE70003C460DE018A3D3E90023F3F76BF9002239
:10CE80000023F3F7ADFD18B1002C0FDB002634466C
:10CE90002346324643EC102BBDE8F08110EE102AF9
:10CEA0000B46F3F757F941EC100BC8E724F00043A9
:10CEB0000C4A33430026B34218BF1446E8E7142D4A
:10CEC00008D00123C5F1340503FA05F5AE1928BFD2
:10CED000FF18CBE70137C9E79C7500883CE4377E33
:10CEE000FFFF0F000000F0BF51EC100B2C4A21F0A7
:10CEF0000043934200B585B027DD2A4A934209DDFD
:10CF000010EE102A0B46F3F723F941EC100B05B095
:10CF10005DF804FB684600F047F800F003000128C4
:10CF20001FD0022830D028B39DED021B9DED000BD1
:10CF300000F066FA10EE100A53EC102B03F10041DA
:10CF400041EC100B05B05DF804FB00209FED121BB7
:10CF500000F0BAFF51EC100B41EC100B05B05DF87E
:10CF600004FB9DED021B9DED000B00F049FA51EC16
:10CF7000100BCAE701209DED021B9DED000B00F098
:10CF8000A3FF51EC100BC0E701209DED021B9DEDAE
:10CF9000000B00F099FFCDE700000000000000004A
:10CFA000FB21E93FFFFFEF7F53EC102B2DE9F0470A
:10CFB000BF4923F0004790B08F4240F39380BD49B2
:10CFC0001C4682468F4229DC002C194610EE100ABE
:10CFD000ADA3D3E9002340F39080F3F7B9F8B64B43
:10CFE000804689469F4200F073810125A8A3D3E9BA
:10CFF0000023F3F7ADF802460B4640464946CAE91E
:10D000000023F3F7A5F8A2A3D3E90023F3F7A0F8D0
:10D01000CAE90201284610B0BDE8F087A7498F424F
:10D0200040F38A80A6498F4200F320813D1510EE1F
:10D03000100A1646A5F21645A7EB05510F46F3F761
:10D04000D9FCF3F7D3F98046894602460B463046B1
:10D050003946CDE90A89F3F77BF80022994BF3F7BB
:10D060002FFA89468046F3F7C5FCF3F7BFF9064669
:10D070000F4602460B4640464946CDE90C67F3F79A
:10D0800067F800228F4BF3F71BFA00220023CDE94B
:10D090000E01F3F77DFC002800F065810023304687
:10D0A00039460022F3F774FC002814BF0123022341
:10D0B000854902202A460191514600900AA800F0B5
:10D0C000E3FA002C054614DADAF804204542DAF8CF
:10D0D0000C3002F1004203F10043CAF80420CAF800
:10D0E0000C3006E000260027002580ED000BC0E98B
:10D0F0000267284610B0BDE8F087F3F72BF86E4BB7
:10D10000804689469F4200F010814FF0FF3560A3B2
:10D11000D3E90023F3F71EF802460B464046494682
:10D12000CAE90023F3F714F859A3D3E90023F3F76E
:10D1300011F8CAE90201DCE7FFF742FE10EE100A1F
:10D1400059EC108B54A3D3E900234946F3F7B8F9FF
:10D1500000225E4BF2F7FEFFF3F74CFC0546F3F7B7
:10D1600045F949A3D3E90023CDE90601F3F7A8F96E
:10D1700002460B4640464946F2F7EAFF804689469A
:10D1800043A3D3E90023DDE90601CDE90289F3F7E2
:10D1900097F91F2D02460B46CDE9042340F3B580D5
:10D1A000DDE90423DDE90201F2F7D2FF804689467A
:10D1B0003F15C9F30A53FB1A102B40F3B38038A371
:10D1C000D3E90023DDE90601F3F77AF980468946C1
:10D1D00002460B46DDE90201F2F7BAFF02460B46B2
:10D1E000DDE90201CDE90823F2F7B2FF42464B46E2
:10D1F000F2F7AEFF804689462BA3D3E90023DDE991
:10D200000601F3F75DF942464B46F2F7A1FF0B46E4
:10D210000246CDE90401DDE90801F2F799FFC1F307
:10D220000A5380468946FF1A312F00F39E809DEDF8
:10D23000087BCAE900898DED027B42464B46DDE959
:10D240000201F2F785FFDDE90423F2F781FF002CEC
:10D25000CAE90201BFF64DAF09F1004401F10043F4
:10D260006D42CAE90084CAE9020342E710EE100ADF
:10D270001946F2F76DFF0025CAE90201CAE900016B
:10D2800037E700BFAFF3008000004054FB21F93FB7
:10D290003163621A61B4D03D83C8C96D305FE43F29
:10D2A0000000601A61B4D03D7370032E8A19A33B4D
:10D2B000FB21E93F7BD90240FB21F93FFB213941AA
:10D2C000FFFFEF7F00007041E02206000000E03F1A
:10D2D00041A3D3E90023F2F73BFF0D46044640A3E8
:10D2E000D3E90023F2F734FF02460B4620462946D5
:10D2F0000125CAE90023F2F72BFF39A3D3E9002364
:10D30000F2F726FFCAE90201F3E640464946F2F782
:10D310001FFF394B6A1E8046894653F82230BB42B4
:10D320003FF446AFCAE9008987E72BA3D3E900237E
:10D33000F2F710FF0D46044629A3D3E90023F2F7C4
:10D3400009FF02460B46204629464FF0FF35CAE941
:10D350000023F2F7FDFE22A3D3E90023F2F7FAFE41
:10D36000CAE90201C5E60323A2E61FA3D3E900230D
:10D37000DDE90601F3F7A4F806460F4602460B4620
:10D38000DDE90801F2F7E4FE8046894602460B46D5
:10D39000DDE90801CDE90289F2F7DAFE32463B46C3
:10D3A000F2F7D6FE06460F4611A3D3E90023DDE9C6
:10D3B0000601F3F785F832463B46F2F7C9FE02460E
:10D3C0000B4640464946CDE90423F2F7C1FE8046AC
:10D3D0008946A7E7AFF300800000601A61B4D03D32
:10D3E0007370032E8A19A33B0000002E8A19A33BF9
:10D3F000C14920259A837B39602206000000000085
:10D400002DE9F04F57EC106B27F00049B9F1795F27
:10D410002DED028BB0EE418AF0EE618A83B072DAB4
:10D4200010EE100A3946F3F7E5FA002800F0ED8017
:10D4300032463B4630463946F3F742F804460D463D
:10D440007BA3D3E90023F3F73BF87BA3D3E90023C5
:10D45000F2F780FE22462B46F3F732F878A3D3E9A1
:10D460000023F2F775FE22462B46F3F729F876A340
:10D47000D3E90023F2F76EFE22462B46F3F720F89D
:10D4800073A3D3E90023F2F763FE22462B46F3F79A
:10D4900017F871A3D3E90023F2F75CFE22462B466E
:10D4A000F3F70EF882468B460022714B2046294640
:10D4B000F3F706F85246804689465B4620462946E1
:10D4C000F2F7FEFF04460D463046394653EC182B62
:10D4D000F2F7F6FF02460B4620462946F2F738FEE1
:10D4E00002460B4640464946F2F732FE02460B46DC
:10D4F00000206049F2F72CFE41EC100B03B0BDECAC
:10D50000028BBDE8F08F10EE102A10EE100A3B4699
:10D510003946F2F7D5FF04460D4645A3D3E900236B
:10D52000F2F7CEFF44A3D3E90023F2F713FE22461D
:10D530002B46F2F7C5FF42A3D3E90023F2F708FE1A
:10D5400022462B46F2F7BCFF3FA3D3E90023F2F7B4
:10D5500001FE22462B46F2F7B3FF3DA3D3E9002399
:10D56000F2F7F6FD22462B46F2F7AAFF3AA3D3E9DB
:10D570000023F2F7EFFD2B462246F2F7A1FF3E4BC8
:10D5800082468B4699458FDD3C4B994544DC002211
:10D59000A9F500130020374990469946F2F7D8FDC7
:10D5A000CDE900010022324B20462946F2F788FFE0
:10D5B00042464B46F2F7CCFD5246804689465B46D2
:10D5C00020462946F2F77CFF04460D463046394690
:10D5D00053EC182BF2F774FF02460B4620462946FF
:10D5E000F2F7B6FD02460B4640464946F2F7B0FD5B
:10D5F00002460B46DDE90001F2F7AAFD41EC100BF3
:10D6000003B0BDEC028BBDE8F08F9FED150B03B0AE
:10D61000BDEC028BBDE8F08F9FED137B4FF000084F
:10D62000DFF85C908DED007BBCE700BFAFF30080BE
:10D63000D43888BEE9FAA8BDC4B1B4BD9EEE213E7F
:10D64000AD529C804F7E923E9015CB19A001FA3EC0
:10D650007751C1166CC1563F4C5555555555A53F90
:10D66000000000000000F03F000000000000E73F65
:10D670000000E03F0000F03F3233D33F0000E93FBD
:10D680000000D23F000000002DE9F04FADF5197DFC
:10D690001E46BF4C0793D31E0390013E84FB030438
:10D6A000DB170B91C3EBA403BA4DA29823EAE371F5
:10D6B000019655F820004B1C099104908F1BA3EB99
:10D6C000830302EBC303059383191AD43B440DF182
:10D6D0008008002400255E1CDDF88C9208E059F8D3
:10D6E00027000137F2F782FEB742E8E8020108D0CE
:10D6F000002FF4DA013720462946B742E8E8020154
:10D70000F6D1049B002B079B4FEAC303029329DB4E
:10D71000039A20A90DF5E07A02EB030801EB030957
:10D7200072AA049B02EBC30B019B002BC0F29C81ED
:10D730004D46039C0026002775E90223F4E8020108
:10D74000F2F7BEFE02460B4630463946F2F702FDBE
:10D75000444506460F46EFD109F10809EAE8026799
:10D76000DA45E1D10499DDE902208B008B460244C1
:10D770000BA89246A3F10802C31808930CAB1344FC
:10D780000A9398ABBBF1000F03EBCB0353E9284599
:10D7900029DD70AB0DF1300903EBCB0800227E4B85
:10D7A00020462946F2F78CFEF3F724F9F2F71EFE25
:10D7B00000227A4B06460F46F2F782FE02460B46DF
:10D7C00020462946F2F7C4FCF3F714F9394649F824
:10D7D000040B304678E90223F2F7BCFC70AB044638
:10D7E0000D469845DAD1DDF8149045EC104B4846CB
:10D7F00000F036FC00224FF07F5310EE100A55EC7B
:10D80000104B2946F2F75CFE41EC100BFFF7E4FAEF
:10D810000022634B51EC100BF2F752FE02460B460E
:10D8200020462946F2F794FC0D460446F3F7E2F849
:10D830008046F2F7DBFD0B46024629462046F2F70A
:10D8400087FC4B4606460F46002B40F3E1800BF168
:10D85000FF320CA9C9F11803C9F1170551F82210BC
:10D8600041FA03F000FA03F38044CB1A0CA943FAFF
:10D8700005F541F82230002D2CDDBBF1000F08F139
:10D88000010840F3A3820C9C002C40F0A780BBF160
:10D89000010F0AD00CA9012251F8044F531C002C8F
:10D8A00040F09E809B451A46F6D1059B002B0EDD6D
:10D8B000012B00F09881022B09D10BF1FF320CAB48
:10D8C0000CA953F82230C3F3150341F82230022D7E
:10D8D00000F0AF800022002330463946F3F758F8B5
:10D8E000002800F075820BF1FF39049B4B4510DCDA
:10D8F0006FF040430CA9002208985B4401EB8303BE
:10D9000053F80419834242EA0102F9D1002A40F097
:10D91000B580049B0CAA013B52F82330002B40F049
:10D92000A1800A9A012352F8041901330029FAD080
:10D9300003EB0B020BF101099145069248DC0999B2
:10D940006FF04048079809EB010300EB0B0501EB72
:10D95000020B984420AB03EBC505A39B03EB88089F
:10D9600070AB03EBC909A39B03EB8B03029358F83D
:10D97000040F05F1080BF2F739FD0B460199024639
:10D980000029C5E9002326DB039C002600270BE0C5
:10D99000ABAAAA2A282406000000703E00007041AD
:10D9A0000000204075E90223F4E80201F2F788FD47
:10D9B00002460B4630463946F2F7CCFB5445064644
:10D9C0000F46EFD1029B5D469845E9E80267CED14C
:10D9D000DDF818B0D5E600260027F3E70123002282
:10D9E000C4F180740CA99B4541F822400EDD51F82A
:10D9F000232001EB8B0001EB83036FF07F4100E0FC
:10DA00001A688A1A43F8042B8342F9D101244CE79F
:10DA100006D10BF1FF330CAA52F82350ED152AE77B
:10DA20000022C34BF2F7D2FF002840F0BB8105462D
:10DA300050E732463B460020BE49F2F789FB0646D6
:10DA40000F46002C3FF446AF05989FEDB50B00F054
:10DA500007FB3046394653EC102BF2F779FB0646AC
:10DA60000F4637E7012363E70026002709F108097D
:10DA7000EAE80267DA457FF457AE73E6059A0CAB25
:10DA8000183A53F82930CDE9068505926BB96FF045
:10DA900040430CA94B4401EB830353F8041909F1EB
:10DAA000FF39183A0029F8D0059205989FED9C0B94
:10DAB00000F0D6FAB9F1000F55EC104BC0F2E68138
:10DAC0000CAA4FEAC9034FF0000ADFF86CB202EB70
:10DAD000890670AA089302EB0308043608F10807C8
:10DAE00056F8040DF2F782FC22462B46F2F7E8FCCA
:10DAF0005B46524667E9020120462946F2F7E0FC00
:10DB00000CAB04460D469E42EAD148AB09F1010236
:10DB1000CDF81490C3464FF0000ADDF8109003933F
:10DB200002920193B9F1000FC0F24D81DFF80C822F
:10DB30005D460024002600277BA3D3E9002303E0F1
:10DB4000544510DCF8E802230134F5E80201F2F74D
:10DB5000B7FC02460B4630463946F2F7FBFAA145C0
:10DB600006460F46ECDA019B0AF1010AABF1080BFD
:10DB7000E3E802670193029B9A45D3D1A29BDDF8AB
:10DB80001490032B28D8DFE813F0F200DD00DD004D
:10DB90003B00079B00200021002B40F055810B9B90
:10DBA0000246C3E900010B460399D1E90001F2F7EF
:10DBB000CFFAB9F1000F0CDD4AAD01240134F5E8CC
:10DBC0000223F2F7C7FAA145F8DA079B002B40F0D1
:10DBD0004B810B9BC3E90201069B03F007000DF587
:10DBE000197DBDE8F08F0BF1FF320CAB0CA953F897
:10DBF0002230C3F3160341F8223068E648AB0393A2
:10DC0000B9F1000F40F35581039B4FEAC9016FF052
:10DC10006040CDF8109003EBC9081A46029109EB59
:10DC2000000191460191D8E900AB78E902675246BC
:10DC30005B4630463946F2F78DFA04460D460246F9
:10DC40000B4630463946F2F783FA52465B46A24607
:10DC5000F2F780FAC145AB46C8E90201C8E90045C0
:10DC6000E3D1DDF81090B9F1010F40F32281019B5F
:10DC70000DF5947BDA00DDE9023102F1080A019228
:10DC80000B448A44D3E900677AE9028932463B466D
:10DC900040464946F2F75EFA04460D4602460B46F8
:10DCA00040464946F2F754FA32463B462646F2F7DA
:10DCB00051FAD3452F46CAE90201CAE90045E3D12A
:10DCC000019C0020039B0021103403F110051C442B
:10DCD00074E90223F2F73EFAA542F9D1039C079EAC
:10DCE000D4E90023D4E90245002E00F0C18003F1FD
:10DCF000004701F100430B992646944605F1004484
:10DD0000C1E90403069B03F00700C1E900C7C1E9AC
:10DD100002640DF5197DBDE8F08F00BFAFF3008000
:10DD2000000000000000F03F00000040FB21F93F30
:10DD30000000E03F0000F03F0000703EF0230600CE
:10DD400048AB0393B9F1000FFFF623AF039D00200A
:10DD5000002105EBC904083474E90223F2F7FAF94B
:10DD6000A542F9D1079B002B3FF419AF6CE0089C4A
:10DD70000020039D002108342C4474E90223F2F7AB
:10DD8000E9F9A542F9D1079B13B101F10043194606
:10DD90000B9BC3E90001069B03F007000DF5197DFD
:10DDA000BDE8F08FBBF1000F08F101084FF002054C
:10DDB0003FF769AD32463B4600203F49F2F7C8F9CC
:10DDC00006460F4686E500260027CCE600246CE5D3
:10DDD000059C47EC106B6042CDE9068500F040F9E8
:10DDE000002210EE100A354B57EC106B3946F2F753
:10DDF000EDFD00B318340022314B3046394605940E
:10DE0000F2F75EFB0BF10109F2F7F4FD0446F2F7BD
:10DE1000EDFA0022294BF2F753FB0B460246394636
:10DE20003046F2F795F9F2F7E5FD0CAB43F82B001D
:10DE300043F8294039E630463946F2F7DBFD0CABB2
:10DE4000D94643F82B0030E601F100430B9C024613
:10DE5000C4E900030B460399D1E90001F2F778F910
:10DE6000B9F1000F3FF7A8AE01F100431946B0E643
:10DE70000B9EC6E90023069BC6E9040103F00700D8
:10DE8000C6E902450DF5197DBDE8F08FA29B032B75
:10DE90003FF6A2AE01A252F823F000BFADDE0400AF
:10DEA00041DD040041DD0400FDDB04000020002111
:10DEB00069E70020002111E70000F03F00007041F9
:10DEC0000000703E000000002DE9F04F55EC104BB3
:10DED00025F000438246B3F1795F2DED028BB0EE61
:10DEE000418AF0EE618A83B007DA10EE100A294603
:10DEF000F2F780FD002800F08E8022462B46204657
:10DF00002946F2F7DDFA06460F4602460B46204642
:10DF10002946F2F7D5FA804689463046394645A368
:10DF2000D3E90023F2F7CCFA44A3D3E90023F2F7B4
:10DF30000FF932463B46F2F7C3FA42A3D3E9002376
:10DF4000F2F708F932463B46F2F7BAFA3FA3D3E9B3
:10DF50000023F2F7FDF832463B46F2F7B1FA3DA353
:10DF6000D3E90023F2F7F6F8CDE90001BAF1000F8A
:10DF700037D000222E4B51EC180BF2F7A1FA824653
:10DF80008B4640464946DDE90023F2F799FA0246FE
:10DF90000B4650465946F2F7DBF832463B46F2F75D
:10DFA0008FFA53EC182BF2F7D3F806460F4640468B
:10DFB00049461DA3D3E90023F2F782FA02460B4635
:10DFC00030463946F2F7C6F802460B462046294647
:10DFD000F2F7BEF841EC100B03B0BDEC028BBDE8CC
:10DFE000F08F02460B4630463946F2F769FA0EA327
:10DFF000D3E90023F2F7ACF842464B46F2F760FA59
:10E0000022462B46F2F7A6F841EC100B03B0BDEC0C
:10E01000028BBDE8F08F45EC104B03B0BDEC028BDA
:10E02000BDE8F08FAFF30080495555555555C53FB4
:10E030000000E03F7CD5CF5A3AD9E53DEB9C2B8AD6
:10E04000E6E55A3E7DFEB157E31DC73ED561C119D5
:10E05000A0012A3FA6F810111111813F0000000015
:10E0600038B553EC102BC3F30A511C46054619BBB7
:10E0700023F0004410EE101A21431CD0384C1946EE
:10E080000022384B10EE100AF2F71AFAA5420246A7
:10E090000B4634DB0C46C1F30A513639294440F2B1
:10E0A000FE70814233DC002912DD2F48204040EA17
:10E0B000015343EC102B38BD40F2FF708142EDD18B
:10E0C00010EE100A1946F2F745F841EC100B38BD76
:10E0D00011F1350F1EDA4CF250318D4243EC112B09
:10E0E00026DD9FED1B0B00F043F819A3D3E90023B5
:10E0F00051EC100BF2F7E4F941EC100B38BD16A30C
:10E10000D3E90023F2F7DCF941EC100B38BD43EC06
:10E11000112BE6E714483631204040EA01531046FF
:10E1200000221946114BF2F7CBF941EC100B38BD28
:10E130009FED090B00F01CF807A3D3E9002351EC75
:10E14000100BF2F7BDF941EC100B38BDAFF30080B6
:10E150009C7500883CE4377E59F3F8C21F6EA50118
:10E16000B03CFFFF00005043FFFF0F800000903CD9
:10E1700011EE900A53EC102B00F0004023F0004108
:10E1800041EA000343EC102B704700BF0A4C1D46C8
:10E190000646236800B5D86885B052B1074C029294
:10E1A00033462A4600910194054900F00DF803F02A
:10E1B0008BFA044C2246F2E754BF022038240600B2
:10E1C000482406003C2B06000EB410B583B0074B64
:10E1D000014605AC186854F8042B2346019402F05C
:10E1E00023FB03B0BDE8104003B0704754BF0220CA
:10E1F000044B054A1B685B6B002B08BF134693F862
:10E200002801704754BF022080C30220044B054AF6
:10E210001B685B6B002B08BF1346D3F8EC007047FC
:10E2200054BF022080C30220024B0146186800F050
:10E230000BB800BF54BF0220024B0146186804F01F
:10E240005FBC00BF54BF02202DE9F04F01F10B0568
:10E2500083B00646162D24D8102900F2D18000F094
:10E2600091FB102518220224CA4F3A445368A2F1A8
:10E2700008018B4200F087815A6803F10809D968C8
:10E28000304622F003029D681344E9608D605A68AD
:10E2900042F001025A6000F07BFB484603B0BDE843
:10E2A000F08F35F0070500F1AB80A94200F2A8809D
:10E2B00000F068FBB5F5FC7FC0F092816B0A0BD0D3
:10E2C000042B40F29680142B00F2C78103F15C040A
:10E2D00003F15B0CE30004E04FF4007340244FF0C3
:10E2E0003F0CAC4F3B44A3F108005B68984206D159
:10E2F0000CE0002980F23581DB68984206D05A682C
:10E3000022F00302511B0F29F3DD64463A69DFF85E
:10E310009CC262457CD0536823F00303591B0F292C
:10E3200000F348810029C7E904CC54DAB3F5007F33
:10E3300080F07281DB080121981003EB010E81400F
:10E3400007EBCE08786857F83E300143A8F1080083
:10E350009360D060796047F83E20DA60A310012016
:10E36000984088425AD8084205D124F0030440005E
:10E3700004340842FBD007EBC409A046CE46DEF8C1
:10E380000C309E4507D12FE1002A80F23681DB68F0
:10E390009E4500F02981596821F003014A1B0F2A8C
:10E3A000F2DDD3F80CE045F0010442F001081D4411
:10E3B00030469E685C6003F10809C6F80CE0CEF8B0
:10E3C0000860C7E90455C5E902CCC5F804805A5075
:10E3D00000F0DEFA61E7134402F1080930465A689A
:10E3E00042F001025A6000F0D3FA484603B0BDE89B
:10E3F000F08FAB0903F1390403F1380CE30070E747
:10E400004FF000090C234846336003B0BDE8F08F9D
:10E41000A3100120796898408842A4D9D7F80890C1
:10E42000D9F8043023F00308A8EB05020F2A13DD06
:10E43000A84511D345F0010342F001024D4409F112
:10E44000080949F8043C3046BD606A6000F0A0FA53
:10E45000484603B0BDE8F08FDFF854B14E4BDBF80F
:10E4600000201B6801322B4400F0358141F20F027D
:10E470004A4C1A4414402146304600F0B5FAB0F137
:10E48000FF3F824600F0F78009EB0800504500F29C
:10E49000F080434B1A6822441A6000F03381DBF8A5
:10E4A0000010013100F04C81AAEB000002441A6018
:10E4B0001AF0070200F01B81C2F1080041F20801C6
:10E4C0008244891A544430460193C4F30B028C1AD7
:10E4D000214600F089FA431C019B00F02E81A0EB3D
:10E4E0000A01214441F001011A68B945C7F808A0A2
:10E4F0002244CAF804101A6017D0B8F10F0F40F286
:10E500001881D9F80400A8F10C014FF0050C21F096
:10E51000070100F0010009EB010408430F29C9F8C5
:10E520000400C4E901CC00F222811E4B1E48196888
:10E53000D7F808908A42016888BF1A608A42D9F8E1
:10E54000043088BF026023F003035A1B0F2A02DD48
:10E550009D427FF66FAF30464FF0000900F018FA89
:10E560009BE61A4403F1080930465168D3E9027565
:10E5700041F00101FD60AF60516000F009FA4846CA
:10E5800003B0BDE8F08FD3689A427FF475AE0234D1
:10E59000BCE600BFECC402205062022000F0FFFF86
:10E5A00020620220486202204C620220F4C4022051
:10E5B000F4C8022045F0010441F0010E154402F1B7
:10E5C000080954603046C7E90455C5E902CCC5F8CE
:10E5D00004E0D15000F0DCF9484603B0BDE8F08F0C
:10E5E000EC0805F108023FE608F101080EF1080EFB
:10E5F00018F0030F7FF4C3AE55E01944DA6899466A
:10E6000030464B6859F8085F43F001034B60EA60FD
:10E61000956000F0BDF940E6590A042932D9142961
:10E6200068D801F15C005B31C00007EB000E385880
:10E63000AEF1080E864551D0416821F003019942A0
:10E6400002D980688645F7D1D0F80CE07968C2E934
:10E65000020ECEF80820C26080E6542B18D9B3F51C
:10E66000AA7F5BD8EB0B03F1780403F1770CE3008E
